:1000000000400020A9710000E9710000EB710000C0
:1000100000000000000000000000000000000000E0
:10002000000000000000000000000000ED71000072
:100030000000000000000000EF710000F1710000FE
:10004000F3710000D152000025760000F37100002A
:10005000F371000000000000F3710000F371000074
:10006000F3710000FD790000D1310000F371000050
:10007000F3710000F3710000F3710000F3710000F0
:10008000F3710000A9760000F3710000F371000025
:10009000F3710000F3710000F3710000F3710000D0
:1000A000F3710000F3710000000000000000000088
:1000B0000000000000000000000000000000000040
:1000C00010B5064C2378002B07D1054B002B02D02E
:1000D000044800E000BF0123237010BD6802002027
:1000E0000000000098E50000044B10B5002B03D081
:1000F0000349044800E000BF10BDC04600000000F6
:100100006C02002098E50000164B002B00D1144B28
:100110009D46402292029A1A924600218B460F4633
:100120001348144A121A0BF0B5FA0F4B002B00D0EB
:1001300098470E4B002B00D0984700200021040068
:100140000D000D48002802D00C4800E000BF0BF065
:1001500061FA2000290007F0B7FA0BF035FAC04623
:100160000000080000400020000000000000000027
:1001700068020020C82F00200000000000000000DE
:1001800002000120104011D1042A0ED91368180969
:1001900080B2002809D001388000031D11180979A8
:1001A000002902D001309842F8D170470020FCE7C6
:1001B0000378002B03D05AB2002A01DB01307047CC
:1001C0003F229343C03B59424B41C01803789343AD
:1001D000802BF4D10130F9E710B500240378002B0F
:1001E00001D1200010BDFFF7E3FF0134F6E770B541
:1001F000002204000D00411C092003F013FB00281D
:1002000006D001236200134343600023A34200DBB6
:1002100070BD9A00A958821891600133F6E770B555
:10022000012803DC1C2001F047F870BD01230D6894
:1002300011201D42F7D04868184206D1042804D97D
:100240000F2302681340042B01D00E20EBE703F0CC
:1002500047F96D100400002D03DDFFF7BDFFA84234
:1002600006DA1220DFE72000FFF7A2FF0400013DBD
:10027000012DF8D120787F2809DDDF280BDCF82359
:100280003F22DB00800118406378134018430123AC
:1002900040001843C9E7EF280BDCFC226378120109
:1002A0009B0113403F220007000C0343A07810403D
:1002B000ECE7F72812DCFC22637892021B03134060
:1002C000E0228004520310403F221843E378134099
:1002D000FC220343A07812018001E8E7012040429C
:1002E000D5E7F8B54D680F00EB0706D4042D04D907
:1002F0000F232E683340092B03D00B2000F0DCFFC6
:10030000F8BD6B683609B6B25C10731EA3420FD8F5
:100310000321200009F07AF86421642803DC01003D
:10032000032800DA03212800891903F0ADFA05003B
:100330002B6800201B099BB2013B9C42E0D23A682B
:10034000A31C9B005A510123013464001C436C60C0
:10035000D6E7F0B585B0012803DC1C2000F0ACFF27
:1003600012E001274B683A000093022806D08B6800
:100370003B4203D05F10002F00DC17000124009BDC
:10038000234203D00120404205B0F0BD009B042B66
:10039000F8D91B680D680F2619003140042921D1B6
:1003A000254205D1042D03D92B681E40042E01D00F
:1003B0000E20D3E70098FFF7E3FEB842E2DB009897
:1003C00003F08EF80600280003F08AF80100781E7A
:1003D00030180BF015FD0028D4D0801B01304000F0
:1003E0002043D1E709293DD1009B5B685B10019355
:1003F0009F42C7DC25422CD1042D2AD92B683340DB
:10040000042B26D1280003F06BF8039602907E1C83
:10041000009AB300D058854201D17800E0E720422D
:100420000ED104280CD90368039A1340042B07D17A
:1004300003F056F8010002980BF0ACFC0028ECD059
:10044000019B37009E42E2DD9CE71F00019B9F421B
:1004500098DC7B1C00999A008A58AA42F5D1780052
:100460000124BDE7032900D08CE71A0992B25B0F83
:1004700092000B40D31A01939F4200DD82E7254290
:1004800029D1042D27D92A681640032E19D1100925
:1004900080B2520F800032402C1D801A019B26181A
:1004A0001B1A0193009B781E0433019A904200DDD1
:1004B00068E722001918B2420FD316D1013040006C
:1004C000CEE7042E07D1280003F00AF80400280024
:1004D000FFF756FEE2E70F2040E70D78AC461578AF
:1004E000AC4502D101310132E5E70130DDE710B55D
:1004F00002F0DAFF43000120184310BDC30711D4F6
:1005000004280FD90F2302681340032B0AD1194086
:100510000133591AC0234907DB051940024B1A4021
:10052000114301607047C046FFFFFF9FF7B507000A
:100530000E001C20012F06DD4C68012322001A400A
:10054000009203D10D2000F0B7FE53E0022F02D03D
:100550008A681A42F6D0012335681D4200D0A9E00E
:10056000042D00D8A6E01C41002C00DC1C000F204C
:1005700029680840092828D16B685B100093022F76
:1005800005D0B368009A5B109A4200DD0093009B8F
:1005900001221D1B0135EB43DB171D40691C09209F
:1005A00003F040F9071E09D001236D001D4303002D
:1005B0003268083345600099A14201DA3800FEBD77
:1005C0000134A100515802C3F5E7042845D12800A1
:1005D00002F086FFFFF700FE0190022F04D0B368FF
:1005E0005B10984200DD0193019BA34204DA0020D6
:1005F00003F08AF90700E1E7280002F071FF070025
:10060000009BA34221DB2800009702F069FF050050
:100610003800FFF7CDFD019B01340700A342F7DA54
:10062000009BC41A200003F06FF9071EC6D002F029
:1006300057FF0190306802F053FF2200009B591BC6
:10064000411801980BF00AF8B8E73800FFF7B0FD41
:10065000009B070001330093D2E703282AD10B093E
:100660009BB2490F9B000140591A022F04D0B26877
:100670005210914200DD1100A14205DA0022032050
:10068000110003F0CFF8B5E703200E1B331DD91777
:100690000140C9188910002203F0C4F8071E00D1D8
:1006A0008CE7013631000334FFF728FF381D291984
:1006B0003200C7E7212046E7F8B5002805DC1C20FA
:1006C00000F0FAFD05002800F8BD01260C68264060
:1006D0000FD06410E343DB171C40E11C891000229B
:1006E000032003F09FF8051EEDD02100FFF706FF61
:1006F000E9E7042C01D80025E5E70F232268134021
:10070000042B1BD12000FFF73BFDC31C0700032077
:10071000D9170140C9188910320003F083F8051E6B
:10072000D1D03900FFF7EAFE200002F0D9FE2B1DE0
:1007300001003A0018000AF091FFC4E7092BDAD152
:100740000320636832005F10FB1CD9170140C918F1
:10075000891003F067F8051ECDD03900FFF7CEFEF3
:10076000FF20BE42AFDA0122B300E3189B681342B8
:1007700008D01341FF2B00DD0300D943C917AA1984
:100780000B4013710136ECE710B57F2902DC0170D4
:10079000013010BD1A4B99420CDC40238A115B4298
:1007A000134303703F230B4080214942194341709A
:1007B0000230EEE7134B994210DC20230A135B4210
:1007C00013433F24802203708B1152422340214067
:1007D00013430A43437082700330DAE70A4B9942AD
:1007E000D7DCF0230370603B4370113B8A11FF3B61
:1007F0001A4382703F2211401943C1700430C8E788
:10080000FF070000FFFF0000FF0F0100F0B50D0023
:1008100085B0002803DC1C2000F04EFD0DE00968C7
:100820000122080010400AD002AC11412000FFF75D
:10083000ABFF011B200003F073F804001AE0042949
:100840003FD90F230C682340092B3AD14B685B102A
:10085000019303239C46019B9A420EDD03F054F85A
:10086000041E07D02E68012502F03AFE2F00019BDE
:100870009D421DDD200005B0F0BD01329300CC5833
:100880000123234001D10D20C6E764107F2C0DDD2C
:100890000D4E0223B44209DD0C4E6346B44205DD21
:1008A00000270B4EE30FA6427B419B00C018D2E706
:1008B0000135AB00F1583942E5D04910FFF764FF2C
:1008C000D5E72120A8E7C046FF070000FFFF000092
:1008D000FF0F010010B504000120084010D10429C9
:1008E0000DD90F230A681340042B08D1080002F029
:1008F000F7FD010020000BF04DFA4342584110BDB6
:100900000020FCE7F7B50F00012803DC1C2000F0F5
:10091000D3FCFEBD01264D682E4006D1042D04D91E
:100920000F222B681A40092A01D00B20EFE76A68D2
:100930001B099BB25410A34200D85C1E39681E48A4
:10094000FFF7C8FF01230190002813D139681B4825
:10095000FFF7C0FF002811D0002C0DD00123621C2E
:10096000013C9C409200535123436B6004E00136EC
:10097000B200AB50B442FADA0020CAE73B680D205F
:10098000DA07C4D55B10002B11DD9C420FDB9B0006
:10099000A200291DEB1889180433994209D10123BB
:1009A000013C9C40AA181C4353606C60E4E7122091
:1009B000ADE758681860EFE727CD00002BCD0000A9
:1009C000002310B50C000B70C30705D50D4942106C
:1009D00020000BF0A3F908E00B49002802D00428FE
:1009E00004D10A4920000BF0B9F910BD0428FCD944
:1009F0000F2302681340042BF7D102F071FD044964
:100A00000200E5E724D7000030CD000036CD00001D
:100A10003BCD0000F0B593B0060002911C20012EE2
:100A20001DDD029B01251B681C002C4000D0ADE0A1
:100A3000042B00D8E6E01A680F231A40092A4AD18D
:100A40000394039A029992008A5817002F4005D107
:100A5000042A03D910681840092806D0222000F083
:100A60002BFC0190019813B0F0BD52685210A418ED
:100A7000039A013203929642E3D1611C012202F0F3
:100A8000D1FE0190002802D100230193EAE7019BE7
:100A90006400190025435D600831029ABB00D058FC
:100AA00002684368120992B25B109A4200D8531E42
:100AB0000022934209DCDA43D21713409B00C91885
:100AC000039B01379F42E8DBCCE794000519AD6832
:100AD00001320D51EDE72700032A59D10193029A03
:100AE000BB00D3582B42B9D1042BB7D91868019950
:100AF0000140032939D1020992B2430F92000B4001
:100B0000D31A1C190137BE42E9D10320E31CD917BF
:100B10000140C9188910002202F084FE01900028CB
:100B2000B2D000252100FFF7E9FC019B1E1D029AAF
:100B3000AB00D45801231C421FD1042C1DD90F2116
:100B400023681940032918D1180980B25B0F80006F
:100B50000B40C01A0023834213DBC343DB1718404A
:100B600001353618BD42E2DB7CE7042900D075E789
:100B70001800FFF705FB2418C4E72000FFF700FB6F
:100B8000E8E7E2181279F2540133E4E700273C0069
:100B90000F25029ABB00D3580122134234D1042BF3
:100BA00032D9186801002940042935D11800FFF70F
:100BB000E7FA24180137BE42EBD1200002F0A4FE70
:100BC0000190002800D15FE7029FB600BB19041D09
:100BD000029301233D681D4229D1042D27D90F26F8
:100BE0002B681E40042E37D12800FFF7C9FA0600F3
:100BF000280002F075FC0100200032000AF02EFDF2
:100C0000A41922E02700C3E7180005A9FFF7D8FEC2
:100C100005A80BF0C9F8CCE7032900D01EE70209AC
:100C200092B2430F92000B40D31A1C19C2E705A9D8
:100C30002800FFF7C5FE05A80BF0B6F805A90500CA
:100C4000020020000AF00AFD6419029B0437BB422F
:100C5000BFD10023237005E7032EF6D11A0992B203
:100C60005B0F92001E40961B291DC5E7F0B50D00D5
:100C700095B0002806DC1C2000F01EFB04002000BC
:100C800015B0F0BD0C68012123000B40009306D184
:100C9000042C04D922680F331A40092A01D00B20F2
:100CA000EAE7626852100392002A03DC009802F01F
:100CB0002BFEE3E73F4A019201280BD06868084207
:100CC00008D1042806D902681340042B02D102F08F
:100CD00007FC019001980BF067F806000F27039BB3
:100CE0000834013B04935E43039B02909B001B1955
:100CF000059301232068184251D104284FD9036875
:100D00003B40042B52D1FFF73BFA059B04343618C5
:100D1000A342EED1300002F0F7FD041EAFD02B68E5
:100D20000593029B002B03D0686802F0D9FB019069
:100D3000200002F0D5FB0500009B059A9B00D3180C
:100D40009F68380002F0CCFB012306001F4201D14E
:100D5000042F04D807A93800FFF732FE07AE300091
:100D60000BF022F807000200310028000AF076FCA0
:100D7000029BED19002B0AD0049B009A934206DDDA
:100D80002800029A01990AF069FC029BED18009B69
:100D900001330093009A039B9342CDD16FE707A9DB
:100DA000FFF70EFE07A80AF0FFFFAEE702F098FB80
:100DB000F9E7C046C8D1000010B50024A04207DD05
:100DC0000B6801341C4003D05C10E343DB171C406C
:100DD000611C0122092002F025FD002803D0012317
:100DE00064001C43446010BD0A6870B51000012502
:100DF000284034D1042A32D90F24136849681C4092
:100E0000092C17D154681B099BB22C41A34200D86E
:100E10005C1E844205DC02200133984206DB002080
:100E20000FE085005519A9600130F2E784001151E7
:100E30000130F2E7032C12D1294203D1132000F034
:100E40003BFA70BD4910FF29F8D81B099BB2043248
:100E50009B00D3189342E2D911700132FAE70B20BC
:100E600000F02AFADBE700000123F7B500254E6801
:100E70000F0033400093AB420ED11D00042E0BD95E
:100E80000F2233681A40092A10D172681B099BB2DD
:100E90005510AB4200D85D1E3968CB0717D54C10F2
:100EA000002C01DDA5421DDA122032E0042A04D113
:100EB0003000FFF765F90500EEE7009D032AEBD14E
:100EC0001D09ADB25B0FAD001340ED1AE4E72E48EB
:100ED000FFF700FD002814D00AF0BCFE290008F03E
:100EE0007BFB4C1C009B002B4CD1042E4AD9326852
:100EF0000F331340092B10D10134A400A459200052
:100F0000FEBD39682148FFF7E5FC2C000028E9D137
:100F1000113000F0D1F90400F1E7042B2AD13000A0
:100F200002F0DEFA0500FFF757F9A042BCDB012C06
:100F30001ADC300002F0D4FA00902800FFF738F9EC
:100F4000461B300002F0E0FC041ED8D002F0C8FAC4
:100F50000190786802F0C4FA009B3200E91A411847
:100F600001980AF07BFBCAE72800FFF721F9013C52
:100F70000500DCE7032B05D13419E478023B64005B
:100F80001C43BCE70B20C4E720CD00002BCD0000A4
:100F9000F7B54D680F002A0001210A402FD1042D1A
:100FA0002DD90F242B68BE681C40092C14D1696808
:100FB0001B099BB24C100192A34200D85C1E3968F9
:100FC0002A48FFF787FC00282DD00F232A681340FA
:100FD000092B1DD1012317E0032C10D10E4203D1A0
:100FE000132000F069F9FEBD72100192FF2AF7D8B4
:100FF0001A0992B25B0F92001C40141BDFE70B2012
:10100000EFE701339A00AE509C42FADA0020EAE79B
:10101000032BFBD12B0001335A1BA242F6DC6A469C
:101020001279DA70F7E73968CB0706D5491000293D
:1010300001DD8C4209DA1220D3E70D48FFF74AFCA4
:101040002100002801D11130CBE70F232A6813407B
:10105000092B03D1013189004E51D7E7032BD5D19C
:101060006B461B796D18EB70D0E7C04627CD0000AA
:101070002BCD000010B50124086820421AD10428A5
:1010800018D90F2102681140092901D1406810BD0B
:10109000032908D113099BB2500F9B000840181A6E
:1010A00040002043F3E7042904D102F019FAFFF7C6
:1010B00093F8F5E70B2000F0FFF8E8E710B5034AD6
:1010C0000B21034804F0C6F910BDC046C8CC00008F
:1010D000C0CC0000002070470420704701207047FA
:1010E00010B5002002F010FC10BD00207047002059
:1010F0007047002070470020704700207047002094
:1011000070470020704700207047000010B5034A68
:101110000C21034804F09EF910BDC046B0CD00007C
:1011200010CE00007047000010B50124044002D02A
:101130004410200010BD042810D90F23026813406A
:10114000042B07D102F0CCF921000A220AF0F4FEA8
:101150000400EEE7032B01D10430F5E70D22014B2B
:101160001A70E6E7A8020020012210B5024018D14B
:10117000042802D903681A0992B201230B4012D144
:10118000042902D90B681B099BB20024934206D1A3
:1011900004309B000431C318984206D30124200078
:1011A00010BD0022E9E70023EFE704780A78002C5D
:1011B00001D1002AF2D0013001319442ECD0002458
:1011C000EDE70000F7B50700009101933049314B7E
:1011D000002A02D002220A70013A00261A601B6817
:1011E000CE54BE4200DBF7BD009AB300D058294B65
:1011F000274D1C68C8239B0065191C1B012318423E
:1012000006D0254A4310210028000AF055FD09E0C8
:10121000224A002802D004281BD1214A210028009C
:101220000AF04AFD1A4C20000AF0BEFD194A019B43
:101230001060002B0BD07B1EB34208DD194B984287
:1012400005D8431C1360202222540022E2540136A8
:10125000C7E7042819D90F2301680B40042B04D1D8
:1012600002F03EF9104A0300CDE7092B03D1436891
:101270000E4A5B10C7E7032B08D10A0992B2490F47
:1012800092000B40D31A0A4ABDE70123094ABAE784
:10129000A9020020CC05002024D7000030CD00009A
:1012A00036CD00001F0300004FDD000080D000009D
:1012B0008FD000009AD00000014B187000207047BA
:1012C000A802002070B501F06BFE094C0100251D3D
:1012D0001F2228000AF080FD28000AF065FD042383
:1012E00004308008000118432060200070BDC04613
:1012F00084020020C368F0B59D00836889B05D1941
:101300000300183306930369069A9F00069B029018
:10131000DF19436901939B00D3180393CD4B1B78CE
:10132000002B26D17F222B68CB491C1213409B0037
:101330005B58043501929F46029B587804F0B8FC34
:101340000023029A137027E0C24B1B78002B10D1A8
:101350002B68019A1C121340BF4A9B009B5804350E
:10136000E9E7069B3A1DD11ABA4BD82928DD1A2283
:101370001A70029BB74C9B6821780193EA1A029B72
:1013800092109B7812021A43029B587804F098FC42
:101390000023029A23701370029B069A9B680193A4
:1013A000ED1A029BAD10DD60069BFE1A029BB61083
:1013B0001E61039B9B1A029A9B10536109B0F0BDFA
:1013C0001B783C60002B01D01700D2E72B680199F5
:1013D0001C120B40A0499B005B5817000435AAE77C
:1013E000069B3A1DD11A9B4BD82902DD1A221A708E
:1013F000BFE728681B78291D3860002B02D0170032
:101400000D00B6E76B6801991C120B4092499B00D6
:101410005B58170008358EE7069B3A1DD11A8D4B95
:10142000D82902DD1A221A70A3E7A4001B782C1910
:101430003C60002B01D017009BE72B6801991C1220
:101440000B4085499B005B581700043573E7069BEA
:101450003A1DD11A7F4BD82902DD1A221A7088E76B
:101460007E49A40061581B783960002B01D0170019
:101470007FE72B6801991C120B4077499B005B5852
:101480001700043557E7043F744B3A68A400E25054
:10149000704B1B78002B00D06BE72B68019A1C1255
:1014A00013406D4A9B009B58043544E76B4BA400E6
:1014B000E058FFF739FE043F06003868FFF734FEB6
:1014C00036180120654B76000643E650614B1B78C9
:1014D000002B00D04DE72B68019A1C1213405E4A86
:1014E0009B009B58043526E7069B3A1DD11A594BA1
:1014F000D82902DD1A221A703BE70698039C0121C5
:10150000A04202D221000C3909681B783960002BF7
:1015100001D017002DE72B6801991C120B404E4992
:101520009B005B581700043505E7069B3A1DD11A4E
:10153000484BD82902DD1A221A701AE70699039837
:1015400081420FD203000C3B1B6845495B106418B5
:10155000E41AA40023583B603E4B1B78002B05D0B7
:10156000170006E7182119700023F4E72B6801998A
:101570001C120B4038499B005B5817000435DAE613
:10158000069B039A934219D213000C3B1B68344A02
:10159000043FA4185B10E31A039A39689B00995022
:1015A0002C4B1B78002B00D0E3E62B68019A1C1211
:1015B0001340294A9B009B580435BCE61822254B52
:1015C0001A70EDE7069B039A93422DD2244B3E1FDF
:1015D000E31814000C3C04932368049A5B10D31A9C
:1015E000039A9B009858FFF79FFD07903068FFF71C
:1015F0009BFD2468049B64101C1B079BA4001F1800
:1016000001207F00039B0743E7503700114B1B78F5
:10161000002B00D0ADE62B68019A1C1213400E4A35
:101620009B009B58043586E618220A4B1A70EDE79A
:10163000069B3A1DD11A074BD82902DD1A221A70CF
:1016400097E60399A40061581B783960002B09D0F4
:1016500017008EE6A802002080CE0000942D002006
:10166000FDFFFF3F2B6801991C120B40D8499B00DE
:101670005B58170004355EE6043F039B3A68A400FC
:10168000E250D44B1B78002B00D072E62B68019AF5
:101690001C121340CE4A9B009B5804354BE6039B1B
:1016A000A4001C192368043F38685E10FFF73CFD56
:1016B00036180120C74B76001B7806432660002BA6
:1016C00000D056E62B68019A1C121340C04A9B00BA
:1016D0009B5804352FE6069BA4003F1BBD4CBB4224
:1016E0000CD82378002B00D043E62B68019A1C12FB
:1016F0001340B74A9B009B5804351CE6B64801F0DE
:10170000DFFE2378002B00D033E62B68019A1C12F1
:101710001340AF4A9B009B5804350CE6A300ED181C
:10172000002C00DA38E6AB4B1B78002B00D020E60B
:101730002B68019A1C121340A54A9B009B58043544
:10174000F9E5043F3B68042B04D1A300ED18002CFD
:1017500000DA21E69F4B1B78002B00D009E62B68AE
:10176000019A1C1213409A4A9B009B580435E2E5EB
:10177000043F3B68042B04D0A300ED18002C00DAD2
:101780000AE6944B1B78002B00D0F2E52B68019AF7
:101790001C1213408E4A9B009B580435CBE53E1F1C
:1017A0003068C3070AD540100138002809DB01233F
:1017B0004000A40018432D193060EDE5FFF7B4FC9C
:1017C000F2E7844B37001B78002B00D0D1E52B6863
:1017D000019A1C1213407E4A9B009B580435AAE5CF
:1017E0003A00069B0C32D31AD82B03DD1A22794B10
:1017F0001A70BEE5FF2361005B001940FE3BFF3B12
:1018000019433960029906988968241204916D1A67
:101810000299AD1089782D020D4303999D40091A54
:10182000891099401D430B43BB60029B7D609C70F7
:10183000E4B26A4BE4000392E358029A9360654A6B
:101840001278002A03D008331D00039F91E51D0084
:10185000019A9B680C351C1213405D4A9B009B58F3
:10186000039F68E53B1F1C68039A069B93422DD19A
:101870000A20E3070CD4042C13D90F232268134049
:10188000042B11D1200001F02BFE0AF08DFA063056
:10189000643003F019FE00280FD1043D069B03932A
:1018A0007AE50720042CF3D02000431E9841FA2348
:1018B0004042FF3318400730EAE7029B2100587886
:1018C00004F010FA0023029A1370E7E7039B039ACF
:1018D0000C3B1B6802995B109B00D31A0C3B1C60ED
:1018E0001F1D1300083B1B685A108A70D2B23B4977
:1018F000D2005B0055589B0A029A9B009560ED1838
:10190000039B069A043B1B685B109B00D318039350
:10191000304B1B78002B00D02BE52B68019A1C1252
:1019200013402B4A9B009B58043504E53B1F186865
:10193000FFF7FAFBA40006003F1B1E2827DC002847
:101940000DDC244B1B78002B00D012E52B68019A8C
:101950001C1213401E4A9B009B580435EBE401F017
:101960000DFB033E361801F009FB1D4B801B98420E
:10197000F9D8184B1B78002B00D0FAE42B68019A99
:101980001C121340124A9B009B580435D3E40123D8
:10199000029A137001F0F2FA029B0A3886195E600F
:1019A000FAE43B1F1868FFF7BFFBA40006003F1BCB
:1019B000002817DC074B1B78002B00D0D9E42B68DC
:1019C000019A1C121340024A9B009B580435B2E452
:1019D00080CE0000A8020020ACD000009C25002092
:1019E0003F420F00D64B984203DD1D22D54B1A70A3
:1019F000BFE40123029A137001F0C0FAFA239B009E
:101A00005E43029B0A3E30185860C5E4A300FF1AEB
:101A1000002320001A003900FFF7D4FBCA4ECB4C3C
:101A20003168200001F07CFFC94B3168186020004C
:101A300003F0FAFF3168200004F05BF9C14B1B781A
:101A4000002B00D095E42B68019A1C121340C14A68
:101A50009B009B5804356EE4BA4BA4001B783F1BD7
:101A6000002B00D085E42B68019A1C121340B94A60
:101A70009B009B5804355EE4029803F089FDB14B4E
:101A80001B78002B00D074E42B68019A1C121340C1
:101A9000B04A9B009B5804354DE43B1F1B68002B4C
:101AA0003ED13B000C3B1B68DA072CD539000122E4
:101AB0005B105800083902430A60002B44DD012204
:101AC00059001143381F0160390008390968114174
:101AD000CB1A39000C390968114224D09B18934065
:101AE000A4001343039AA350964B1B78002B00D0FD
:101AF0003FE42B68019A1C121340964A9B009B58A6
:101B00000435FFF718FC042B06D90F211A680A4088
:101B1000092A01D15B68C9E719228A4B1A7028E4A7
:101B20005B10013BC9E7042909D90F200A6802406C
:101B3000092A04D102339B005B58A400D2E7192282
:101B4000804B1A70FFF715FC0435CDE7A300069A09
:101B5000FB189B1AD82B13DC0122631E002C14DC0B
:101B6000784B1B78002B01D0FFF703FC2B68019A00
:101B70001C121340774A9B009B580435FFF7DBFB90
:101B80001A22704B1A70FFF7F4FB3A601C000437FE
:101B9000E3E7069A3B1D9B1A6A4ED82B03DD1A23F6
:101BA0003370FFF7E6FB069B039AA40093422AD208
:101BB0003B1F1868FFF7B8FA011E21DD039B0C3BA1
:101BC0001A68521082421BDB9007801A624B401841
:101BD000C018039B8000C2583B1B1A60594B3F1B27
:101BE0001B780437002B01D0FFF7C3FB2B68019A49
:101BF0001C121340574A9B009B580435FFF79BFB70
:101C000020233370EAE71823FBE7514BA4001A683E
:101C10003B1B1F001A604B4B04371B78002B01D075
:101C2000FFF7A7FB2B68019A1C121340494A9B003F
:101C30009B580435FFF77FFB3B1F1A68042A11D11C
:101C4000A4002D193F4B1B78002B01D0FFF791FB0F
:101C50002B68019A1C1213403E4A9B009B58043586
:101C6000FFF769FB1F00EDE73A1F1368042B04D050
:101C7000002313603A00A4002D19324B1B78002B6F
:101C800002D01700FFF775FB2B6801991C120B405F
:101C900030499B005B5817000435FFF74CFBA3004D
:101CA0009C46FE1A002C17DC1C22264B1A700023BF
:101CB00033606346FF1A234B04371B78002B01D097
:101CC000FFF757FB2B68019A1C121340214A9B0017
:101CD0009B580435FFF72FFB002033685A10830010
:101CE000F15801230B4003D10D21164A1170DFE793
:101CF00049108A4200DD0A0001308442EFDC0123F2
:101D000052001343D4E7A3009C46FE1A002C25DCA6
:101D10001C220C4B1A70002333606346FF1A094BD8
:101D200004371B78002B01D0FFF723FB2B68019AA7
:101D30001C121340074A9B009B580435FFF7FBFA1F
:101D400080EE3600A8020020CC050020A902002069
:101D50000800002080CE0000FCFFFF3F0020336819
:101D60005A108300F15801230B4003D10D21E04AA2
:101D70001170D1E749108A4200DA0A00013084422A
:101D8000EFDC012352001343C6E73B00083B186811
:101D9000FFF7CAF93B1F06001868FFF7C5F90023D3
:101DA000864200DA0433A4003A1B17001360D04BBC
:101DB00004371B78002B01D0FFF7DBFA2B68019A60
:101DC0001C121340CB4A9B009B580435FFF7B3FA13
:101DD0003B00083B1868FFF7A7F93B1F060018688F
:101DE000FFF7A2F9F30FC217B0425341A4003A1B08
:101DF00017009B001360BE4B04371B78002B01D0EB
:101E0000FFF7B7FA2B68019A1C121340B94A9B00DE
:101E10009B580435FFF78FFA3B00083B18683B1FBF
:101E20001968A600BE1B0423814202D0042802D8F0
:101E30000023336018E001239C461842F8D10F2399
:101E400002681A40042AF3D163461942F0D10429EA
:101E5000EED90B680B321340042BE9D1FFF784F95C
:101E6000431E984180003060A14BA4001B783F1BAB
:101E70000437002B01D0FFF77CFA2B68019A1C1263
:101E800013409C4A9B009B580435FFF754FA3B00D3
:101E9000083B18683B1F1968A600BE1B002381423F
:101EA00002D0042802D80423336018E001239C46A2
:101EB0001842F8D10F2302681A40042AF3D163466E
:101EC0001942F0D10429EED90B680B321340042BD0
:101ED000E9D1FFF749F94342584180003060844B13
:101EE000A4001B783F1B0437002B01D0FFF741FAF9
:101EF0002B68019A1C1213407E4A9B009B580435A4
:101F0000FFF719FA3B00083B1868FFF70DF93B1F74
:101F100006001868FFF708F9F317C20F864253410D
:101F2000A4003A1B17009B001360714B04371B7809
:101F3000002B01D0FFF71DFA2B68019A1C121340E9
:101F40006C4A9B009B580435FFF7F5F93B00083BB2
:101F50001868FFF7E9F83B1F06001868FFF7E4F878
:101F60000023864200DD0433A4003A1B17001360EF
:101F70005F4B04371B78002B01D0FFF7FAF92B6871
:101F8000019A1C1213405B4A9B009B580435FFF7D3
:101F9000D2F93B1F1B68A400043B5A1E93413A1B15
:101FA00017009B001360524B04371B78002B01D0A5
:101FB000FFF7DFF92B68019A1C1213404D4A9B0072
:101FC0009B580435FFF7B7F93B00083B1868FFF74B
:101FD000ABF83B1F06001868FFF7A6F8321801207F
:101FE000A4003B1B1F00520002431A60404B043701
:101FF0001B78002B01D0FFF7BCF92B68019A1C124B
:1020000013403C4A9B009B580435FFF794F93B0072
:10201000083B1868FFF788F83B1F06001868FFF7B1
:1020200083F8321A0120A4003B1B1F005200024318
:102030001A602F4B04371B78002B01D0FFF799F95A
:102040002B68019A1C1213402A4A9B009B580435A6
:10205000FFF771F93B00083B1868FFF765F83B1F75
:1020600006001868FFF760F802000120A4003B1B7F
:102070001F007243520002431A601D4B04371B7845
:10208000002B01D0FFF775F92B68019A1C12134041
:10209000184A9B009B580435FFF74DF93B1F186801
:1020A000FFF742F8061E17D11F23114A1370A40030
:1020B0003B1B1F001E600E4B04371B78002B01D00A
:1020C000FFF757F92B68019A1C121340094A9B002D
:1020D0009B580435FFF72FF93B00083B1868FFF7C2
:1020E00023F8310007F092F9012640000643DEE7AD
:1020F000A802002080CE00003B1F1868FFF714F8EC
:10210000061E17D11F23F14A1370A4003B1B1F00AA
:102110001E60EE4B04371B78002B01D0FFF729F926
:102120002B68019A1C121340E94A9B009B58043506
:10213000FFF701F93B00083B1868FEF7F5FF310097
:1021400007F04AFA012649000E43DEE73B1F1868F4
:10215000FEF7EAFFC217801850400122A4003B1B83
:102160001F00400010431860D84B04371B78002B29
:1021700001D0FFF7FEF82B68019A1C121340D44AD5
:102180009B009B580435FFF7D6F8A300FE1A306871
:10219000012C24D1FEF7C8FF0494079009F05AFDE2
:1021A0000799002900DC012107F016FA049BA4001E
:1021B000C918012349001943C44B3F1B1B783160E8
:1021C0000437002B01D0FFF7D4F82B68019A1C12BA
:1021D0001340BF4A9B009B580435FFF7ACF8FEF74D
:1021E000A3FF04907068FEF79FFF049B0130C31AA1
:1021F0000793D3E7A300FE1A31002000049301F0F7
:1022000015FD049B3060FF1AB04B04371B78002B80
:1022100001D0FFF7AEF82B68019A1C121340AC4AAC
:102220009B009B580435FFF786F83B00083B186875
:10223000FEF77AFF3B1F06001868FEF775FF0200E5
:102240000120A4003B1B1F003240520002431A60D1
:102250009E4B04371B78002B01D0FFF78AF82B68C0
:10226000019A1C1213409A4A9B009B580435FFF7B1
:1022700062F83B00083B1868FEF756FF06003B1F5C
:102280001868FEF751FF320002430120A4003B1BF7
:102290001F00520002431A608C4B04371B78002B3E
:1022A00001D0FFF766F82B68019A1C121340884A88
:1022B0009B009B580435FFF73EF83B00083B18682D
:1022C000FEF732FF06003B1F1868FEF72DFF3200B5
:1022D00042400120A4003B1B1F00520002431A6031
:1022E0007A4B04371B78002B01D0FFF742F82B689C
:1022F000019A1C121340764A9B009B580435FFF745
:102300001AF83B1F1868FEF70FFFC0430122A40014
:102310003B1B1F004000104318606C4B04371B78B8
:10232000002B01D0FFF725F82B68019A1C121340EF
:10233000674A9B009B580435FEF7FDFF3B00083BB6
:102340001868FEF7F1FE06003B1F1868FEF7ECFE6A
:102350003200824051000122A4003B1B1F000A43AF
:102360001A605A4B04371B78002B01D0FFF701F895
:102370002B68019A1C121340554A9B009B58043548
:10238000FEF7D9FF3B00083B1868FEF7CDFE0600BC
:102390003B1F1868FEF7C8FE3200024151000122BF
:1023A000A4003B1B1F000A431A60484B04371B78EC
:1023B000002B01D0FEF7DDFF2B68019A1C121340A1
:1023C000434A9B009B580435FEF7B5FF3B000C3B8E
:1023D0001868FEF7A9FE3B00083B06001868FEF7E8
:1023E000A3FEF1170200C317300007F047F93B1FA7
:1023F000049005911868FEF797FE0200049805996D
:1024000007F0F0F843000120A4003E1B37001843FA
:102410002E4B30601B780437002B01D0FEF7A9FF4C
:102420002B68019A1C121340294A9B009B580435C3
:10243000FEF781FFA300FE1A310020000493FEF78F
:10244000BBFC049B3060FF1A204B04371B78002B29
:1024500001D0FEF78EFF2B68019A1C1213401C4A14
:102460009B009B580435FEF766FFA300FF1A390056
:102470002000FEF7B9FC154B1B78002B01D0FEF7AE
:1024800078FF2B68019A1C121340114A9B009B583D
:102490000435FEF750FFA300FE1A3100200004931C
:1024A000FEF7E2FC049B3060FF1A084B04371B78F0
:1024B000002B01D0FEF75DFF2B68019A1C12134020
:1024C000034A9B009B580435FEF735FFA802002005
:1024D00080CE0000A300FF1A39002000FEF758FD4F
:1024E000E44B1B78002B01D0FEF743FF2B68019AC9
:1024F0001C121340E04A9B009B580435FEF71BFF5B
:10250000A300FE1A310020000493FEF7B3FD049BE4
:102510003060FF1AD74B04371B78002B01D0FEF731
:1025200028FF2B68019A1C121340D34A9B009B582A
:102530000435FEF700FF3B1F186800F0D1FF3A009A
:10254000083A12680300A400D10729D4042A0CD940
:1025500010680F221040013808280FD806F0C2FE7C
:10256000052026220E0E0E0E2400C449180009F084
:1025700011FC434258413B1B80001860BD4B3F1B80
:102580001B780437002B01D0FEF7F3FE2B68019A6D
:102590001C121340B84A9B009B580435FEF7CBFE33
:1025A000B749E3E7B749E1E7B749DFE7B749DDE70F
:1025B000069B3E1DF31AAF4CD82B03DD1A23237064
:1025C000FEF7D7FE00F0E4FC430001201843237817
:1025D0003860002B02D03700FEF7CBFE2B68019A43
:1025E0001C121340A44A9B009B5837000435FEF789
:1025F000A2FE069B3E1DF31A9E4CD82B03DD1A2328
:102600002370FEF7B6FE00F0B9FCA14B4000184065
:102610000123184323783860002B02D03700FEF7DF
:10262000A8FE2B68019A1C121340934A9B009B58EA
:1026300037000435FEF77FFE069B3E1DF31A8D4CD6
:10264000D82B03DD1A232370FEF793FE00F0A0FCC5
:10265000904B1A68831A904201D28F4A9B1801202E
:102660005B0003433B602378002B02D03700FEF76A
:1026700080FE2B68019A1C1213407F4A9B009B58D6
:1026800037000435FEF757FE00F082FC814BA400B2
:102690001860784B3F1B1B78002B01D0FEF769FEBA
:1026A0002B68019A1C121340734A9B009B580435F7
:1026B000FEF741FE0123A600BE1B20001A003100D8
:1026C000FEF780FD754C2068643002F0FDFE0028A6
:1026D00002D1043DFEF760FE029B21685A787048E3
:1026E00003F015FB0123029A3700137000F046FC3B
:1026F0006C4B22681B68063253431818029B5860C3
:10270000FEF74AFEA600BE1B200001230022310076
:10271000FEF758FD614C2068643002F0D5FE0028B9
:10272000D7D05F4803F070F8DCE7A4003E1BFEF74B
:10273000C9FD37004F4B30601B780437002B01D0A8
:10274000FEF717FE2B68019A1C1213404A4A9B00A1
:102750009B580435FEF7EFFD464BA4001B783F1B4A
:10276000002B01D0FEF705FE2B68019A1C121340C6
:10277000414A9B009B580435FEF7DDFDA4003E1B3B
:10278000300000F038FC37003A4B30601B780437DB
:10279000002B01D0FEF7EDFD2B68019A1C121340AF
:1027A000354A9B009B580435FEF7C5FDA4003E1B2F
:1027B000300000F022FC37002E4B30601B780437CD
:1027C000002B01D0FEF7D5FD2B68019A1C12134097
:1027D000294A9B009B580435FEF7ADFDA300FE1A65
:1027E00031002000049300F00BFC049B3060FF1AC2
:1027F000204B04371B78002B01D0FEF7BAFD2B6865
:10280000019A1C1213401C4A9B009B580435FEF78A
:1028100092FDA4003F1B380000F024FC154B1B78F0
:10282000002B01D0FEF7A5FD2B68019A1C12134066
:10283000114A9B009B580435FEF77DFDA300FE1A4C
:1028400031002000049300F035FC049B3060FF1A37
:10285000084B04371B78002B01D0FEF78AFD2B684C
:10286000019A1C121340044A9B009B580435FEF742
:1028700062FDC046A802002080CE0000BCD000004F
:10288000C4D00000CBD00000D2D00000D7D00000D0
:10289000FEFFFF7FD405002037894100CC050020D2
:1028A000A902002004000020A4003F1B380000F013
:1028B00043FCFC4B1B78002B01D0FEF75AFD2B6824
:1028C000019A1C121340F84A9B009B580435FEF7EE
:1028D00032FD0121200000F017FCF24B1B78002B89
:1028E00001D0FEF746FD2B68019A1C121340EE4AF8
:1028F0009B009B580435FEF71EFD0021200000F0D0
:1029000003FCE84B1B78002B01D0FEF732FD2B684F
:10291000019A1C121340E44A9B009B580435FEF7B1
:102920000AFDA4003E1B300000F028FC3700DD4B00
:1029300030601B780437002B01D0FEF71AFD2B689E
:10294000019A1C121340D84A9B009B580435FEF78D
:10295000F2FCA4003E1B300000F024FC3700D14BF9
:1029600030601B780437002B01D0FEF702FD2B6886
:10297000019A1C121340CC4A9B009B580435FEF769
:10298000DAFCA4003F1B380000F0E6FBC54B1B78C7
:10299000002B01D0FEF7EDFC2B68019A1C121340AE
:1029A000C14A9B009B580435FEF7C5FCA4003F1BA1
:1029B000380003F007FDBB4B1B78002B01D0FEF75E
:1029C000D8FC2B68019A1C121340B74A9B009B58F5
:1029D0000435FEF7B0FCA4003E1B300003F08CFD74
:1029E0003700B04B30601B780437002B01D0FEF766
:1029F000C0FC2B68019A1C121340AB4A9B009B58E9
:102A00000435FEF798FCA4003F1B380003F08AFC55
:102A1000A44B1B78002B01D0FEF7ABFC2B68019A6E
:102A20001C121340A04A9B009B580435FEF783FC00
:102A3000A4003E1B300003F08BFC3700994B306044
:102A40001B780437002B01D0FEF793FC2B68019A0A
:102A50001C121340944A9B009B580435FEF76BFCF4
:102A6000A300FF1A3900200001F024FC8D4B1B78D5
:102A7000002B01D0FEF77DFC2B68019A1C1213403D
:102A8000894A9B009B580435FEF755FCA300FF1AAA
:102A90003900200001F022FA824B1B78002B01D074
:102AA000FEF767FC2B68019A1C1213407E4A9B00BC
:102AB0009B580435FEF73FFCA300FF1A39002000A5
:102AC00001F030FB774B1B78002B01D0FEF751FC57
:102AD0002B68019A1C121340734A9B009B580435C3
:102AE000FEF729FCA300FF1A3900200001F042FB89
:102AF0006C4B1B78002B01D0FEF73BFC2B68019A36
:102B00001C121340684A9B009B580435FEF713FCC7
:102B1000A300FE1A31002000049303F085FD049BFE
:102B20003060FF1A5F4B04371B78002B01D0FEF793
:102B300020FC2B68019A1C1213405B4A9B009B5897
:102B40000435FEF7F8FBA300FE1A310020000493C1
:102B500003F072FD049B3060FF1A524B04371B7860
:102B6000002B01D0FEF705FC2B68019A1C121340C4
:102B70004D4A9B009B580435FEF7DDFBA300FE1A6F
:102B800031002000049303F05FFD049B3060FF1AC6
:102B9000444B04371B78002B01D0FEF7EAFB2B686F
:102BA000019A1C121340404A9B009B580435FEF7C3
:102BB000C2FBA300FE1A31002000049303F01CFBAB
:102BC000049B3060FF1A374B04371B78002B01D071
:102BD000FEF7CFFB2B68019A1C121340324A9B0070
:102BE0009B580435FEF7A7FBA300FF1A390020000D
:102BF00001F0ACF92B4B1B78002B01D0FEF7B9FB91
:102C00002B68019A1C121340274A9B009B580435DD
:102C1000FEF791FBA300FF1A3900200001F0D2FA61
:102C2000204B1B78002B01D0FEF7A3FB2B68019AE9
:102C30001C1213401C4A9B009B580435FEF77BFB7B
:102C4000A300FE1A31002000049301F037FA049B20
:102C50003060FF1A134B04371B78002B01D0FEF7AE
:102C600088FB2B68019A1C1213400F4A9B009B584B
:102C70000435FEF760FBA300FF1A3900200001F0C5
:102C8000E5F9084B1B78002B01D0FEF772FB2B688F
:102C9000019A1C121340044A9B009B580435FEF70E
:102CA0004AFBC046A802002080CE0000069B029A84
:102CB000FB1A9B101361A300FF1A3900200002F0D9
:102CC000E1FD184B1B78002B01D0FEF752FB2B685F
:102CD000019A1C121340144A9B009B580435FEF7BE
:102CE0002AFB069B029AFB1A9B101361A300FE1A93
:102CF00031002000049302F0C5FD049B3060FF1AF0
:102D0000084B04371B78002B01D0FEF732FB2B68F1
:102D1000019A1C121340044A9B009B580435FEF78D
:102D20000AFBC046A802002080CE00000023F7B5B1
:102D30005A1E0192002B07DA01F0D2FA02F0D2FEFD
:102D400003F044F81923019300263000194B196849
:102D5000B14212DD184B1A6801328A420FDAF024B0
:102D60001A601D68154F6C43E35D002B1FD0E419FA
:102D7000022B06D12000FEF7BDFA019BD8E7002206
:102D8000EDE7012B0DD1002801D100F0F7F8F0227A
:102D90006A43BB185B680A49C31A8B4201D80223F5
:102DA000BB54F0235D43054BEB5C022BE2D00136B4
:102DB000CCE7C046D0050020000000203C1C0020CD
:102DC0003F420F00012200210A4B0B481A611950A3
:102DD00004301950A2210420C9005850C121C0203C
:102DE0008900800258501A60044BFC311960044B72
:102DF0001A70704700A000400405000000E100E0E8
:102E0000FB05002004207047F8B550C901232200BB
:102E10001A40101E2DD03340181E2AD064100020F6
:102E20001C2C26D81D4B761035009E4200DD1D005F
:102E30001B4F3B5D012B05D00121200004F02AFE31
:102E400001233B55174B1B78002B01D1FFF7BAFF2D
:102E50000023154A9E420DDCFF2514491448D65C18
:102E6000B44202D15E007052D5540133042BF6D126
:102E70000420F8BDD15C8C4203D10C4A5B009D520A
:102E8000F6E70133042BF5D10023D15CFF2901D1F2
:102E9000D454F2E70133042BF7D1E9E7881300009B
:102EA000DC050020FB0500201C0000200E00002097
:102EB000DC05000070B530C9012322001A40101E45
:102EC0001BD02B40181E18D064101C2C00D90024D5
:102ED000174E335D012B05D00121200004F0DAFDEF
:102EE0000123335569100800124A1038124B9042E2
:102EF00004D9012252421A60042070BD1C600F48A0
:102F000006F084FA0E4B18800E4B1B78002B02D172
:102F1000FFF758FFF0E701220B4B9A64A922D20079
:102F20009A588018A82280B2D2009850E4E7C04690
:102F3000DC050020908601001800002020A1070079
:102F40000C000020FB05002000A00040030010B58D
:102F50000120002B02DC1B30FEF7AEF910BD04206F
:102F6000704710B5002803DC1C20FEF7A5F910BD42
:102F70000B680020DB07FAD40D30F6E70122034B83
:102F80001A64A822D20098587047C04600800040BA
:102F900010B5FFF7F3FFFA21890006F0ADF910BD77
:102FA0000048704734D100001D20704770B5054EB1
:102FB0000400335C0D008B4202D004F06BFD3555EC
:102FC00070BDC046DC05002070B50024084D635D6F
:102FD000012B09D10021200004F082FD00212000F6
:102FE00004F058FD0023635501341D2CEED170BD53
:102FF000DC05002070470D2070473B207047000023
:10300000F8B501240B6806000D00234204D10D2001
:10301000FEF752F92000F8BD5B102000052BFAD80E
:103020000E4A9B009C580E4F3B5D002B05D00021A3
:10303000200004F02FFD00233B55012E06DD6B68B8
:10304000042B03D10221200004F024FD200004F011
:10305000CFFB012440002043DDE7C0461CD1000027
:10306000DC050020F8B501260568354202D0446829
:10307000344203D10D20FEF71FF9F8BD6D101C2D51
:10308000FBD80A4F7B5D012B04D03100280004F0EF
:1030900001FD7E55064964108C4202DCE143C917EC
:1030A0002140280004F02AFCE7E7C046DC050020A8
:1030B000FF03000070B501240D68254204D10D20E6
:1030C000FEF7FAF8200070BD6D101C2D17D80024F3
:1030D000012804DD4C68043C63425C416400094EF5
:1030E000735DA34204D02100280004F0D3FC745582
:1030F000280004F013FD03000420012BE3D000207E
:10310000E1E7C046DC05002070B504000D001C2876
:103110000ED8084E335C012B04D0012104F0BAFC18
:1031200001233355290020004D1EA94104F0D8FC8D
:1031300070BDC046DC050020036810B5DA0703D473
:103140000D20FEF7B9F810BD4168581004394A4205
:103150005141FFF7D9FFF6E737B569460A00064B3C
:1031600030CB30C203680220042B02D100F0DAFF1A
:1031700037BD00F0FFFFFBE7E4D0000010B5084CBE
:103180006379002B05D00021052004F083FC002387
:103190006371052004F0C2FC43425841800010BD19
:1031A000DC05002010B5084CE37A002B05D0002187
:1031B0000B2004F06FFC0023E3720B2004F0AEFC44
:1031C00043425841800010BDDC05002070470000DC
:1031D000F7B5304D304E6B6C002B15D0A824002372
:1031E000E40037596B642D4B186800280CDB2C4B1E
:1031F00019784A425141C9B2197004F071FC294B47
:103200001B88DF19BFB23751AB6C002B39D00021BE
:10321000254B264FF458A9643A780C340193244D79
:103220008A4206D02B68032B03D8224AD05C04F0D4
:1032300057FC2B68204A0133134004D50422013B7C
:103240005242134301331B4900228C462B60042B4E
:1032500018D06046C05C591CFF2802D10B00012227
:10326000F5E7002A00D02B60012104F039FC01238E
:103270003B702B68114A5B009B5AE418019BA4B277
:10328000F450F7BD01235B422B6000233B700C4BD5
:10329000F3E7C046FCA0004000A00040180000205A
:1032A000FA0500200C00002044050000F90500206C
:1032B000D80500201C000020030000800E00002024
:1032C00050460000084B094AFF201A805A809A8015
:1032D000DA800023064A07491370074A08704870CD
:1032E0008870C870136070470E000020DC05000075
:1032F000F90500201C000020D80500200122024B07
:1033000052421A607047C0461800002010B5034AA8
:103310000621034802F09EF810BDC046ECD0000024
:1033200056D80000E12170B54902194803F0D4FFD6
:10333000002401220320174B17491A615C50043105
:1033400058508018083158501A60063004F04AFA74
:10335000FF21124AA15401341D2CFBD1012200206F
:103360000F4B01001A6004230E4A0F4D1468002C05
:10337000FCD02C680002013B20431160002BF5D1EA
:1033800001220A4B1A6004F063F901F0F5F870BDF0
:10339000C41B00200080004004050000DC05002064
:1033A00000D0004000D1004008D5004004D00040CB
:1033B000F8B50B4E070030000D0003F0D5FF0400F8
:1033C000A84200DD2C003D00EB1B9C4205DD3000D7
:1033D00003F0D4FF28700135F6E72000F8BDC046A1
:1033E000C41B002010B50100014803F07DFF10BD93
:1033F000C41B002010B5054C200003F083FFE12121
:103400002000490203F068FF10BDC046C41B002025
:10341000C3070CD4064B1B68834208D8054B1B68B6
:10342000984204D8031F1B68002B00D01800704777
:1034300004060020000600200023012210B50A48DF
:10344000990001334250642BFAD1084C084B0021FB
:103450001A602000074A08F01DF9074B074A63600D
:10346000074B1A6010BDC046942D002008060020AE
:1034700008000020D4090000302700000C060020BE
:10348000FC05002010B5044B044A1A60044B054AA1
:103490001A60FFF7D1FF10BD0406002008060020C7
:1034A00000060020DC0F0020044B1B681868000990
:1034B00080B20238C343DB1718407047FC05002078
:1034C00000B59BB00200054901A808F027FC01A83F
:1034D00002F0B6F902F07AFCFCE7C046B8D1000071
:1034E0000B4BC20704D4042804D80A4B00D00A4B63
:1034F000180070470F2203681A40031D042AF7D0F2
:10350000064B092AF4D0064B032AF1D0054BEFE70E
:1035100092D1000036CD000030CD00009CD10000DB
:10352000ACD10000A3D100000020064A0649131FB9
:10353000186013681B099BB202339B00D2188A42A1
:10354000F5D370470C060020DC0F0020F7B50F24E0
:103550000126314B314A1968314B324D18681368D6
:103560001F002740072F26D813681B099BB2023380
:103570009B00D218AA42F2D300242B4EA500AD190D
:103580002868FFF745FF01342860642CF6D1274CEA
:103590002068FFF73DFF2060254C2068002802D0FE
:1035A000FFF736FF20600025224B1B680093009B2D
:1035B0009D4214DBF7BD1B099BB29B00D3189A42B6
:1035C000D2D01F68374208D1B94206D2B84204D3DC
:1035D000043F3F68002F00D01F60043BEFE7F0235B
:1035E0006B43154A9B181A78002A01D10135DEE792
:1035F0001F693C2300266B43DB199B0001930136B6
:10360000BB1BF3D4019BB4001C1B0B4B1C19A06902
:10361000FFF7FEFEA061F2E7040600200C06002082
:1036200000060020DC0F0020942D00200800002060
:10363000DC0F0020D00500203C1C0020F7B5012441
:10364000204246D1234B1B689C46984241D3224BD3
:103650001B68019398423CD8031F1B68002B38D18C
:103660000200036800941B099BB2002B0FD1009944
:10367000131F196090422CD015682B1F1B689900EE
:1036800069180C68013B14600A602A00EDE79D0090
:1036900055192968009C214219D18C4517D8019CE5
:1036A0008C4214D30E1F3468002C10D10F680F34D5
:1036B0003C40072C08D92F60151F2B600B680A604F
:1036C0001B099BB20A00D0E700993160CDE7013BAE
:1036D000CBE7F7BD04060020000600200D4970B5B9
:1036E0000A000D4D1368141F1B0926689BB2981C15
:1036F000002E0BD000238A4200D00B0023608300F1
:10370000C91880001218AA42ECD370BD1B011360C7
:10371000F7E7C0460C060020DC0F0020F8B5124C7D
:1037200027000F223B681D09ADB213420DD06E1C5D
:10373000B600A74204D032003900200007F097FFFE
:103740000022A3190436A4191A600235AD00074BF4
:103750007F199F42E5D31B1B9B10013B1B0123607C
:10376000034B1C60F8BDC0460C060020DC0F002097
:10377000FC050020F0B59BB0FFF700FC002407001B
:10378000214AA300D0580134FFF758FF642CF7D129
:103790001E4B1868FFF752FF1D4B1868002801D018
:1037A000FFF74CFF00261B4B1B689E4217DBFFF701
:1037B00095FFFFF7CBFEFFF7B1FFFFF7DFFB164BDF
:1037C000C21B1B6815491B6801A81B099BB2023B61
:1037D00008F0A4FA01A802F033F81BB0F0BDF02500
:1037E00075430F4BED182B78002B01D10136DAE72A
:1037F0002B695C1E002CF9DBA300EB189869FFF71E
:103800001DFF013CF6E7C046942D00200800002073
:10381000DC0F0020D0050020FC05002072D1000044
:103820003C1C0020F7B5174D4F1C2B6806001B6889
:103830000C001B099BB201929F420BDBFFF79AFF22
:103840002B681B681B099BB29F4203DB0A20FDF714
:1038500033FDFEBD2868A71CBA00DB1B81181B01C5
:103860000B6029600021031F19600F231E40030015
:103870002401264340C3083A9A189A42E9D901998B
:1038800002C3FAE7FC050020F7B50300012213404C
:1038900004000D000193002B2BD1174B1B688342B2
:1038A00027D8164B1B68834223D90F23144F386047
:1038B00000681840FFF7B6FF019B3C68061E3B609E
:1038C00017D0236804301B099BB29D4200DD1D0008
:1038D000AA00211D251F07F0C1FEFFF725FE2E605F
:1038E000FFF734FE00232B602268064B1340236051
:1038F00034002000FEBDC046040600200006002063
:10390000DC0F0020F0FF0F000323043010B5C117B7
:1039100019400918891000220420FFF783FF10BD09
:1039200070B5050008000C00FFF7EEFF002300282B
:1039300004D170BDE95CC21811710133A342F9DBF7
:10394000E343DB171C40002304192371F1E7F0B5B2
:103950000C009BB0022804DC1C20FDF7ADFC1BB062
:10396000F0BD01230868184206D1042804D90F26A7
:1039700001683140042901D00E20EEE761680D0096
:103980001D40F9D10429F7D90A683240042AF3D13D
:10399000A2681A4201D10D20DFE7FFF7A1FD060062
:1039A0006068FFF79DFDA768010001AC7F10300043
:1039B000257003F028F839006423220003F088F80A
:1039C000200008F0F1F901002000FFF7A9FFC6E789
:1039D00010B51C4CA544041E02D1FFF795FF0BE067
:1039E00002F02AFF0138062828D805F07BFC0909D7
:1039F00011182904240000208023DB009D4410BD01
:103A0000200002F095FF011B2000FFF789FFF3E77C
:103A1000200002F03BFF430001201843ECE7802226
:103A20006946D200200002F048FF684608F0BCF961
:103A300001006846E9E704210348E6E70020CCE7F7
:103A40000420D9E700FCFFFF00D2000070B50C0095
:103A5000022803DC1C20FDF72FFC70BD0123086841
:103A6000184206D1042804D90F25016829400429E9
:103A700001D00E20EFE761681942FAD10429F8D984
:103A80000A682A40042AF4D1A2681A4201D10D2002
:103A9000E1E7FFF725FD05006068FFF721FDA46859
:103AA00001006410280002F0AEFF210002F0EBFFDD
:103AB000FFF78EFFD1E770B50D00012803DC1C2055
:103AC000FDF7FAFB70BD01240868204206D10428E6
:103AD00004D90F2102680A40042A01D00E20EFE722
:103AE0006A682242FAD1042AF8D913680B40042BE1
:103AF000F4D1FFF7F5FC06006868FFF7F1FC010060
:103B0000300002F080FF03F002F840002043D9E7C4
:103B1000F8B507000C001C20012F0BDD01250868FB
:103B2000284206D1042804D90F2102680A40042A39
:103B300003D00E20FDF7C0FBF8BD62682A42F8D121
:103B4000042AF6D913680B40042BF2D1FFF7C8FC06
:103B500006006068FFF7C4FC0100022F14D0A468BF
:103B60002C4211D06410300002F04DFF050002F02D
:103B700063FE012811D1002C02DD0135012C06D194
:103B80002800FFF725FFD7E701246442EBE7280070
:103B900002F0DAFE013C0500F0E70228F0D1002C2B
:103BA000EEDD0135012CEBD000222800110002F0DF
:103BB000FDFE02F0C9FE013C0500F3E710B501244B
:103BC0000868044016D04410200005F0B3FE1549E3
:103BD00005F07EFD07F064FC04F0B6F80022124BFD
:103BE00006F018FE04F058F807F0EAFB4300012045
:103BF000184310BD042810D90F2302681340042B6A
:103C000007D1FFF76DFC21000A2208F095F90400A6
:103C1000DAE7032B01D10430F5E70D20FDF74CFB6B
:103C2000D2E7C046D30237390000D040086870B5EB
:103C300001240500254006D1042804D90F23026879
:103C40001340042B03D00E20FDF736FB70BDFFF7A9
:103C500047FC03782900233B5A4253411022C018E5
:103C600008F06AF980239B05C218044B9A4201D9D7
:103C70001420E9E740002043E8E7C046FFFFFF3F8C
:103C800010B5034A0621034801F0E4FB10BDC0460D
:103C9000D0D10000C9D100000020704710B51E200F
:103CA000FDF70AFB10BD10B51E20FDF705FB10BD8A
:103CB00010B51E20FDF700FB10BD10B51E20FDF74E
:103CC000FBFA10BD10B51E20FDF7F6FA10BD10B5B9
:103CD0001E20FDF7F1FA10BD10B51E20FDF7ECFA1D
:103CE00010BD10B51E20FDF7E7FA10BD10B51E205F
:103CF000FDF7E2FA10BD10B51E20FDF7DDFA10BD8C
:103D000010B5034A0B21034801F0A4FB10BDC046C7
:103D10003CD2000094D200000120034B1860034BFA
:103D20001B6883401843704700100020E00F0020FC
:103D3000F0B5EFF310810123194083F31088134C81
:103D4000134AA4461268134E013A9340124F134A85
:103D5000002B17D0146803420FD03D682C60C0467A
:103D6000C046C046C046C046C046C046C0460C4CD1
:103D70001568246825605B08EAE765462C601468CE
:103D80003460F8E781F31088F0BDC04608050050A4
:103D9000200000200C050050EC0F0020F40F002044
:103DA000E80F002030B585B001AD0C22064928008F
:103DB00007F054FC0024285D01210134FFF7F6F8D8
:103DC0000C2CF8D105B030BD29D30000F7B56A46F8
:103DD0003B4B01AE13800A2393703A4B33801C2374
:103DE000B370FFF7CBF8384B384DC0182B689842AA
:103DF00001D200232B602C68002C41D1375D0121BA
:103E00003800FFF7D3F801340021380003F068FED2
:103E1000032CF3D1002401276B461E5D39003000CE
:103E2000FFF7C4F801343900300003F059FE032CC9
:103E3000F2D1C8200138C046C046C046C046C04680
:103E4000C046C046C046C046C046C046C046F1D186
:103E50006B4600211878FFF7A9F86B4600215878C7
:103E6000FFF7A4F86B4600219878FFF79FF8FFF75B
:103E700085F8FA2300241B01C01828602000FEBD2D
:103E8000FFF77CF82B6800249842F7D3032003F057
:103E9000AFFC0600042003F0ABFC36180A2003F048
:103EA000A7FC0B4B9B1B181A0A4BA04206DB1860A1
:103EB0000023094A2B6013600124DFE71C60F7E749
:103EC000030400001A1B000010270000F80F002058
:103ED000E3030000E00F0020001000200022054B4B
:103EE00010B51A60044B1B68934201D002F044FCE9
:103EF000002010BDFC0F0020E81A002010B5041EA1
:103F000010DA00240A4BA400E25801239340094A26
:103F100009491360094A1160094A0A4911600A4AAD
:103F2000136010BDFFF740F8A042EADDEAE7C046A3
:103F300050E00000F40F002008050050EC0F0020B6
:103F4000E80F00200C05005018050050F0B53B4B61
:103F500085B01B680C00002B03D101204042FFF705
:103F6000CDFF246801222700174028D0FF236012CC
:103F7000184033496714661040431F401E4005F047
:103F800045FA050438002E49784305F03FFA00024F
:103F9000054330002A49704305F038FA294B28437D
:103FA0001B68202B06D16400A40E274BA400E35805
:103FB00000021843FFF7BCFE002005B0F0BD042C42
:103FC000FAD90F2321680B40092BF5D163680392BE
:103FD0005B100193019B9F42EEDABB00E3189E68E1
:103FE000039B1E4228D0FF237012184072101A4003
:103FF0001349751440431D40009205F007FA03046D
:1040000028000F496843029305F000FA029D000260
:10401000054300980A49404305F0F8F9094B284345
:104020001B68202B06D17600B60E074BB600F5585C
:1040300000022843FFF77CFE0137CBE7F40F002096
:10404000590600002000002010D50000020008687A
:1040500010B5C3070FD540101823012A03DD4A68A5
:10406000042A00D10833054A1360FEF7C3FFFFF7A7
:1040700045FF002010BD01204042EDE72000002058
:1040800010B50124044002D04410200010BD0428C3
:1040900010D90F2302681340042B07D1FFF720FA31
:1040A00021000A2207F048FF0400EEE7032B01D1AC
:1040B0000430F5E70D20FDF7FFF8E6E70868F8B5EE
:1040C000C3071AD5FFF7DCFF0300203B5E2B25D882
:1040D0000520434301221D180020114E9D4219D096
:1040E00005211024F75C3C4200D0801801395200B1
:1040F00064100029F7D10133F0E704280ED90F220C
:1041000003681A40042A09D11B099BB2002B05D071
:104110000379DAE7012340001843F8BD0120FCE7EA
:1041200035D3000070B508680D00FFF7A9FF040043
:104130006868FFF7A5FF621E0100042A14D8451E17
:10414000042D11D805236B439B18012215009D40B7
:104150002B00064805682B430360054B1B68002BAA
:1041600002D0200002F009FB002070BDFC0F0020EF
:10417000E81A002070B508680D00FFF781FF040001
:104180006868FFF77DFF621E0100042A13D8451EF0
:10419000042D10D805236B439B1801229A40074831
:1041A000036893430360064B1B68002B03D0002277
:1041B000200002F0E2FA002070BDC046FC0F002093
:1041C000E81A0020F0B5050089B008680C00FFF778
:1041D00057FF0690022D36DD6068FFF751FF019012
:1041E000A068FFF74DFF04000127231D661E0793FB
:1041F000731C0293079B9E4235D00523734305939E
:10420000019B019D05330493049BAB421ED0042EF9
:1042100016D86B1E042B13D80122059B2349013BA2
:104220005B199A409446224A0B681068069A3A40F5
:1042300003920DD062461A430A60012200280DD174
:104240007F000135E0E701240194CDE7029ECFE72E
:10425000624693430B600028F2D0039A029928002B
:1042600002F08BFAECE7019B1E1D042E1AD8012CDC
:1042700018D1002505273B0021006B439B1999406D
:104280000B000A4A013511689943094B11601B68FC
:10429000002B05D0019B0022581D290002F06DFA69
:1042A000052DE8D1002009B0F0BDC046FC0F00206C
:1042B000E81A0020086810B5C30703D5FFF7E0FE31
:1042C000054B1860054B1B68002B03D0024B186888
:1042D00002F054FA002010BDFC0F0020E81A002064
:1042E0007FB5A04C2368002B0AD19F4A1268002A90
:1042F00006D19E4B1B68002B01D0FFF767FD7FBDE9
:104300009B4D2A68002A26D1984A1268002A1BD0A1
:10431000FFF75CFD0028F2D0FFF744FD924B2468C4
:104320001A681C60002A16D0002C14D101AD0C2292
:104330009049280007F092F9285D00210134FEF72A
:1043400035FE0C2CF8D1DAE7874A1268002AE5D14D
:10435000002BE3D0E0E700211A2003F0C1FB00218D
:104360001B2003F0BDFB00211C2003F0B9FB2E68CD
:10437000012E5CD0022E00D1A2E0002E50D10136D9
:104380003100794C03202368994303F0A9FB0420F2
:10439000216801404B42594103F0A2FB10212368E0
:1043A0000A2019404B42594103F09AFB80212368AF
:1043B000090119404B425941062003F091FB80212D
:1043C0002368090219404B425941072003F088FB3A
:1043D00080212368490219404B425941092003F0CA
:1043E0007FFB80212368890219404B4259411920E3
:1043F00003F076FB80212368C90219404B425941E2
:10440000182003F06DFB802321681B0319404B42E9
:104410005941172003F064FB31001A2003F060FBC0
:104420002B680321581C05F0D7F8296067E70221A3
:104430004D4C1720236819404B42594103F050FB63
:1044400008212368182019404B42594103F048FBCA
:1044500080212368C90019404B425941042003F0D0
:104460003FFB80212368490119404B4259410A20F2
:1044700003F036FB80212368C90119404B425941A2
:10448000032003F02DFB80212368890319404B4250
:104490005941092003F024FB802321681B041940A3
:1044A0004B425941192003F01BFB3100062003F059
:1044B00017FB3100072003F013FB31001B20ADE791
:1044C0002021294C1720236819404B42594103F001
:1044D00007FB40212368182019404B42594103F043
:1044E000FFFA80212368192019404B42594103F0FB
:1044F000F7FA80212368490019404B4259410920AD
:1045000003F0EEFA80212368890019404B4259419B
:10451000072003F0E5FA80212368890119404B4206
:104520005941062003F0DCFA802123684903194031
:104530004B4259410A2003F0D3FA80212368C90372
:1045400019404B425941032003F0CAFA80232168E5
:104550005B0419404B425941042003F0C1FA012188
:104560001C205BE7FC0F0020F00F00200010002053
:10457000E40F002029D30000012010B54042FFF7CE
:10458000BDFC10BD10B5034A0921034800F062FFCD
:1045900010BDC04610D6000058D600008023F0B5EC
:1045A00002255B051A690A4C0A4BA1261D510327F7
:1045B0008025F600ED00BA43884202D300221A514A
:1045C000F0BD5F59002FFCD098518018F4E7C04629
:1045D0000405000000E0014010B5002806D1C0200D
:1045E000B02140028902FFF7D9FF10BDB020802121
:1045F0008002C902F7E7000043425841064B40429F
:104600001840B0239B02C018036800201A0E532ADA
:1046100001D11B02180A704700C0FEFF30B501240B
:104620008025054B054AED009C505C59002CFCD0C0
:1046300001600021995030BD00E0014004050000F8
:1046400043425841074B40421840B0239B02C018D8
:10465000A62310B50902DB05090A1943FFF7DEFF9F
:1046600010BDC04600C0FEFFF0B5012480260D4BF2
:104670000D4DF6005C51002902DC00225A51F0BDBC
:10468000577814783F022743947824042743D4783A
:10469000043224063C439F59002FFCD010C001393E
:1046A000E9E7C04600E001400405000070B50500E0
:1046B0004B680A009C1C2100A400FFF7D5FF2819B5
:1046C00070BD0000134B1B68002B0CD08022B02360
:1046D000D2029B0200280BD11A1D5B681B0E522BC5
:1046E00000D110007047B022C02392025B02F1E7B4
:1046F00082420DD903681B0E522B09D14368023345
:104700009B00C018824203D903681B0E522BE9D0CC
:104710000020E7E704110020F0B50020B7B0002426
:10472000FFF7D0FF270005002600002D2ED1284DD1
:104730002868FFF761FF32003B0001900094254993
:1047400004A807F0EBFA04A801F07AF8224B6420E1
:104750001C682B68A0215A425341204A5B421340F7
:10476000B02292029B18E41A6043490204F04EFE04
:10477000A0225202030000921949220004A807F067
:10478000CDFA04A801F05CF837B0F0BDFF226B68E9
:1047900029689C460233FF180B12013613409C42D5
:1047A00000DA1C00FF200A14024003926246014016
:1047B00001920091039A0B4904A807F0AFFA04A8EC
:1047C00001F03EF82800FFF77DFF0500ADE7C04689
:1047D0000411002062D700000811002000C0FEFF75
:1047E0000CD700004ED7000070B50020FFF704FF83
:1047F00004000120FFF700FF844200DA04000A4BA6
:104800001D686A42554128001D60FFF7E5FEA022A1
:104810006B4252021340054A28009B18044A611C4F
:104820001360FFF70DFF70BD04110020048001002C
:1048300008110020F8B50020FFF7DEFE0700012078
:10484000FFF7DAFE3E00204D0643204C0DD18021BB
:10485000C020C9024002FFF7A1FE01213000FFF78E
:10486000EFFE1B4B2E6023601DE0874209DD002315
:10487000B0212B60164B890223602368002001259C
:1048800017E0012380212B60124BC9022360F4E75B
:10489000120E522A08D0002800D023600E4800F0E3
:1048A000CFFFFFF7A1FFF8BD28005A68023292003F
:1048B0009B188B4205D21A68561CE9D10028F2D009
:1048C000D1E72160EFE7C046041100200811002065
:1048D0000480010004C0020027D7000070B500204A
:1048E000FFF7F0FEFF260500002801D1280070BD6B
:1048F00003681C143440FFF7E5FEDA2CF4D1050000
:10490000F2E700008022F0B55200A1B00021674814
:1049100006F0C0FE802200215200654806F0BAFE73
:10492000644BFF271B681A00049353425A4110003E
:104930000592FFF751FE049C0020631E9C415E4BD4
:1049400064421C405D4BE418FFF7C8FF0600002ED0
:104950002DD10498FFF750FE411C0598FFF770FE1B
:10496000059A574D534B2C601A60FEF743FD514B8F
:1049700064201B68A0215A4253414F4A5B421340B6
:10498000B0222C6892029B18E41A6043490204F09A
:104990003DFDA0225202030000924A49220007A8CE
:1049A00007F0BCF907A800F04BFF21B0F0BD32685A
:1049B000131412123A403B4003921A000A3A092A91
:1049C00049D83A4B039A995C002931D110223E48CC
:1049D00006F060FE35002B6803991A123A409142A6
:1049E00009D11A143A400B2A27D0132A2DD00A2AAB
:1049F00001D1354B1D602800FFF764FE051EEAD18A
:104A0000314B196800290FD02000FFF74FFE04003A
:104A10002D4B5B195968002903D02000FFF746FE93
:104A2000040004350C2DF3D1204B0121039A995435
:104A30003000FFF747FE060089E73B40022BDADC37
:104A4000214A9B00D3185D60D5E7102200211E4843
:104A500006F020FECFE71A00153A082AE8D8144AD3
:104A60000399525C002AE3D13500152B00D01500C4
:104A7000300003681A143A40152A0FD01D2A00D1BD
:104A80000025FFF71FFE0028F3D1002D04D02000E1
:104A90002900FFF70BFE0400054BC6E7039A1B1223
:104AA0003B409A42EDD10500EBE7C04604100020E0
:104AB0000C1100200411002000C0FEFF04C0020001
:104AC00008110020F1D60000242F002010B5FFF7B8
:104AD00019FF10BDF0B585B0039203220333DC1734
:104AE000294D1440E4182B68284F5A425341802224
:104AF0005B42D202A4103B409B18A21C0291244EA0
:104B0000910000910190316800980A18934215D2E3
:104B1000FFF7F8FE2B685A42534180225B421F4048
:104B2000D202BF183368009A9B189F4206D21948D8
:104B300000F086FE0025280005B0F0BD029B356818
:104B400019066B461A7BA423DB051343FF222F00B3
:104B5000090C1943019B12041B041340194328003C
:104B6000FFF75CFD0837281D21003760FFF756FD71
:104B7000002C04D00A9A21003800FFF775FD009B35
:104B8000083BFF183760D6E70411002000C0FEFF85
:104B900008110020CBD6000070B59AB0FFF74AFE8E
:104BA000FF221E4CD2000021200006F073FDFF25DD
:104BB000FFF794FE0026002814D10200C300E3583A
:104BC0000130591E8B41D218FF28F7D1144901A892
:104BD00007F0A4F801A800F033FE124800F030FE00
:104BE0001AB070BD03681A142A400A2A0AD11A1290
:104BF0002A40FF2A03D0D200A1180B71A050FFF762
:104C000061FDD8E7132AFAD11B122B40FF2BF6D0F7
:104C1000DB00E2181671E650F1E7C0469C25002043
:104C200097D70000ABD700000021094B094A596013
:104C30000131516059680029FCD00021196101231C
:104C400093600222044B8131FF315A501A60704741
:104C5000FC1000400010004000E100E00222064B82
:104C60000121DA670022054B5A61054A11615A6930
:104C7000002AFCD07047C04604E100E0FC10004070
:104C80000010004010B5044C2378002B01D0FFF732
:104C9000E5FF0020207010BD0D12002080230120B0
:104CA0005B055B6E5B001843704700000120024B00
:104CB0001B685B0018437047901200200120024BD4
:104CC0001B685B0018437047240000200120024B42
:104CD0001B685B00184370479412002070B50400F5
:104CE0000D001600FEF754F9802301215B055A6E72
:104CF0002670002653006170E1706272010A5A0A40
:104D00006071A171A272010C5A0C000E5B0EA670AC
:104D10002571E1712072E272237370BD10B5044CED
:104D2000200007F041F801002000FEF7F9FD10BD5A
:104D3000991200200E4B10B51B680E4C5A1C0FD058
:104D40000D4C002B0CD00D4C012B09D00C4C022B20
:104D500006D0094C042B03D00A4C052B00D1074C7C
:104D6000200007F021F801002000FEF7D9FD10BD5A
:104D7000280000203CD80000C4D0000047D8000024
:104D8000CBD0000041D8000070B5214C2278002A19
:104D90003DD1204B01215A608022D20511605A6812
:104DA000002AFCD0002207201B4B1C4901255A5029
:104DB0000439585008315A5019481A4958501A495C
:104DC0001A485A501A495A50A622D2009D50082219
:104DD00018495A5004315850022017495850174961
:104DE0001748585017480439585018201649585039
:104DF000C12189005A500539FF3958589218024389
:104E00005A501249124A9950FFF70EFF257070BD93
:104E10000D120020FC000040001000400C050000B6
:104E2000746962751C05000024050000200004025E
:104E30002C05000014050000340500003C050000AE
:104E4000FFFF000021100100540500000E12002099
:104E50000405000070B50E4B06001B78002B01D135
:104E6000FFF792FF00200B4D2C7884420ED00A4BA6
:104E7000202219780323091B1940084B4901C9183E
:104E8000300006F0EBFB0120013C2C7070BDC046E9
:104E90000D120020981200200C1200200E1200208B
:104EA000002370B588B0984235DD0D6801262C00CE
:104EB00034409C422FD12300042D2CD90F222B6883
:104EC0001A402300092A26D16A683F2A23DD684652
:104ED000FFF7C0FF230000281DD06B461978330070
:104EE000A14203DB6B461B5D5B003343A200AA18A3
:104EF00001349360202CF2D1092169444A780B785F
:104F000012021A438B781B041A43CB781B061343F7
:104F1000024A13600423180008B070BD94120020E8
:104F200070B5454B8AB01B78002B01D1FFF72CFFE1
:104F300002AC2000FFF78EFF002802D100200AB04B
:104F400070BD23780B2BF9D96378012BF6D1E37868
:104F5000012BF3D100231120384E394D33602B70D3
:104F600068442379374A4178136002780902114373
:104F7000827812041143C27812060A4332490A6049
:104F8000002B0ED1152169444A780B7812021A437E
:104F90008B781B041A43CB781B0613433360002322
:104FA00018E0012B1AD1152169444A780B781202B6
:104FB0001A438B781B041A43CB781A211B06134320
:104FC00033600E23627C6944934200DD13000022AB
:104FD0009A422CD100220420EA54B0E7022B03D1DC
:104FE000627B10331621EEE7042B0DD11521082228
:104FF0006944684606F032FB0098019902F0BCFD56
:1050000006F0DEF93060CAE7052BC8D11521082269
:105010006944684606F022FB0098019902F0ACFD55
:1050200006F0CEF93060627D0A231E21CBE7885C52
:10503000A8540132CCE7C0460D1200209012002087
:1050400099120020280000209412002010B5134B64
:1050500004001B78002B01D1FFF796FEFFF7FEFD41
:1050600000200F4A0F49104B545058600130106017
:1050700058680028FCD00020186101309060186941
:105080000028FCD0094B0A481B785B011B185350C1
:10509000FFF7E4FDFFF7C8FD10BDC0460D1200206C
:1050A0000010004004050000FC1000400C1200201D
:1050B0000E12002010B588B000281DDD0A680121FD
:1050C00013000B4018D1042A16D90F201468204071
:1050D000092811D150683F280EDD9800101880680B
:1050E0000024084201D04010C4B26846C4540133C1
:1050F000202BF2D1FFF7AAFF002008B010BD00005E
:1051000010B5002813DD0C68E30710D56410532C8C
:105110000DD8084B1B78002B01D1FFF735FEFFF7A8
:105120009DFDA123044ADB00D450FFF77DFD002044
:1051300010BDC0460D1200200010004010B5002820
:105140000EDD0C68E3070BD56410FF2C08D8054B67
:105150001B78002B01D1FFF717FE034A034BD450F5
:10516000002010BD0D12002000100040240500009A
:1051700013B5002814DD0C68E30711D5094B641042
:105180000093094B0193072C0AD8084B1B78002B7E
:1051900001D1FFF7F9FD6B46054A1957054BD15070
:1051A000002016BDE2ECF0F4F8FC00040D12002023
:1051B000001000400C05000070B588B0002820DD0C
:1051C0000124086804401CD104281AD90F2302685E
:1051D0001340042B15D1FEF783F9060006F0E4FD19
:1051E0000500122800D912252A0002210D32684636
:1051F000FFF774FD6B465D73A54205DC6846FFF75B
:1052000025FF002008B070BD2300325D6B449A7307
:105210000134F1E7F0B50D008BB0012832DD0868EC
:105220000122040014402DD104282BD90F2301683A
:105230000B40042B26D16B68134223D0FEF750F9A4
:105240006E6807007310019306F0AEFD05000E288E
:1052500000D90E252A000121113202A8FFF73EFDD8
:105260006A46127902AB5A7302AA73129373019BB6
:1052700076141B0ED67313745574A54205DC02A870
:10528000FFF7E4FE00200BB0F0BD3A5D02A9631801
:105290009A740134F1E730B589B0002814DD0C6848
:1052A000E30711D5102268460021FFF717FD6B4672
:1052B0006A4665105D73684663122D0E641493731D
:1052C000D4731574FFF7C2FE002009B030BD000092
:1052D000174B184A5968002903D000215960013141
:1052E0009160196900291FD0002018618023DB001C
:1052F000D3581149012B18D1A923DB00D3585B42A5
:105300000B600E490B78032B01D801330B7003207F
:105310000B490B78013303400B700A495B015B18A2
:10532000094953500123936070470860FAE7C0466B
:10533000FC100040001000402400002098120020C3
:105340000C1200200E1200200405000010B5034AC4
:105350001021034800F07EF810BDC046BCD7000005
:10536000B3D70000044A05491368C85401339B05AC
:105370009B0D13607047C046C8160020C81200205D
:1053800070B5114C114A2368834202DC002323606C
:1053900016E0155C411C2E00FA3E012E05D89942FC
:1053A0000FDA555C013D1F2D01D90800ECE7010023
:1053B000151A565C6E5401318B42FADC181A2060C3
:1053C00070BD1570FAE7C046D41A0020D41600202C
:1053D00010B5FDF7D3FD064B1A68824201D90022B1
:1053E0001A601B68C31A034898428041404210BDAE
:1053F000C4120020204E000010B5094C094A236851
:105400001268934200D110BD074AD05CFDF7EAFF55
:105410000028F8D0236801339B059B0D2360ECE73F
:10542000CC160020C8160020C812002010B50400B9
:10543000064B074A1B6812689B1ADB439B059B0DB2
:10544000A34200DB10BDFFF7D7FFF1E7C81600202D
:10545000CC16002070B5074E33680B2B08DC0C25EA
:105460005D43054C0133285164196160A2603360CB
:1054700070BDC046D0160020342F002010B5FBF7B9
:105480001DFEFFF77FF8FBF741FEFDF73FFFFEF73C
:10549000F7FBFEF735FCFFF759FF00F067FF01F05F
:1054A0006FF901F0B9FB10BD962210B51201002171
:1054B000034806F0EFF80022024B1A6010BDC04608
:1054C0003C1C0020D0050020064B074A1B681268D0
:1054D0009B1ADB439B059B0D0122834200DC0022CB
:1054E00010007047C8160020CC160020F8B5050043
:1054F0000C0016001F1E0ED10320FFF7E5FF002849
:1055000008D0FA20FFF72EFFE8B2FFF72BFFE0B23A
:10551000FFF728FFF8BD501DFFF7D6FF0028F9D090
:10552000FB20FFF71FFFE8B2FFF71CFFE0B2FFF719
:1055300019FFF0B2FFF716FF3012C0B2FFF712FFEB
:105540003C00E31B9E42E5DD2078FFF70BFF0134B2
:10555000F7E7000070B50024F0250B4B1B68A34251
:1055600002DCFFF7A1FF70BD2B006343074A9B18C5
:105570001A78002A05D05978002311201A00FFF765
:10558000B5FF0134E9E7C046D00500203C1C0020EF
:10559000F8B507000024F0252B0063430C4A0134C2
:1055A0009E18B74211D0317800290BD00133D15C5D
:1055B000002311201A00FFF799FF2A000021300074
:1055C00006F068F80A2CE7D1F8BD024B1C60F9E739
:1055D0003C1C0020D0050020F0B5150001222F0052
:1055E000754C1740A54401900291002F11D005ABD6
:1055F0001A706A105A70120E1A7105226912997087
:105600006D140299DD70FFF771FFCF239B009D445D
:10561000F0BD042D1ED90F202A681040042826D181
:10562000022304AA28001371FDF75AFF040006F0B4
:10563000BBFB624B984200D91800B84204DC421C04
:1056400005AB02990198DEE701377B1EE35C05AAF2
:10565000D355F2E7042D00D0A9E0032304AA043DAA
:1056600013716B425D4105AB55710222E9E70928D0
:105670007ED1042205AB1A706A6851100091694608
:10568000521209789A70009A59701F2A01DD20225F
:1056900000926A46127806ACDA70009BBB4202DCCC
:1056A00005ABE21ACDE70126BB00EB18986806406F
:1056B00006D1042837D90F210368194002290CD1DB
:1056C000012323704310637042121B0E4014A2701A
:1056D000E070237105340137DFE7042921D102236B
:1056E0002370FDF7FDFE039006F05EFBA31C0C2863
:1056F00009D86070864201D19C19ECE7039A925D4B
:105700009A550136F6E70C226270039A925D9A551B
:105710000136092EF9D12E23E372237363730E34FD
:10572000D9E7012907D103230438237043425841A4
:1057300060700234CFE7092909D10423237043683C
:105740005A1062705B12A370E6700434C3E7032939
:105750000BD1052323700068020992B2430F920017
:105760000B40D31A63701B12EDE726700134B2E7C9
:10577000032800D049E7052105AB1970110989B24A
:10578000520F890002408A1A111299705A70110042
:10579000642A00DD64210420D970C9B2041FA1422B
:1057A00001DC04324DE72C5C1C540130F6E7002D7F
:1057B00000D02AE751E7C046C4FCFFFF23030000E6
:1057C00070B502000024F0210D4E080060438019DE
:1057D0004578954203D001340A2CF6D170BDF022F1
:1057E000002105F057FF074A1368013BA34200D18F
:1057F0001460002329001A001120FFF777FEEDE75F
:105800003C1C0020D005002010B5B2B002236A462F
:105810000400137006F0C8FAC72800D9C720002377
:10582000984207DC421C6B46FE211420FFF75EFE07
:1058300032B010BD694601335A1EA25CCA54EFE76C
:1058400030B5B3B002236A460500137006F0ACFA17
:105850000400C72800D9C72400239C420BDC200089
:105860003230FFF7E3FD621C6B46FF211420FFF787
:105870003DFE33B030BD694601335A1EAA5CCA549E
:10588000EBE70000F0B5BBB004900C00012803DC8E
:105890001B20FBF711FD51E02A4B08680293C30758
:1058A00009D4042807D90F2302681340042B02D11E
:1058B000FDF716FE0290234B60680393C30709D4DB
:1058C000042807D90F2302681340042B02D1FDF7E7
:1058D00007FE039000271C4B1B680693069BBB42E8
:1058E0000BDC039B194A0093C821029B08A806F011
:1058F000E3F908A8FFF7A4FFCAE70C267E43144B80
:105900000299F618306806F045FA051E05D173684D
:10591000B6680793079B9D4201DB0137DEE73068DD
:105920000399059606F036FA0836002808D12100BA
:105930000498059B083102385B6898473BB0F0BD7E
:105940000135E7E7C8D10000D016002018D90000C3
:10595000342F0020F7B5234B06001B68F02100937D
:105960000023009A9A4211DC0024F0231A006243BB
:10597000019201991C4A55182F78002F12D001343A
:105980000A2CF3D11948FFF75BFF29E00A005A43BC
:10599000154882185078B04202D11278002A1FD1DF
:1059A0000133DEE7F0223900280005F073FE022300
:1059B0000D4A0199EB6053540D4AF1008A58009B3F
:1059C0006E70AE70AA602F616F61A34202DC054B5E
:1059D00001341C60002331001A001020FFF786FDFF
:1059E000F7BDC046D00500203C1C002061DD000052
:1059F0009C25002010B5FFF7ADFDFF24084AE30009
:105A00005B429B18074AD35C043B012B03D8E0435D
:105A1000C0B2FFF79FFF013C002CEFD110BDC04684
:105A2000FC0700009C250020F7B50F00FF247F2510
:105A300001901E4AE300D31A1D4A9A181278062ACA
:105A400001D0032A20D1FF22D2009B181868836856
:105A50002B401C2B18D1C3681A002A40042A13D1EA
:105A600002692A40192A0FD11B0A01339B000C300E
:105A7000C018FDF735FD03780600002B10D006F0A6
:105A800093F90023B84209D0013C002CD1D1F7BDD5
:105A9000019AF15CD25C9142F6D101339F42F7DC6E
:105AA000E043C0B2FFF756FFEEE7C0469C2500205A
:105AB000FC07000070B50500FF24084AE3005B42C4
:105AC0009B18074AD35CAB4203D1E043C0B2FFF757
:105AD00041FF013C002CF0D170BDC046FC07000026
:105AE0009C250020F7B5FDF749FA574B1A6882420A
:105AF00001D900221A601A685449821A8A420DD9C3
:105B0000FF2253491860D3005248CB1A1B181B7848
:105B1000073B022B0CD9013A002AF4D1F7BD07202C
:105B2000FFF7C8FF4C4B27E00820FFF7C3FF38E022
:105B3000FDF72EFA071E00D101270020FDF71EFBFE
:105B400001900020FDF72EFB019B0090434C444D3B
:105B5000002B12D02368002B6ED12B682760002BFE
:105B60006ED0404B01261B78002BD8D10920FFF7BF
:105B7000A1FF394B1E703B4B1E70009B002B12D0B7
:105B80002B68002B0FD123682F60002B1ED0324BC7
:105B900001261B78002BC7D10920FFF78BFF2E4B66
:105BA0001E70304B1E702368002B0FD02A4E3278A7
:105BB000002A0BD19F4200D227602368FB1A312BA9
:105BC00004D90720FFF776FF012333702B68002BE1
:105BD0000FD0244E3278002A0BD1BB4200D92F605F
:105BE0002B68FF1A312F04D90820FFF763FF012328
:105BF00033702368002B0CD0019B002B09D1164E6B
:105C00003378002B02D10720FFF754FF00232360D5
:105C100033702B68002B00D180E7009B002B00D055
:105C20007CE7104C2378002B02D10820FFF742FFBD
:105C300000232B60237071E7009A002AA0D1B5E7FA
:105C4000009B002B9FD1AEE7C01200200F27000061
:105C50009C250020FC070000B4120020B012002098
:105C6000B8120020BC12002037B500240500FFF751
:105C700071FC01A80194FDF76FFA21002000FEF7E6
:105C80002DF9FEF72DFBFDF7A1FAFDF71BFBFDF744
:105C900035FBFEF771FCFDF797F9A54204D0FDF73F
:105CA000CBFB0248FFF7CCFD37BDC04652DD0000FC
:105CB000002310B501001A001120FFF717FC10BDDA
:105CC00007B56B46197069465A7013128B7013141E
:105CD000120ECB700A716B46010005221320FFF7EC
:105CE00005FC07BD10B50A0001001220FFF774FC87
:105CF00010BD70B5050008000C003230FFF796FBB0
:105D00002B00220000211B20FFF7F0FB70BD10B517
:105D10000C000300110014202200FFF7E7FB10BD68
:105D2000012370B5FF24084A41185B42884201D321
:105D3000D84370BD06781D0A234073409B009B58D2
:105D400001306B40F2E7C04634D9000013B50400BF
:105D5000FE2813D80A4BC200D05800280ED0436842
:105D600008309900FFF7DCFF01900920FFF75EFB88
:105D700001AB042221001720FFF7B8FB13BDC0467A
:105D80009C250020F7B50190FEF7A8FD0125040031
:105D9000FF276D42002C01D12800FEBD2668331478
:105DA0003B40152B0DD121000198083105F0F2FF81
:105DB000002801D135123D402000FEF783FC04008D
:105DC000E8E71D2BF8D101256D42F5E7F0B58027F6
:105DD0009FB0FFF711FBB54CB54D2068FF00391A95
:105DE0004019FDF7E5FA23680600C3182360002B6D
:105DF0000ED11FB0F0BD2068391A2818FDF7D8FA67
:105E0000236806001B182360FDF7B8F8A94B18603B
:105E1000002EF0DC2B78FA2B00D00EE12368022B49
:105E200007DCFFF7D5FA0028E3D00120FFF7A8FA36
:105E3000DFE76B78AC78981E182800D9F2E003F001
:105E400051FA0D2024282B34F13E707A7E94CDDE59
:105E5000F1F1F1F1F1F1F1F1F1F1EC00FF2C0ED0E3
:105E60002000FFF7ADFC0022934BE100CA505B1805
:105E70001A712100009213001320FEF72BFE03205D
:105E8000D4E72000FFF766FDF9E72000FFF798FC54
:105E9000F5E7FFF7AFFDF2E7FFF75CFB0020FFF748
:105EA000E3FE8648FFF7CCFCE9E7632CE7D8844B98
:105EB000A200D25821001520FFF78EFBDFE7FEF786
:105EC0000DFDFF270400002CD9D025682B143B4082
:105ED000152B04D02000FEF7F5FB0400F3E72000AB
:105EE000083005F061FF06000530FFF79FFAFB2040
:105EF000FFF738FA2D121D20FFF734FAE8B2FFF74A
:105F000031FAF0B2FFF72EFA3012C0B2FFF72AFAD8
:105F100025002B1B9E42DDDD287AFFF723FA013591
:105F2000F7E700211D2000910B000A00FEF7D2FDCB
:105F3000FDF782FAA3E72000FFF708FF9FE7FDF7D0
:105F40002FF805AC5F4A642100905F4B200005F0FC
:105F5000B3FE02232000237005F026FF2300020079
:105F600000211620FFF7C2FA89E70026524AF30003
:105F70009B181C68002C28D01B7903936368083495
:105F80009F00B81D0293FFF751FAFB20FFF7EAF9D3
:105F900001207D1CFFF7E6F9F0B2FFF7E3F9E8B264
:105FA0002D12FFF7DFF9E8B2FFF7DCF90398FFF7EE
:105FB000D9F9E719A7420CD8FFF71EFA0523029872
:105FC000584301F063FBFFF717FA0136FF2ECDD1DE
:105FD00055E72078FFF7C6F90134EBE70024FFF717
:105FE000B9FA2200210000942300DA20FEF772FDA6
:105FF000FF222100D200304805F04CFB98E7012C2D
:1060000002D1FEF789FB3AE7022C02D1FEF75EFDD2
:1060100035E70120FFF728FE31E7002321001A00B1
:106020001A209FE71A00C83A052A00D927E700225C
:1060300018001100FBF776F821E7FB2B00D0F4E6FF
:106040002268042A00DCECE62E79E8781F4B360241
:1060500006439E4200DDE8E6331D9A4200DCE0E69E
:10606000EB5CFE2B00D0E0E66878AC78771E1B284E
:1060700000D17DE02ED8072863D0082838D0012829
:106080002DD1FF2C10D02000FFF79AFB6D79104A1C
:10609000B31E009221002A000A20FEF71BFD064BCA
:1060A000E400E0501B191D71701DBFE6D41A0020DA
:1060B000D4160020C41200209C25002034DD0000EE
:1060C000942D00204BDD000046DD0000F6030000AB
:1060D000DA1600201D285DD04FD31E2871D0030092
:1060E000C83B052BE0D8404A3900FBF71BF8DBE73B
:1060F000632CD9D86A79022A13D0032A1BD0012A2B
:10610000D2D1E979AB79090219432B7AA4001B0497
:1061100019436B7A1B060B435B001343334AA350AE
:10612000C2E7002FC0DDB11E3148FDF7F9FB2F4B50
:10613000A400E050B8E7AB79A4005A1E93419B003D
:10614000ECE7632FB0DC05AD3A002749280005F0E5
:1061500085FA00232800EB55FFF714FE0028A3DB87
:10616000224B8000C25821001520FFF735FA9BE72B
:1061700039001D48FFF758FC96E7FF2C94D06A7948
:10618000022A91D81A490B2000912100B31EFEF774
:10619000A1FC89E7632F00DD6327002305A9BB422B
:1061A0000ADBFB430022DB173B40CB181A7015209B
:1061B00000917B1C2100EAE7EA185279CA540133A6
:1061C000EDE7012C00D06FE7002F00DC6CE76B7966
:1061D000002B03D01C00322B00DD322464235C43EF
:1061E000044B1C6060E7C046D9160020942D0020A7
:1061F000DA160020040000200122094B1A60094A27
:106200001368002BFCD00322074B1B68D8171040E3
:10621000C018012380100638400018437047C0465C
:1062200000C0004000C1004008C500400120704788
:1062300010B5064C200000F01FFE0549200000F0BC
:106240005DFE0122034B1A6010BDC0460C1B0020EE
:10625000801A0600D81A002010B501210D20FCF785
:10626000A5FE01210E20FCF7A1FE00210F20FCF766
:106270009DFE044C200000F041FD1021200000F0A4
:1062800059FD10BDEC1A0020F8B501250C682C4210
:1062900003D10D20FBF710F8F8BD64102DD4FCF7E6
:1062A00083FEA04229DB00212000FCF77FFEFA22BA
:1062B0002900D200200001F01BFA00281DD0002583
:1062C00000270726FA2201219200200001F010FA8F
:1062D000002812D0282802DD0123B3401F43013ECD
:1062E000F0D20E4EAF550135052DE9D10122062120
:1062F0000920FDF797FA002801D10020CCE70B23F5
:10630000012443600023F25C9900520041182243AB
:1063100001338A60052BF6D1BEE7C046DC1A0020A7
:106320000120704710B504680D20E30703D5641001
:10633000FF2C03D91720FAF7BFFF10BDFFF78CFF22
:10634000E1B2024800F018FD0020F6E7EC1A002048
:1063500010B5FFF781FF0021034800F00DFD430059
:106360000120184310BDC046EC1A002010B5034AA6
:106370000A210348FFF76EF810BDC04678DD000023
:10638000C8DD00000D4B70B51B6804000E00150041
:10639000002B01D1FFF74CFFE1B2094C200000F0C7
:1063A00044FEF1B2200000F033FDE9B2200000F01D
:1063B0002FFD200000F0A4FE70BDC046D81A0020BA
:1063C0000C1B002010B501240368234205D041684E
:1063D000214202D08268224203D10D20FAF76CFFDD
:1063E00010BD5810802801D91520F7E74910FF2962
:1063F00001D91620F2E75210FF2A01D91720EDE744
:10640000FFF7C0FF0020EBE7F7B501221400904230
:1064100022DD0D682A421FD01D4B15411B684C68B8
:10642000002B01D1FFF704FFE9B201272500194E27
:106430003D40300000F0F9FD002D0FD03C41300010
:10644000E1B200F0E5FC300000F05AFE0024A0426A
:1064500002D02320FAF730FF2000FEBD042CF2D931
:106460000F2322681340092BEDD163685B10019361
:10647000019BAB42E7DDAB00E3189968394204D0D9
:106480004910C9B2300000F0C3FC0135F0E7C04646
:10649000D81A00200C1B0020154B70B51B68050096
:1064A0000E00002B01D1FFF7C3FE124CEDB2290004
:1064B000200000F0BAFDF1B2200000F0A9FC00219C
:1064C000200000F0BDFD002801D0404270BD72B632
:1064D00001222900200000F0A3FD62B6200000F098
:1064E00088FC0028F2D0200000F088FCEEE7C046CF
:1064F000D81A00200C1B002010B501240368234289
:1065000002D04168214203D10D20FAF7D5FE10BD1B
:106510005810802801D91520F7E74910FF2901D923
:106520001620F2E7FFF7B8FF40002043EFE7000036
:1065300010B50D211D20FFF7AFFF164C5A2809D1C9
:1065400001222A2122703D38FFF71CFF0122124B45
:106550001A6010BD0F211920FFF79EFF332805D1C7
:1065600002235F22237020211A38EDE70D211E201F
:10657000FFF792FFC7280AD1032300222A21A93856
:106580002370FFF7FFFE1B222A211E20DCE70023D9
:106590002370DBE72C000020E41A0020204B10B50C
:1065A0001B680400002B01D1FFF7C2FF1D4B1B78B5
:1065B0005BB2022B0AD0032B29D0012B2CD1210056
:1065C0001D200124FFF768FF644205E0012C13D170
:1065D00029211920FFF760FF7F2801DD0138FF38EE
:1065E00003007F3301DA7F204042C8237F215843D4
:1065F00002F00CFF604310BD032C0BD12B2119209E
:10660000FFF74AFF043CE7E72D211920D9E72100D5
:106610001E20D6E7052CF7D0012400206442E4E7D1
:10662000E41A00202C00002010B50120FFF7B6FF6F
:1066300043000120184310BD10B50320FFF7AEFF43
:1066400043000120184310BD10B50520FFF7A6FF39
:1066500043000120184310BD144B70B51B68002B7C
:1066600002D10120FFF79AFF114B1B785BB2013377
:1066700001D1FFF75DFF0120FFF790FF0400032029
:10668000FFF78CFF05000520FFF788FF6D4364438B
:1066900040436419201804F0C9FE01F09DFB04F08A
:1066A0008FFE43000120184370BDC046E41A00204D
:1066B0002C000020F8B501231C0098422BDD0F6848
:1066C0003B4228D04E6835001D4024D1042E22D9EB
:1066D0000F2231680A40092A1DD173685C10202CF2
:1066E00000DD2024144B1B68002B01D1FFF7A0FD17
:1066F00072B67F10F9B2114F2200380000F090FC02
:1067000062B6A54214DA380000F073FB002804D109
:1067100001246D002C432000F8BD380000F06EFB12
:106720000122AB004000F31810439860AD18E8E771
:1067300064000125EEE7C046D81A00200C1B00209B
:1067400000207047012070470020704700207047EC
:1067500001207047002070470020704700207047DC
:1067600000207047002070470020704700207047CD
:106770000020704700207047704770477047000046
:1067800010B5034A0E210348FEF764FE10BDC04653
:106790002CDE00009CDE00000378013B1F2B00D99B
:1067A00070470130F8E710B5FFF7F6FF0378002BCC
:1067B0000BD00130222B11D10378002B03D0421CC7
:1067C000222B03D11000FFF7E7FF10BD5C2B03D194
:1067D0004378002B00D0821C1000EDE73A2BF2D05A
:1067E0002C2BF0D07B2B0BD1FFF7D6FF0378002B9F
:1067F000E9D07D2B01D10130E5E7FFF7D4FFF5E7C4
:1068000020225B2B14D1FFF7C7FF0378002BDAD0CF
:106810005D2BF0D0FFF7C7FFF7E7202BD3DD2C2B44
:10682000D3D0190091435D29CFD0222BCDD0013098
:106830000378002BF1D1C6E7002210B5904216D0A4
:10684000FFF7AAFF03780422222B10D0023A7B2BF9
:106850000DD0013A5B2B0AD01900303902320929D8
:1068600005D92D2B05D14178303909290AD81000D6
:1068700010BD0522742BFAD00132662BF7D00132FD
:106880006E2BF4D0581E83415A42F0E770B5FFF7E3
:1068900083FF037801222D2B01D18018023A0023B7
:1068A0000A2502E06B430130CB1801783039CCB2B5
:1068B000092CF7D95A43100070BDF8B50C0015002B
:1068C000FFF76AFF0378222B02D000232370F8BD64
:1068D0000D236A1E210008250C260A279C4601303C
:1068E0000378222B02D100230B70F0E7002BFAD0A3
:1068F000441C5C2B0BD14378841C622B0ED0662B7E
:106900000ED06E2B0ED0722B0ED0742B0ED0002A10
:10691000E9DD0B70013A01312000E1E72B00F6E7D9
:106920003300F4E73B00F2E76346F0E70923EEE7C4
:1069300010B50400FFF737FFA04202D90378202BDF
:1069400000D910BD0138F7E710B5002815D003783D
:10695000002B13D0FFF720FF2021037802008B4388
:1069600000205D2B09D01000FFF71DFF03782C3BA2
:106970005A425341C018FFF70FFF10BD1800FCE743
:106980000300002070B50C0081420EDD1A785B2AEE
:106990000BD1581CFFF700FF0125AC4205D0FFF7D3
:1069A000D3FF002801D00135F7E770BD70B50C00AA
:1069B0001500002901D000230B70002820D0037897
:1069C000002B1ED0FFF7E8FE037806002C2B03D126
:1069D0000130FFF7E1FE0600337800207D2B0FD059
:1069E000844204D02A0021003000FFF766FF300007
:1069F000FFF7D9FE03783A2B02D10130FFF7CCFE26
:106A000070BD1800FCE7F0B50D0004009DB02E78B5
:106A1000002E35D02E21280005F0AEF9071E14D027
:106A2000431B0193303E092E14D82800FFF72EFF98
:106A300001002000FFF7A4FF0400002C20D0002F4D
:106A40001ED0019B0133ED18E1E7280005F0ACF9F9
:106A50000190E7E723787B2B11D1601C642203A906
:106A6000FFF7A4FF041E0BD0019A290003A805F02C
:106A7000A2F90028E1D02000FFF795FEEEE7002400
:106A800020001DB0F0BD70B5050000200C00814253
:106A90001DDD2800FFF7D0FE0300681C012B14D079
:106AA0000020022B13D10022681C1100FFF77EFF8B
:106AB000012C0CD0FFF748FF00221100FFF776FFF2
:106AC000013CF5E7FFF740FF013C012CFAD170BD16
:106AD000F8B5050000200C0016001F0081420DDDF6
:106AE0002800FFF7A9FE03000020022B06D1681C36
:106AF0003A003100FFF75AFF012C00D1F8BDFFF733
:106B000023FF3A003100FFF751FF013CF4E710B5D5
:106B10000024A04218D0FFF73FFE03787B2B0AD158
:106B2000013000221100FFF741FF00280CD0FFF7D1
:106B30003AFE0134F5E75B2B06D10130FFF704FF85
:106B4000002801D00134F9E7200010BDF8B5002875
:106B500016DD0D68EB0713D56D10013D0124FDF71F
:106B6000BDFE0026FF27644200280CD1002E21D054
:106B7000300005F019F901003000FCF7D1FEF8BD36
:106B800001256D42EAE703681A143A40152A0BD131
:106B90001B123B409C4200DA1C009D4201D10600C2
:106BA0000836FDF78FFDDFE71D2AFAD10124002604
:106BB0006442F6E70120013464002043DFE700006F
:106BC00010B508680C00FCF78BFCFFF7DBF8002819
:106BD00003DB6268024B8000C250002010BDC0463B
:106BE000942D002010B50868FCF77AFCFFF7CAF86E
:106BF0000123002802DB024B8000C358180010BD9F
:106C0000942D002010B50868FCF76AFCFFF7BAF86D
:106C1000C043C00F800010BD10B5034A04210348D3
:106C2000FEF718FC10BDC0462CDF000025DF000079
:106C300010B5FCF777FBFCF725FCFEF71FFC0448BA
:106C4000FEF7FEFDFDF7A8FFFEF7D4FE10BDC0461F
:106C50007BDF000010B5FCF769F810BD70B50025AA
:106C600004AC24780573A94205D10A4B0A4A2321B2
:106C70000A4804F085FC01600949920052589B00C3
:106C800002715B58A40083716358856043710223CD
:106C9000C37170BD93DF0000F2DF0000A1DF0000D0
:106CA00050E00000037B002B04D143738373036126
:106CB00001330373704700001FB50191A021002428
:106CC0000068C900D2B24450012A10D0A24209D0B3
:106CD000032A0AD0074A8350074B019AC250012366
:106CE00043501FBD02221343F4E70422FBE70622B0
:106CF000F9E7C046540500002405000010B5040063
:106D0000FFF7D0FFA1222368A179D20099506179C1
:106D1000064A20009950217904329950044B196891
:106D20005A689B68FFF7C8FF10BDC0460C050000FD
:106D3000001B00204BB2002B0FDB80233F290FD814
:106D40001F290FD80F290FD807290FD803290FD8CB
:106D50001B060168074A8B50704780239B04F8E7A5
:106D6000DB04F6E71B05F4E75B05F2E79B05F0E7BC
:106D7000DB05EEE7240500000368074A99501A0076
:106D8000FC32D1680029FCD0A321C9005858002347
:106D9000C0B2D3607047C0461C05000007B5802212
:106DA000074BD2051A6000229A6002321A710F2333
:106DB0000C3200930349023B0348FFF74FFF07BD26
:106DC000001B002000300040EC1A0020F8B5050040
:106DD0000E0017000024BC4208D02B68315D1B68F0
:106DE00028009847002801D00134F4E72000F8BDBE
:106DF000704710B51C3000F0BDF910BD10B51C3047
:106E000000F0AAF910BD10B51C3000F0B9F910BDA2
:106E100070B5437E0D00002B01D1002070BD6430A1
:106E2000040000F0B6F90028F7D12000290000F096
:106E300084F90120F2E70000F7B50193FA23002559
:106E400004009B0083600B4B4560083303601C30DB
:106E50000F00160000F066F92000643000F062F9BF
:106E60006B461B79276166756576A5762000A3754C
:106E7000FEBDC04630E000000123827DC3751B4B80
:106E80009200F0B5D4582022210011404D1EA94196
:106E9000457DC026AD005D59A0272A40531E9A416A
:106EA00053421F2214402A402500B6004942C135F2
:106EB000FF0531403340FF350D4EC919AD006E500E
:106EC0001100C131FF31DB198900CE50CC21056999
:106ED000084B4904E95005210569243BE950016943
:106EE0000833CC500169044BCA50F0BD50E000009B
:106EF0000C060000240500000C050000A022002361
:106F000010B50469D200A3500A4CA1420FD90A4C13
:106F10008C425B4109495B420B40CD21C9045B189F
:106F200004690749635005210369995010BDCC23BA
:106F30005B04F5E7A086010090D00300000098FDF7
:106F400024050000F7B5040000200D0001938242E3
:106F500065D01600402A00D9402627001C3738008B
:106F600000F0F6F8B1232269DB00D550802201231E
:106F7000216992008B50A27E002A03D122691362FC
:106F8000226913600025731EAB4207D1019B002BC1
:106F900004D08022022123699200995001222369A2
:106FA0001A622369FC33DA68002A02D19A6A002A3D
:106FB000F9D09A6A002A0BD1DA60A3232269DB0098
:106FC000D1583800C9B2013500F0B7F8B542DAD36C
:106FD000019B2269002B0FD11300FC339B6A002B0D
:106FE0000AD10133A376D3612369FC33DA6C002A1A
:106FF000FCD00022DA640AE000230121A37651616B
:107000001A002369FC3399680029FCD09A6023692F
:10701000FC339A6A002A01D000229A62E8B2FEBDCF
:1070200010B50123FFF78EFF10BD0300AC3310B580
:1070300004001970643000F08BF80123637610BDF2
:107040000023020070B5AC3243760D001178B122F6
:1070500004000069D20081508022216992008B5087
:10706000226901331362226993602600643630007E
:1070700000F080F8002812D0300000F06DF81E4BB0
:107080002269D0502369FC331A6A002A02D19A6A15
:10709000002AF9D09A6A002A01D11A62E5E7236929
:1070A0000122002D0DD11900FC31896A002908D177
:1070B000DA612369FC33DA6C002AFCD00022DA643E
:1070C00007E05A612369FC339A68002AFCD0002249
:1070D0009A6000202369FC339A6A82420BD098623E
:1070E0002169064A8B588B501800022B03D0181FB9
:1070F000431E9841033070BD1C050000C40400000D
:1071000010B50121FFF79CFF10BD000010B513233F
:10711000142202490248FFF78FFE10BD00400040D4
:107120000C1B002010B540220021040004F0B2FA2C
:10713000002320002364636410BD10B53F24026C5B
:10714000531C2340446C9C4201D08154036410BD05
:107150000023036443647047436C026C934206D07F
:107160003F21C25C01330B40436410007047012093
:107170004042FBE7036C406C181A00D54030704762
:10718000436C026C934201D0C05C704701204042C6
:10719000FBE73F22036C406C01331340181A434253
:1071A0005841C0B27047000003210A4802680A43F0
:1071B0000260094802680A4302600849084A094B0C
:1071C0009B1A03DD043BC858D050FBDC00F012F8DA
:1071D000F8F79AFF2405004054050040A4E500009C
:1071E0000000002068020020FEE7FEE7FEE7FEE761
:1071F000FEE7FEE72D4B10B51A68D2B2012A0FD177
:107200002B4A126812070BD12A4AE0241168F02297
:107210000800104021422DD12749096811422CD085
:107220001A68D2B2012A12D12149096809070ED180
:10723000F020204909680140402908D11E49096809
:10724000014204D18020C121C005C90042501B6801
:10725000DBB2012B0DD1164B1B681B0709D1154B57
:107260001A68F0231A40A02A0FD1134A12681A4252
:107270000ED010BD3028CFD0D2E7104A104911608F
:107280008021104A09021160CAE7D02AF1D1ECE747
:107290000D4B1A68012A04D00C4A1A601A68012A98
:1072A000FCD1C0220A4B1A60E3E7C046E00F00F0B1
:1072B000E40F00F0E80F00F0EC0F00F004050040D0
:1072C000DFFF07C0186C004000EC0640759300001B
:1072D00014EC06400120704710B503681322DB69E7
:1072E000984710BD70470000054B0269D1500369F3
:1072F000FC331A6A002AFCD0002201201A6270476F
:107300001C050000030010B55C331A781F231A40D7
:107310001E3B19009140114AD167C2220421046921
:107320009200A150026953600269D360A023002239
:107330000169DB00CA5001230169094A5B428B5095
:107340000169084A8B5001690C3A8B500169083277
:107350008B501430FFF7FCFE10BDC04604E100E086
:107360000C0500001405000010B51430FFF702FFF3
:1073700010BD10B51430FFF703FF10BD10B5143069
:10738000FFF7EAFE10BD0000030070B55E331A7807
:107390000469724BE25003005D331A780469704B44
:1073A000E250030061331C7802696E4B012C00D05F
:1073B0009EE005005F352E78A225ED0056510200B3
:1073C00060321578A1220669D200B5500269D45006
:1073D0009623DB00994200D88CE096231B0199424A
:1073E00000D88AE096235B01994200D888E0962372
:1073F0009B01994200D885E0E1239B01994200D886
:1074000082E09623DB01994200D880E0E123DB0192
:10741000994200D87DE096231B02994200D87AE079
:10742000E1231B02994200D877E096235B02994240
:1074300000D874E0E1235B02994200D871E0E123B7
:107440009B02994200D86EE0474B994200D86CE00D
:10745000E123DB02994200D86AE0E1220023120313
:107460008A425B41414A5B421340802252059B188D
:1074700001693F4A8B50A02304220169DB00CA50F6
:1074800000210369FC33D9600369FC3319620123CD
:1074900001690B6001698B60C12104698900625038
:1074A0001F215C3002780A4093406231314AFF313B
:1074B00053500021415600293CDA0F230B40083B72
:1074C0002D4C9B089B001B1903242140A140FC3438
:1074D0008C40DD69A5432C00C0258D402900214347
:1074E000D9611F23017819401E3B8B40136070BD8A
:1074F00000246CE79E23DB02BAE79D231B03B7E75A
:107500001E4BB5E71E4BB3E7EC239B03B0E71D4BC7
:10751000AEE71D4BACE71D4BAAE71D4BA8E71D4B83
:10752000A6E71D4BA4E71D4BA2E78023DB049FE7E2
:107530001B4B9DE78C080F4BA400E41803230B4062
:10754000FF21C025DB009940AD0066598E43310014
:10755000C0269E4033000B436351C2E70C05000078
:10756000140500006C05000090D0030000D0BEFEA2
:107570002405000000E100E000ED00E000B0130091
:107580000050270000A04E0000F0750000509D0044
:1075900000F0EB0000903A0100E0D70100B0AF032B
:1075A00000705F07F7B5009308AB1B7800250193C7
:1075B000FA2304009B0083600E4B45600833036090
:1075C00014300F001600FFF7ADFD23005C33276178
:1075D0001E70009B084A9B00995823005D33197068
:1075E000019B20009B009A5823005E33DD701A70C7
:1075F000FEBDC046D4E0000050E00000036910B5B5
:107600001A00FC32D2680400002A0AD0A322D20059
:1076100099581430C9B2FFF790FD00222369FC335A
:10762000DA6010BD10B50248FFF7E8FF10BDC04694
:10763000C41B0020162307B5022200930249013B18
:107640000248FFF7AFFF07BD00200040C41B002029
:1076500010B5002801D004F0D9FA10BD0849094A34
:10766000094B10B51B688858FA22190A1B061843E3
:107670009200002302F002F84904C00B084310BD39
:107680000010014004050000281C002070B5041EF5
:1076900009D0FFF7E3FF050000F014F8FFF7DEFF65
:1076A000401BA042F8D370BD0022044B9A60044AEC
:1076B00013680133DBB213607047C046FC10014011
:1076C000281C00207047704710B500F061F8FFF7E4
:1076D000FAFF0120FFF7DAFFFFF7AAFAFFF7BAFA7D
:1076E000024B002BFAD000E000BFF7E700000000DB
:1076F000F8B516004C1EA1411F220125104B800039
:10770000104FC3584C42134038680F499D4001F058
:10771000F3FD0A21704301F0EFFD2C40030022002D
:1077200029000A4800F016F8FA21094C8900444360
:10773000386801F0E1FD0100200001F0DDFDF8BD39
:1077400050E000003000002040420F0010050050C3
:107750001027000030B504680C40944206D1013B6C
:10776000002BF8D112E0013B002B0FD004680C4035
:107770009442F8D1002405680D40954204D10134AB
:107780009C42F8D1002002E0201C00E0181C30BD13
:10779000C420114B80001A5810491140C022120217
:1077A0000A431A50C0218022490092025A501A609E
:1077B0008023A3220021DB05D20099500122F93059
:1077C0009A60074BFF301950C120023180001950D8
:1077D000403019501A60704700E100E0FF00FFFFE1
:1077E00000100140014B18607047C0467C0000202B
:1077F000F7B5002320285AD8384B8000C258042AF5
:107800005BD007D8022A54D055D80423012A09D0C6
:1078100000234CE0062A54D051D31A2A53D0022315
:107820001B2AF5D12E4A116808294ED909294FD0B3
:107830000A240226A02001252A4AC00015502A4801
:107840002A4D07681C20BF0007402948019700689F
:107850005759009027481B0207401F43C023009838
:107860009B020340FF2057515759000207401F4316
:10787000019B1F43009B58016023184007433E4370
:10788000565101251C4B156058680028FCD000207B
:107890005860A1230125DB00D3585560A025ED00D9
:1078A00050511BB2A14202D015D2611ACB40180030
:1078B000FEBD0823B6E71023B4E72023B2E7402338
:1078C000B0E78023AEE70123ACE708240026B1E748
:1078D0000C000126AEE7091B8B40E8E750E00000F2
:1078E00078000020007000403400002004050000F3
:1078F00038000020FF00FFFFFC700040F0B520289A
:107900005BD8364B8000C258354B1E68002E30D1F4
:10791000C227344BBF00D859334C03250440C02044
:1079200000022043D851C0248020640080001851F8
:107930002E4F18602E4B803CD859FF3CA043D851A5
:107940000437D859A8432043D8510837D8590C35A3
:10795000A8438446072065462843D851A820C00084
:107960001E50C1208026800076021E501C601C4BD9
:107970001C60142500202B001E4C2E004643365957
:10798000771C1BD14343E250A0230325C132FF32B1
:107990009200DB05D550184B1A68082A14D114231D
:1079A0004343E3189A6812485132FF3292005960FB
:1079B0001150DA68C1239B00C250F0BD9642E1D05D
:1079C00001300328D9D1F8E7082A02D9083AD14072
:1079D000E5E708239A1A9140E1E7C04650E000002D
:1079E0002C1C002000E100E0FF00FFFF0405000068
:1079F000009000403C0000207C0000202149F0B5B0
:107A00004A6C2148002A14D0A025A1260023012475
:107A1000ED05F600C258571C06D0C7187F68002F26
:107A200002D027009740AF5114333C2BF2D10023F2
:107A30004B64A0230121DB0500260F009C46142384
:107A40004B43C3181A1F1268104C0E4D92001419A4
:107A50005219526C002A10D01A00143A1268551CA0
:107A600009D0103B1B68FF2B05D03B0093406546B7
:107A70001A00074BEA50FC34666401310429DED158
:107A8000F0BDC046FC9000403C000020009000404B
:107A90000C05000000B5202818D8104A8000835833
:107AA000C0209A068000D2170240A020C0051218FC
:107AB0001F200340032909D80800C133FF339B006E
:107AC00001F010FC020905070021995000BD0C21AE
:107AD000FBE70421F9E70321F7E7C04650E0000087
:107AE000202812D80B4B8000C258C020930680007B
:107AF000DB170340A020C0051B181F2010400122E7
:107B00008240002902D104495A507047A121C9007E
:107B1000FAE7C04650E000000C050000030000201A
:107B2000202B12D8C021094A9B009A58890093063D
:107B3000DB170B40A021C9055B18A221C9005858CA
:107B40001F231A40D0401E3B1840704750E00000F1
:107B5000F7B506000D000C008B180193019B671B05
:107B60009C4207D0336821781B6830009847013465
:107B70000028F3D13800FEBDF0B5C64600B5CB0FE6
:107B80009846404A4B005B0D9A1882B00D000400E5
:107B9000132A2FDC002A49DB3B4F17413E000E40E1
:107BA000064323D07F08390029400C430AD03749C7
:107BB000BD438C4663445C425C418023DB0213413D
:107BC000E4071D434146CE0031492B008E192200A7
:107BD000346875682000290001F0F6FE00900191DC
:107BE0000098019922002B0003F086F802B004BC33
:107BF0009046F0BD332A08DD8023DB009A42F5D1A0
:107C000002000B0001F0E0FEF0E7224A9446012258
:107C100063445242DA400242E8D052080242D1D0D4
:107C200094438022D2051A411443CBE74B005B08F2
:107C30000343DBD00B031B0B1C4363422343802411
:107C40004D0C24031B0B23406D042B4319004346AA
:107C5000DA000F4B9B181C685D6802000B002000C7
:107C6000290001F0B1FE00900191009801992200D5
:107C70002B0003F041F842464B005B08D607334324
:107C80001900B3E701FCFFFFFFFF0F00EEFBFFFF52
:107C900008E10000EDFBFFFFF8B5274A4B005B0D44
:107CA0009A180C000700132A10DC002A36DB234B3D
:107CB00013410B423AD0802424031441002064185D
:107CC0009C430600250030002900F8BD332A0EDD54
:107CD00080230600DB000D009A42F4D102000B0065
:107CE0003800210001F070FE06000D00EBE7144D96
:107CF0000600AC46012563446D42DD40AC46634658
:107D00000D000342DFD033239A1A323B93401818F8
:107D1000874200D94C1C63469843D2E7C90FCC0771
:107D20000020531CCDD1074B1C43CAE706000D00B1
:107D30000028C0D1C7E7C04601FCFFFFFFFF0F00CE
:107D4000EDFBFFFF0000F03F30B5214A4B0087B04C
:107D50005B0893421EDD1F4A934205DD02000B00C3
:107D600002F0CAFF07B030BD02AA00F095F8032365
:107D70001840049A059B012813D002281DD0002822
:107D800014D00298039900F06FFB80231B069C46D9
:107D90006144E7E7002300220093002301F0DEF8AE
:107DA000E0E70298039900F05FFBDBE7012402980B
:107DB0000399009401F0D2F8D4E7012402980399C2
:107DC000009401F0CBF880231B069C466144C9E770
:107DD000FB21E93FFFFFEF7FF0B54746CE4680B578
:107DE0008DB004000D0000F067FA294B06001B78E7
:107DF0000F005BB29846013310D022002B00200008
:107E0000290003F0C1FA8146002807D1002200238F
:107E10002000290001F00AFC002806D130003900BA
:107E20000DB00CBC90469946F0BD01230293194B4E
:107E30000694079503934B460A934346049405958D
:107E4000002B15D0002300221900100002F0D8F8F2
:107E5000434608900991022B0ED103F0AFFB21237A
:107E600003600A9B0193002B0CD1089E099FD5E764
:107E7000002300240893099402A801F0C1F9002806
:107E8000EFD1EAE703F09AFB0A9B01930360ECE76A
:107E90008000002018E10000F0B54E464546DE4661
:107EA0005746E0B5E14B4C008FB0904689466408D8
:107EB0009C4200DC87E0DE4B9C4222DCDD4A00294C
:107EC00000DC92E0DC4B02F017FFDB4B06000F00FA
:107ED0009C4200D17EE1D94AD94B02F00DFF02004D
:107EE0000B00414630000A604B60390002F004FF8D
:107EF000D34BD24A02F000FF434601259860D96077
:107F00006BE0D04B9C4200DC8FE0CF4B9C4200DD0D
:107F100055E1CE4A231592469A4451460905631A03
:107F200019001D00040003F04BFA03F07FFA020071
:107F30000B00200029000892099302F0DDFE0022C8
:107F4000C34B02F067FC0F00060003F039FA03F0A0
:107F50006DFA04000D0002000B00300039000A9495
:107F60000B9502F0C9FE0022B94B02F053FC00222F
:107F700000230C900D9101F053FB002800D192E1F9
:107F8000002300222000290001F04AFB4342434124
:107F90000133B04A41460192022208A8009252469B
:107FA00000F07CFB4B460500002B16DA802243468E
:107FB0001206944642465B68454263445360D36868
:107FC0006344D36009E00B00020041460A604B6045
:107FD0000022002300258A60CB6028000FB03CBC43
:107FE00090469946A246AB46F0BD934B01F0ECFC9F
:107FF000914B06000F009C4200D13DE18F4A904B0F
:1080000001F0E2FC02000B00414630000A604B60C8
:10801000390002F071FE894A894B01F0D5FC012537
:1080200043466D429860D960D7E701F049F88A4A23
:108030008A4B06000F0002F0EDFB0022884B01F096
:10804000C3FC03F0BDF9050003F0F0F9794A7A4B5F
:108050000490059102F0DEFB02000B0030003900B5
:1080600002F04AFE754A06000F0004980599744B09
:1080700002F0D0FB029003911F2D00DCC7E0029AB2
:10808000039B3000390002F037FE83468A46534690
:108090005B0024155B0DE31A102B6CDD0498059929
:1080A000D322674B520502F0B5FB02000B003000F3
:1080B00039000292039302F01FFE0A000100130030
:1080C0000691079202003900300002F015FE029A74
:1080D000039B02F011FE06000F0004980599614A07
:1080E000614B02F097FB32003B0002F005FE069E5A
:1080F000079F0B000200390030000292039302F048
:10810000FBFD4B005B0D83468A46E41A312C32DDC1
:1081100004980599B822544B920502F07BFB0300AA
:108120000C000200029303940B000698079902F0DA
:10813000E3FD02000B0006000F000698079902F00D
:10814000DBFD029A039B02F0D7FD484A029003919F
:1081500004980599464B02F05DFB029A039B02F0DE
:10816000CBFD02000B00300039000292039302F0B5
:10817000C3FD83468A465A465346414630000A604C
:108180004B60390002F0B8FD029A039B02F0B4FD87
:1081900044460B000200A260E3604B46002B00DB6C
:1081A0001BE75B46236080231B06534463608023E8
:1081B0001B069C466144A060E1606D420DE70B0028
:1081C000020002F099FD434600259860D9601860CE
:1081D000596002E7D3221A4B520502F08DFD214A65
:1081E000214B0D00040002F087FD02000B00414608
:1081F00020000A604B60290002F07EFD1A4B194AEC
:1082000002F07AFD434601259860D960E5E6020058
:108210000B003000390002F06FFD6B1E154A9B0009
:108220009B5883468A46A342A5D130E7FB21E93F0C
:108230007BD9024000004054FB21F93F3163621AB0
:1082400061B4D03DFB213941FFFFEF7FEAFBFFFF27
:1082500000007041A0E1000083C8C96D305FE43FB9
:108260000000E03F7370032E8A19A33BC14920250B
:108270009A837B3920E10000D3220C4B520501F098
:10828000A3FB0B4A0B4B04000D0001F09DFB020009
:108290000B00414620000A604B60290002F02CFDD3
:1082A000034A044BB9E6032373E6C04661B4D03DEC
:1082B0007370032E8A19A33BF8B54746CE46674B29
:1082C00080B50A000F00190005003940994200D11D
:1082D0009BE004000100002F69DD3F1500D1B4E0F0
:1082E0005F4B12039C468023120B5B0313435B001E
:1082F000CA0F67449B184A00F80703D5D20F5B00EA
:108300009B188A0079108C4600218020162489460B
:1083100080030D189D4202DC29185B1B8144D50F98
:108320005B00013C5B1952004008002CF1D1002099
:108330008046802020250027000609E08B425CD083
:10834000D40F5B00013DE31852004008002D16D009
:10835000C4198B42F2DD27180E00002C49DB5B1A92
:10836000A242894149425B1A121BD40F5B00013DB6
:1083700080443100E31852004008002DE8D1134337
:108380004ED143465B0837494A4688464946521013
:108390004244C90702D5802109060B4361460F05F7
:1083A000BD18180029000CBC90469946F8BD7B000A
:1083B0005B0803433900002BF5D0002F3CD1E30AC2
:1083C000153A6405002BFAD08020400303423FD1C8
:1083D000002700E00F005B00791C0342FAD0250063
:1083E00020208D40401A2900D71B2200C2401A438A
:1083F00076E7FE43F60F8E19B1E79442A0D827180E
:10840000002CF6DB1E000023AEE702003B00280034
:10841000390002F0FFF92A003B0001F0D5FAC2E76B
:108420004346013303D0434601335B08ABE70123E6
:1084300098460023C144A6E73B00020002F05CFC22
:1084400002000B0001F0DCFDADE713000022BBE7EA
:108450000127210020207F42C6E7C0460000F07FB0
:1084600001FCFFFF0000E03FF0B54746CE4680B577
:1084700087B000920193754B4F00814688467F0874
:108480009F4263DC02F09CFF002800D1D4E04A4602
:1084900043464846414602F0BDF904000D006C4ACF
:1084A0006C4B02F0B7F96C4A6C4B01F08DFA22006C
:1084B0002B0002F0AFF96A4A6A4B02F01DFC220061
:1084C0002B0002F0A7F9684A684B01F07DFA220000
:1084D0002B0002F09FF9664A664B02F00DFC220069
:1084E0002B0002F097F9644A644B01F06DFA220008
:1084F0002B0002F08FF9029003910022604B2000C4
:10850000290002F087F9029A039B06000F00200061
:10851000290002F07FF9009A019B04000D004846F3
:10852000414602F077F902000B002000290002F01A
:10853000E3FB02000B003000390002F0DDFB02001B
:108540000B0000204F4902F0D7FB70E002000B0047
:1085500002F060F904000D003D4A3E4B02F05AF96A
:108560003D4A3E4B01F030FA22002B0002F052F956
:108570003B4A3C4B02F0C0FB22002B0002F04AF9C0
:10858000394A3A4B01F020FA22002B0002F042F95E
:10859000374A384B02F0B0FB22002B0002F03AF9C8
:1085A000354A364B01F010FA2B00220002F032F966
:1085B000354B029003919F429FDD344B00229F4236
:1085C0003DDC334900207B182E4916001F0002F0C5
:1085D00093FB049005910022294B2000290002F012
:1085E00019F932003B0002F087FB029A039B060058
:1085F0000F002000290002F00DF9009A019B0400F1
:108600000D004846414602F005F902000B0020002B
:10861000290002F071FB02000B003000390002F06B
:108620006BFB02000B000498059902F065FB07B094
:108630000CBC90469946F0BD00201249F7E7154B57
:10864000002604920593144FC5E7C046FFFF3F3E46
:10865000D43888BEE9FAA8BDC4B1B4BD9EEE213EAF
:10866000AD529C804F7E923E9015CB19A001FA3EF0
:108670007751C1166CC1563F4C5555555555A53FC0
:108680000000E03F0000F03F3233D33F0000E93FFD
:108690000000E0FF0000E73F0000D23FF0B5DE46FB
:1086A0004E4645465746E0B5DC4CA5440D911400B6
:1086B0001900A49A0993DA4B9200D6584D1E0390E4
:1086C0001821E01E0696029500F0A0FEC3430100AB
:1086D000DB1719404B1C9A009B1ADB001B190B91EE
:1086E00005934C1B771918D4A59BA5009C463F19F0
:1086F00022AE6544013707E0286802F097FE013496
:1087000003C60435BC4208D0002CF5DA0020002155
:10871000013403C60435BC42F6D1069B002B01DAB6
:1087200000F0FDFB069B03990133DB009A46099B91
:10873000DA00944600920022914672AA0492B94A45
:108740006144934688469AAB63449B44029B002B4A
:1087500000DABCE15D4600260027039C4D442A68F0
:108760006B6803CC02F056F802000B0030003900B1
:1087700001F02AF9083D06000F004445EFD1049BA3
:108780004B441E605F6008239C46E144D145DDD127
:108790000EA804218446494261448C46069A9300FF
:1087A0009C44614684460A910399083B63448C4685
:1087B0000C93009B009263449B46009A0498D1005E
:1087C00003008C46634408911E685F68002A33DD0D
:1087D000954980468C466244D300984470AB9A46D3
:1087E0000EAB99460022914B3000390002F012F88E
:1087F00002F0E6FD02F01AFE00228D4B04000D008F
:1088000002F008F802000B003000390002F074FAA0
:1088100002F0D6FD4B4601C39946434620001A6834
:108820005B68290001F0D0F808235B429C46E044D5
:1088300006000F00D045D5D1059B30001A00390045
:10884000984600F0DFFCFF2300229B0504000D008A
:1088500001F0E0FF00F038FC0022764B01F0DAFF77
:1088600002000B002000290002F046FA0D0004006F
:1088700002F0A6FD814602F0D9FD02000B002000A7
:10888000290002F039FA060040460F00002800DCFB
:10889000EEE0009B18215A1E92000EAB9B58091A5D
:1088A0001D000D41A9448D405D1B0EAB9D5017234B
:1088B0001B1A1D41002D2DDD01239C46009BE14428
:1088C000002B00DC1CE20E9C0123002C00D0B5E044
:1088D000009A012A09D099000EAA54580133002C9D
:1088E00000D0ACE0009A9A42F5D1059B002B0EDD3A
:1088F000012B00D1A8E1022B09D1009B0EA95A1E21
:1089000092000EAB9B5807939B029B0A8B50022D43
:1089100000D1C1E0002300223000390000F080FEC9
:10892000009B002800D194E2069A591E8A4210DC6E
:10893000414A0A9894460EAA6344944600229B003A
:1089400063441C68043B22438342FAD1002A00D0CE
:10895000C0E0069B0EAA013B9B00D358002B00D021
:10896000B3E001220C9B043B596801320029FAD084
:10897000009B9C466244110007921A0001338B420F
:1089800046DC0B9863468046A59C4344A046099C60
:108990009B00A1464A449844D30022AA9146049AD7
:1089A00099449446089BA59A63448446614494463E
:1089B0009A468B00634400934346586802F036FDA4
:1089C0004B4618605960029B002B24DB4D46039CEC
:1089D0000026002701E0286869680CCC01F01AFF26
:1089E00002000B003000390000F0EEFF083D0600E9
:1089F0000F005C45EFD153469E60DF6004239C4628
:108A00000433E0449C46009BE144E2449845D3D1C2
:108A1000079B0093D1E600260027ECE794FDFFFFBB
:108A2000E8E2000018FEFFFFFFFFFF1F0000703E9E
:108A30000000704100002040FFFFFF3F0021802226
:108A40005204141B0EAA5450009999420EDD0EA830
:108A500084469B000EAA8900D25861446344CF48E3
:108A600000E01A68821A04C38B42FAD101243CE761
:108A7000059B002B06D1009B0EAA013B9B00D558FD
:108A8000ED1517E70022C64B300000F0EDFD002881
:108A900000D024E100253DE732003B000020C14921
:108AA00002F02AF906000F00002C00D132E7059AE7
:108AB0000020BC4900F0A6FB02000B00300039008A
:108AC00002F01AF906000F0024E7012250E7002601
:108AD000002754E64B46059A079388468B000EA95B
:108AE000CB58183A08950592002B0DD18C4641467B
:108AF000AD4B43449B006344043B58680139183A2A
:108B00000028F9D088460592059A0020A54900F072
:108B100079FB434604000D00002B00DA05E29E00BD
:108B20000EAB9C464346DB0066449C46059370AB07
:108B30009946049F67440097306802F077FC220052
:108B40002B0001F067FE002238607960974B20000F
:108B5000290001F05FFE083F04000D00043EB94506
:108B6000EAD14AAB03939B4600239A46069B4246B2
:108B7000994643460132029204934B46002B00DA99
:108B8000AAE080208A4B009D9846C00589490026AE
:108B90000027002408E008239C460835E04454459B
:108BA00011DC4346186859682A686B6801F032FE88
:108BB00002000B003000390000F006FF013406000F
:108BC0000F00A145E7DA5B46C0C39B4601239C46E4
:108BD000009BE244083B0093029B9A45CDD1049B45
:108BE0009846A49B022B00DD8EE0002B37DC1FD1C2
:108BF000059B00271D00039B00249C461E00654426
:108C0000083E2A686B683800210000F0DDFE083D50
:108C100007000C00AE42F4D1089B002B03D0802348
:108C20001B069C4664443A0023000D990A604B6081
:108C30000720079B18409B239B009D443CBC90460B
:108C40009946A246AB46F0BD009B0EA95A1E920063
:108C50000EAB9B5807935B025B0A8B5057E643466B
:108C6000002B00DA70E100200021DB004AAAD618B0
:108C700048AF32687368083E00F0A6FEB742F8D1EC
:108C8000089B002B00D025E10B0002004A984B996D
:108C90000D9C2260636002F02FF8434607000C0031
:108CA000002B13DD01254CAEB14638002E0021000B
:108CB0004C4601360CCC00F087FEA146B045F7DAF1
:108CC000089B07000C00002B00D015E13A002300A0
:108CD0000D998A60CB60ABE70026002773E701237C
:108CE0009C46009BE1440225002B00DDEBE53200B1
:108CF0003B0000202B4901F0FFFF06000F0009E6B2
:108D00000024F2E54AAB0393A49B032B00D08FE72A
:108D10004346002B00DC14E1039ADB009B46130062
:108D200091465B441E685F68234B43440293DB001B
:108D3000994448AB9A464B465C681B681800210072
:108D400032003B000090019100F03EFE04000D0057
:108D500002000B000098019901F0CEFF3B003200A9
:108D600000F032FE4B469860D9601C605D600823BD
:108D70005B429C46E14426002F00CA45DBD14346B6
:108D8000012B00DCE3E0039A13005B441E685F687C
:108D9000029BDB0099464A44904610E0FFFFFF002B
:108DA0000000E03F0000F03FFFFFFF3F0000703E8B
:108DB000A8E20000FB21F93FFFFFFF1F9846434652
:108DC0005C681B681800210032003B000090019194
:108DD00000F0FAFD04000D0002000B00009801995C
:108DE00001F08AFF32003B0000F0EEFD4346039A9B
:108DF0009860D9601C605D60083B26002F009A4295
:108E0000DCD14D469446002600244746083565448B
:108E10002A686B683000210000F0D6FD083D06008E
:108E20000C00AF42F4D1039B4A9F5D689968D868F3
:108E3000089B002B65D08022120694460D9B65444A
:108E4000604464441F605D609960D8601E615C612D
:108E5000EEE69A464B460793059B30005A4239008E
:108E6000089500F0CFF900223A4B06000F0000F001
:108E7000FBFB002824D0384B00223000390001F0E1
:108E8000C9FC02F09DFA52460400950002F0CEFAA9
:108E90000022304B01F0BEFC02000B003000390014
:108EA00001F02AFF02F08CFA0EAA50510122059B14
:108EB000524418339046059393000EAAD45023E6EB
:108EC0005346300039009C0002F07AFA0EAB18517C
:108ED000D04619E680230D9A1B06CB18106053600C
:108EE0000B0002004A984B9901F006FF4346070029
:108EF0000C00002B00DDD5E680231B069C46644455
:108F0000E4E62B003A000D9D2A606B600A00030026
:108F1000AA60EB60320023002A616B6188E6099B3E
:108F2000DB00009372AB049332E4A49B022B00DDC0
:108F3000E8E6002B00DD92E600D079E60027002469
:108F40006AE6002600246EE70020002198E600264D
:108F5000340068E7000070410000703EF0B5CE4676
:108F6000474680B587B000920193474A4B0081463F
:108F700088465B08934207DC4146484602F020FAE7
:108F80004146031E484666D04A4643464846414647
:108F900001F040FC04000D0002000B004846414671
:108FA00001F038FC394A3A4B06000F002000290036
:108FB00001F030FC374A384B01F09EFE22002B00B6
:108FC00001F028FC354A364B00F0FEFC22002B0055
:108FD00001F020FC334A344B01F08EFE22002B00BE
:108FE00001F018FC314B324A00F0EEFC0E9B02906F
:108FF0000391002B34D00098019900222D4B01F0F1
:1090000009FC029A039B049005913000390001F09D
:1090100001FC02000B000498059901F06DFE22008E
:109020002B0001F0F7FB009A019B01F065FE224A3C
:1090300004000D00214B3000390001F0EBFB020071
:109040000B002000290000F0BFFC02000B00484686
:10905000414601F051FE07B00CBC90469946F0BD68
:1090600002000B002000290001F0D4FB124A134B30
:1090700001F042FE32003B0001F0CCFB4A46434681
:1090800000F0A2FCE7E7C046FFFF3F3E7CD5CF5A89
:109090003AD9E53DEB9C2B8AE6E55A3E7DFEB15779
:1090A000E31DC73ED561C119A0012A3F1111813FBF
:1090B000A6F810110000E03F495555555555C53FDC
:1090C00049004B0819007047474AF0B54F46914692
:1090D0004B005B0D99444646D6464A46C0B505004E
:1090E0000C000E0088460700132A27DC002A4BDB01
:1090F0003E4B13419A460B0052461340034318D08F
:109100003B4A3C4B2800210000F05EFC002200237B
:1091100000F0A0FA002847D0002C04DA80234A4649
:109120005B03134198444646534600279E4338004C
:1091300031001CBC90469946A246F0BD332A08DD9A
:109140008023DB009945F4D102000B0000F03CFCC9
:10915000EFE7294A9446012263445242DA4092469C
:109160000242E6D0224A234B2800210000F02CFCCA
:109170000022002300F06EFA002815D0002C1EDB20
:10918000534646469F430FE0194A1A4B28002100D8
:1091900000F01AFC0022002300F05CFA002803D043
:1091A000002C04DB0027002638003100C1E76400F2
:1091B000640825430027002DF6D0104EF4E74B46F7
:1091C000142B0BD03422D21A012393405D19BD42D7
:1091D00008D201239C462F00E044D1E7133B9C4674
:1091E000E044CDE72F00CBE701FCFFFFFFFF0F00BE
:1091F0009C7500883CE4377EEDFBFFFF0000F0BF6C
:10920000002070474B0070B55B0D14000A00002B66
:109210001AD14B005B08034315D0234B002201F009
:10922000F9FA224B9C422DDB0A004B005B0D363BCA
:109230001F4DE318AB422ADC002B0DDD1D4C1B0536
:1092400022401A43110070BD1B4DAB42F0D1020009
:109250000B0000F0B9FBF6E71D00353519DA174BA6
:1092600002009C4209DD0B001548164900F032F857
:10927000134A144B01F0CEFAE5E70B0012481349EC
:1092800000F028F8104A114B01F0C4FADBE70200A5
:10929000E9E7084C363322401B051343190000222E
:1092A0000B4B01F0B7FACEE700005043B03CFFFF94
:1092B000FE070000FFFF0F80FF07000050C3000003
:1092C0009C7500883CE4377E59F3F8C21F6EA501F7
:1092D0000000903C30B54A00DB0FDB0752081A4310
:1092E000110030BD02B4714649084900095C4900CB
:1092F0008E4402BC7047C046002243088B4274D3A0
:1093000003098B425FD3030A8B4244D3030B8B4286
:1093100028D3030C8B420DD3FF22090212BA030C8F
:109320008B4202D31212090265D0030B8B4219D370
:1093300000E0090AC30B8B4201D3CB03C01A524190
:10934000830B8B4201D38B03C01A5241430B8B42D8
:1093500001D34B03C01A5241030B8B4201D30B03C1
:10936000C01A5241C30A8B4201D3CB02C01A5241E8
:10937000830A8B4201D38B02C01A5241430A8B42AB
:1093800001D34B02C01A5241030A8B4201D30B0294
:10939000C01A5241CDD2C3098B4201D3CB01C01AAE
:1093A000524183098B4201D38B01C01A52414309B8
:1093B0008B4201D34B01C01A524103098B4201D3A6
:1093C0000B01C01A5241C3088B4201D3CB00C01A13
:1093D000524183088B4201D38B00C01A524143088B
:1093E0008B4201D34B00C01A5241411A00D20146B0
:1093F000524110467047FFE701B5002000F0F0F839
:1094000002BDC0460029F7D076E7704703460B43FC
:109410007FD4002243088B4274D303098B425FD36D
:10942000030A8B4244D3030B8B4228D3030C8B4299
:109430000DD3FF22090212BA030C8B4202D312127F
:10944000090265D0030B8B4219D300E0090AC30B54
:109450008B4201D3CB03C01A5241830B8B4201D301
:109460008B03C01A5241430B8B4201D34B03C01AEA
:109470005241030B8B4201D30B03C01A5241C30A62
:109480008B4201D3CB02C01A5241830A8B4201D3D3
:109490008B02C01A5241430A8B4201D34B02C01ABD
:1094A0005241030A8B4201D30B02C01A5241CDD262
:1094B000C3098B4201D3CB01C01A524183098B42AD
:1094C00001D38B01C01A524143098B4201D34B0196
:1094D000C01A524103098B4201D30B01C01A5241F9
:1094E000C3088B4201D3CB00C01A524183088B4280
:1094F00001D38B00C01A524143088B4201D34B0069
:10950000C01A5241411A00D20146524110467047DA
:109510005DE0CA0F00D04942031000D340425340DF
:1095200000229C4603098B422DD3030A8B4212D39F
:10953000FC22890112BA030A8B420CD389019211D1
:109540008B4208D3890192118B4204D389013AD00E
:10955000921100E08909C3098B4201D3CB01C01AE3
:10956000524183098B4201D38B01C01A52414309F6
:109570008B4201D34B01C01A524103098B4201D3E4
:109580000B01C01A5241C3088B4201D3CB00C01A51
:10959000524183088B4201D38B00C01A5241D9D269
:1095A00043088B4201D34B00C01A5241411A00D2EA
:1095B0000146634652415B10104601D34042002BE6
:1095C00000D54942704763465B1000D3404201B565
:1095D000002000F005F802BD0029F8D016E770471A
:1095E0007047C046D0400B1C1141203A03D49C4622
:1095F0001341184363465242934018437047C04694
:109600008446101C62468C46191C634600E0C04626
:109610001FB501F097F8002801D40021C8421FBDF2
:1096200010B500F0EFFF4042013010BD10B501F061
:1096300089F8002801DB002010BD012010BDC046C4
:1096400010B501F07FF8002801DD002010BD0120D9
:1096500010BDC04610B501F011F8002801DC002053
:1096600010BD012010BDC04610B501F007F800285C
:1096700001DA002010BD012010BDC046F0B5CE4675
:10968000474615042D0C2E0080B50704140C3F0C22
:109690009946030C7E435D43674363437F19340C53
:1096A000E4199C46A54203D980235B029846C44432
:1096B0004B4643435143250C36046544360C240481
:1096C000A4195B19591820000CBC90469946F0BDAE
:1096D000F0B54E4657464546DE46E0B543025B0AC6
:1096E000450083B00F1C99462D0EC60F002D57D094
:1096F000FF2D24D08020DB00C004184300238146C6
:109700009A469B467F3D7C027A00FB0F640A120E4C
:10971000984623D0FF2A4BD0E30080240020E404A5
:109720007F3A1C43AD186B1C474601935346774064
:109730003A000F2B48D87D499B00CB589F46002B01
:1097400000D085E008339A46063B9B467C027A00AF
:10975000FB0FFF25640A120E9846DBD1002C00D0C7
:1097600090E0524601231A4392460120DBE74C4623
:1097700058461700022824D0032800D1CFE0002249
:10978000002301284DD15802D205400AFF0710439B
:10979000384303B03CBC90469946A246AB46F0BD68
:1097A000002B5BD104239A46033B00259B46AAE786
:1097B000FF35002C60D1524602231A439246022004
:1097C000B1E7FF220023DEE74B461B0C9C464B46CD
:1097D0002604360C180461463300220C6446000C43
:1097E00043434E435043544380191A0C1218964277
:1097F00003D9802149028C4664441B041B0C1004CD
:10980000C01883015E1EB341800E1843130C1B1950
:109810009B0103431C00230179D5012362081C40EE
:109820001443019A7F32002A4DDD630704D00F23D1
:109830002340042B00D00434230103D53C4B019A70
:109840001C408032FE2ABCDCA3015B0AD2B29AE73C
:109850000C239A46093BFF259B4654E7180001F06C
:1098600071FE4A46431F76259A4000236D42914679
:109870002D1A9A469B4646E7524603231A439246C0
:10988000032050E7200001F05DFE431F2D1A9C408D
:10989000763D002047E780230027DB03FF2272E7A5
:1098A000424666E74C463200584662E780234A4605
:1098B000DB031A4222D01C4220D123435B025B0A05
:1098C0004746FF225FE701239A1A1B2A21DC230067
:1098D0000199D3409E318C401A0023005C1EA341A5
:1098E00013435A0704D00F221A40042A00D004332D
:1098F0005A0111D49B015B0A002244E780234A46A7
:10990000DB0313435B025B0A3700FF223BE7019551
:1099100087E70022002336E70122002333E7802374
:10992000DB0323435B025B0AFF222CE7F8E2000023
:10993000FFFFFFF770B500283DD0C317C5185D4085
:10994000C40F280001F0FEFD9E22121A962A07DCA1
:10995000D2B2082833DD083885406802400A23E087
:10996000992A0BDD052329001B1AD94003001B335C
:109970009D402B005D1EAB4119430D00052801DD04
:10998000431F9D402B000F490B406E0709D00F2647
:109990003540042D05D004335D0102D59F220B40D4
:1099A000121A9B01580AD2B24002D205400AE407BB
:1099B0001043204370BD002400220020F4E7680219
:1099C000400AF1E7FFFFFFFBF0B54F464646D6469B
:1099D0000C000903C0B5490A470F5E0039431F0355
:1099E000DB0F9C4665007B0A570F1F436D0DE40F8C
:1099F000760DA146C000B846D200AB1B64457BD0B3
:109A0000002B5FDD002E00D0A4E03E00164300D105
:109A100012E15E1E002E00D09EE1871A4346B84236
:109A200080410125C91A4042091A0B0200D431E1D4
:109A300049024E0A002E00D16EE1300001F082FD95
:109A40000300083B1F2B00DD61E120223900D21A00
:109A50009E40D1409F400E439D4200DD51E15D1B81
:109A60006B1C1F2B00DD7CE12021C91A3D0030005A
:109A70008F408840DD40791E8F4131000722284306
:109A8000D940002507433A40002A09D00F233B4024
:109A9000042B05D03B1DBB42BF417F42C9191F00AB
:109AA0000B0200D426E26A1CC64B55056D0D9A4286
:109AB00000D106E1C44AFF080A40530752023B4363
:109AC000120B8EE0002B00D0B8E06B1C5B055B0D29
:109AD000012B00DC30E1871A4346B842B641CB1A6D
:109AE00076429E1B330200D54CE13B003343A1D1AB
:109AF00000220024002570E0002B00DCE5E0002EB1
:109B000000D183E0AF4EB54260D0802636043743A3
:109B1000B846382B00DC3EE1434613431F007A1E53
:109B200097413F1887428041404209180B0200D4F8
:109B3000B0E0A44B01359D4200D1C3E0A24A7B08AE
:109B40000A4001210F401F435108D30707221F433A
:109B50003A4099E79B4EB54238D0802636043743C9
:109B6000B846382B00DDDCE01F2B00DC30E11E00A6
:109B70004746203EF740BC46202B04D04026F31A2F
:109B800046469E403243170063467A1E97411F4364
:109B9000CCE0002B00D104E24346134300D159E14D
:109BA0004B07C00818438023C9081B03194208D07B
:109BB0004546ED081D4204D14346D00859070843E5
:109BC0002900420FC9007F4D1143C0004B07CA084E
:109BD0007C49C00803438D4268D012036D05120B07
:109BE0006D0D002112031800130B0A0D12051A4304
:109BF000764B2D0513402B435B00E4075B082343A2
:109C000019001CBC90469946A246F0BD3E00164382
:109C100012D05E1E002E00D000E1871887428041DE
:109C200041444042091801250B0233D5022585E73E
:109C300064463300414610001D00C7E7002D00D0E8
:109C4000DAE00C000443F3D05C1C00D19FE15D4CD2
:109C5000A64200D12FE1DB43382B00DD66E11F2B4C
:109C600000DD83E120240500E41A0F00DD40D94027
:109C7000A0404346A7405B1A441EA04198462F438C
:109C80003843171ABA42924143465242991A6446DF
:109C90003500CAE607223A40002A00D0F6E64B0714
:109CA000CA084849FF083B438D4296D11900114329
:109CB00000D19EE1802109030A431203120B414D9A
:109CC0008FE71500002200238BE7002B00D0C7E0B0
:109CD0006B1C5F057F0D012F00DCF1E0394DAB42BD
:109CE00000D1B9E085180A008542894142444942C1
:109CF00051180722CF076D082F4349083A401D002D
:109D0000C2E607223049ED1A31403A40BCE63E0037
:109D10002838864000279FE6380001F013FC2030E9
:109D20008EE6434613431F007A1E9741C71BB84275
:109D300080414042091A78E60E003B000643134377
:109D4000002D61D1002E00D0F4E0002B00D11BE1EA
:109D500064463900100039E71A4FBB427AD033000D
:109D6000FFE630001F3DE840202B03D04021CB1AF6
:109D70009E4037437B1E9F41072207433A40002104
:109D8000002589E7171A4346BA42B641591A764266
:109D90008E1B64464EE61F2B00DDADE020264746B5
:109DA000F61AB740B9461700B246DF404E463E436A
:109DB00037005646B240561EB24117434246DA407B
:109DC0008918AEE6FF070000FFFF7FFFFFFF0F804F
:109DD00020264746F61AB740B9461700B246DF407C
:109DE0004E463E4337005646B240561EB2411743D8
:109DF0004246DA40891A99E77F4CA6425BD080241C
:109E000024045B42214327E7002E0CD1002B00D114
:109E1000CBE0644639001000774DD7E6764FBB4261
:109E200018D0330075E6002B14D04B07C008184338
:109E30008023C9081B03194207D0FC081C4204D127
:109E40007907D0080843E14621004C46420FC9007B
:109E50001143C000684DB9E61D0000220023C0E692
:109E6000002D5BD10D00054300D1E2E65D1C00D161
:109E7000B0E0614DAE421FD0DB43382B71DC1F2BAD
:109E800000DD96E020250F00ED1AAF40B94607002F
:109E9000AA46DF404D463D432F005546A840D940D5
:109EA000451EA84188440743BF189742924151423A
:109EB000414435003AE6644635004146100085E6E7
:109EC0000B000343002D00D063E6002BF5D0434682
:109ED000134300D17AE68718874280410722414424
:109EE000404209183A400B0200D4D5E6434B0135F5
:109EF0001940C9E5380069E61E004746203EF74094
:109F0000BC46202B04D04026F31A46469E403243DE
:109F1000170063467A1E97411F4302E6364DAE4254
:109F2000CAD080252D045B422943A6E70843411E81
:109F30008841A6E6002B00D148E6871A4346B8427E
:109F4000B641CB1A76429E1B33024BD5171A4346B5
:109F5000BA429241591A5242891A072264463A403B
:109F600092E501430F00791E8F419DE71C000F0011
:109F7000203CE740202B03D04024E31A99400843BB
:109F8000411E884138437CE60022002425E6171A4A
:109F90004346BA429241591A5242891A64463500E0
:109FA00043E541461000144D10E6802200241203C0
:109FB00080E61D000F00203DEF40BC46202B03D063
:109FC0004025EB1A9940084307006346781E8741F5
:109FD0001F4369E7871897429B4141445B42C91878
:109FE0003500A3E53B003343CED0072231003A4091
:109FF00052E600231A00F4E5FF070000FFFF7FFF91
:10A00000F0B55746DE464E464546E0B58346070066
:10A010000E03480085B092461C00360B400DCD0F54
:10A02000002800D19DE0954B984239D08023F6005E
:10A030001B041E43924A7B0F334399469446030008
:10A040006344009300230026FF00029323031B0BAD
:10A0500098466300E40F52465B0D019400D1B3E0D3
:10A0600086498B4200D19EE04246D10080221204F4
:10A070000A435146490F11438B46814952468C464B
:10A0800000996344CB1A0021D20000932B00634057
:10A090009A460F2E00D905E17A4BB6009B599F4690
:10A0A0005B463343994600D0B8E0022308260027D8
:10A0B00000900293CAE7CB463A0002990195019BB2
:10A0C0009A46022927D0032900D180E2012944D0F1
:10A0D0006D49009B8C4663441C00002C38DD5307FF
:10A0E00000D013E2D2085B46DB0109D55946674B25
:10A0F00019408B468021C9008C46009B63441C009C
:10A10000634B9C4207DC5B4664055F075B021743B9
:10A110001B0B620D02E000230027584A00211B039D
:10A120001C0B0B0D1B05234314055A4A3800134022
:10A130001C4353466400DB0764081C43210005B040
:10A140003CBC90469946A246AB46F0BD0122524225
:10A1500001231B1B382B00DCADE10022002300276C
:10A16000DCE75B46334399465ED0002E00D18AE19E
:10A17000300001F0E7F903000B3B1C2B00DD7BE115
:10A180001D22D31A5A460100DA4008398E401300C6
:10A190005F46334399468F403F4B00261B1A00937E
:10A1A0000023029352E7414653460B433B499B46EB
:10A1B0008C46009B634400935B46002B3BD10223FB
:10A1C00000221E43022161E7434613439B4637D0DA
:10A1D0004346002B00D162E1404601F0B3F9030091
:10A1E0000B3B1C2B00DD53E102004146083A914035
:10A1F00088461D21CB1A5146D9400B0041460B43DE
:10A200009B46534693401A00009B25499C46604458
:10A2100003008C4663440093002137E70323B146D3
:10A2200000900C26029311E70023009301330426CB
:10A23000002702930AE70323C3461E43032125E7B1
:10A2400001331E430022012120E700239A46802388
:10A2500000271B03094A61E7802349461B03194273
:10A2600000D1E2E05946194200D0DEE00B431B0367
:10A2700017001B0BA246014A50E7C046FF0700002B
:10A2800001FCFFFF38E30000FF030000FFFFFFFEBB
:10A29000FE070000FFFF0F800DFCFFFF01F8FFFF2E
:10A2A000F3030000D94500D9CBE000D1C6E03C0063
:10A2B00048460027009B013B00935B46160E1B029D
:10A2C0001E431302984633041B0C9946310C01912E
:10A2D000FFF798F84A4642430B04210C0500194346
:10A2E0008A4207D98919013D8E4203D88A4201D991
:10A2F000851E8919881A0199FFF784F809048C468C
:10A300004A46210464464243090C030021438A4221
:10A3100004D98919013B8E4200D8F1E02D041D4378
:10A32000AB464346891A4246280C12041D0C5B4674
:10A33000140C22001B041B0C5A4303946B4344432C
:10A34000029568431B19150CEB189C4203D9802415
:10A350006402A44660441C0C15041B042D0C201838
:10A360005D19814277D373D00C1AA24A7D1BAF428C
:10A37000BF419446009B7F426344E01B1C00864221
:10A3800000D1DBE00199FFF73DF84A4642430B0458
:10A39000290C070019438A4207D98919013F8E42C7
:10A3A00003D88A4201D9871E8919881A0199FFF7B3
:10A3B00029F809044A46894629044D464243090CB6
:10A3C000030029438A4207D98919013B8E4203D8E9
:10A3D0008A4201D9831E89193F04891A3A00039FD2
:10A3E0001A43380013041B0C584381460298150C7D
:10A3F0006F43434345434846000C8446DB1963449E
:10A400009F4203D9802040028446654448461F0C81
:10A4100000041B04000C7D191818A94200D284E026
:10A4200000D17FE001231A4357E680234A461B03ED
:10A4300013431B031B0BAA466F4A6FE6BA4200D9AF
:10A4400035E74B46DC0758087B081C43FF0734E719
:10A450000024AF4289D247444745A4415B46644249
:10A46000A4196418013BA6421ED2A0426DD800D1A7
:10A47000B6E0241A9B4678E703005A46283B9A40E8
:10A480000027914688E6584601F05CF8203072E6D5
:10A4900003005246283B9A4093460022B4E65046B9
:10A4A00001F050F820309AE6A642E2D1B845DCD956
:10A4B000341A9B4659E71F2B65DC504C0099A44683
:10A4C0005C46614408008C4011008240D940501E17
:10A4D00082410C4314435A46DA401300620709D004
:10A4E0000F222240042A05D02200141D94428941E3
:10A4F00049425B181A0262D50122002300270DE6AB
:10A500008A4200D80AE7831E891907E70F23134000
:10A51000042B00D1E6E5171D9742924153429B441C
:10A52000FA08E0E5002800D1D7E57118531EB142C2
:10A5300027D3A94215D358D01A0073E7002B00DCAB
:10A5400004E6012300229B44CDE50223474447450E
:10A5500089415B429C46494289190C19E344241AFB
:10A5600003E743465F0047459B41B8465B429E195F
:10A57000023A8919A94200D054E7404500D051E77A
:10A58000ABE51A00F6E71F215F4649420C1BE74086
:10A59000202B07D01A49009B8C46634418005B4669
:10A5A00083401A43501E82413A4307270023174035
:10A5B00009D00F21002311401400042995D1220055
:10A5C0005F075B021B0BD20817430022A6E580231E
:10A5D00059461B030B431B0317001B0B064A9DE543
:10A5E000BD42B2D89B460024BFE68045B9D31A00CD
:10A5F000C3E7C046FF030000FF0700001E04000081
:10A600003E040000F0B54F464646D6468446C0B5E7
:10A610008046194E18030F034D00000B5C00824664
:10A620003F0B6D0DC90F9146640DDB0F0120B54244
:10A630000AD0B44203D0A54201D157450CD01CBC6E
:10A6400090469946A246F0BD66463E43F7D1AC42DD
:10A65000F5D154461443F2D10120C845EFD19942B7
:10A6600007D0002DEBD163461F433800471EB84189
:10A67000E5E70020E3E7C046FF070000F0B54F46DE
:10A680004646D6464D00C0B50E03C90F8A462C4932
:10A690001F035C008046360B6D0D91463F0B640D29
:10A6A000DB0F8D421ED08C4216D0002D1ED13043C0
:10A6B0008446002C01D13A4323D06246002A1AD0A6
:10A6C0009A4529D0514602200139084001381CBC66
:10A6D00090469946A246F0BD39001143E5D00220CC
:10A6E0004042F4E73043FAD1AC420FD0002C0FD1F6
:10A6F0003A43E7D00CE00122013B934318000130BC
:10A70000E5E763460020002BE1D0DBE73A43E6D1E2
:10A710009A45D7D1A542D5DCA54205DBBE42D1D8AA
:10A7200008D00020BE42D2D25046012301389843BF
:10A730000130CCE7C845C5D80020C845F4D3C6E7EA
:10A74000FF070000F0B54F464646D6464D00C0B55F
:10A750000E03C90F8A462E491F035C008046360B44
:10A760006D0D91463F0B640DDB0F8D4218D08C426E
:10A7700011D0002D18D130438446002C1ED13A430D
:10A780001CD163460020002B30D0514602200139F5
:10A79000084001382AE039001143EAD0022025E0C0
:10A7A0003043FBD1AC4226D0002C26D13A4324D1F1
:10A7B0005146022001390840013817E06246002A5C
:10A7C0000FD09A45E1D1A54205DBBE42DDD819D0B4
:10A7D0000020BE420AD2504601230138984301307E
:10A7E00004E00122013B9343180001301CBC904659
:10A7F0009946A246F0BD3A43D0D19A45C5D1A5426B
:10A80000C3DCE0E7C845C0D80020C845E3D3EDE786
:10A81000FF070000F0B55746DE464E464546E0B518
:10A82000834606000F03480087B092461D003F0B89
:10A83000400DCC0F002800D16FE0DE4B984238D09D
:10A840008023FF001B041F43730F3B430193DA4B2C
:10A850000027994600239B46F60081442B0369009C
:10A860001B0B52469846490DED0F002900D185E09B
:10A87000D04B994200D173E04346DA0080231B0499
:10A8800013435246CC48520F84461343524600208D
:10A890006144D20089442100694000918C46012125
:10A8A00049448A460F2F00D990E0C449BF00CF59D0
:10A8B000BF465B463B43019300D06AE10223082771
:10A8C000002681469B46C9E732005846019B6146F7
:10A8D0000091022800D175E0032800D1FEE1012893
:10A8E00000D02CE100230027002600253F032A0D7D
:10A8F0003F0BB34812053A4302401B051343009A2D
:10A900005B00D1075B080B433000190007B03CBC6B
:10A9100090469946A246AB46F0BD5B463B43019349
:10A9200000D12FE1002F00D1A5E1380000F00AFE90
:10A9300003000B3B1C2B00DD96E11D22D31A5A4667
:10A940000100DA405E4608398F4013008E403B43D9
:10A9500001939C4B00271B1A994600239B467DE7D9
:10A96000414653460B4393498C46E144002B00D0AB
:10A970001AE102220220174300228CE7134300D180
:10A980000DE14346002B00D181E1404600F0DAFDA5
:10A9900002000B3A1C2A00DD72E10100434608392F
:10A9A0008B4098461D239A1A5346D3401A004346BB
:10A9B000134352468A404946081A824989468144CF
:10A9C000002068E77B4B002700268EE7140C12045A
:10A9D000120C1100370C3604350C794328008C46D4
:10A9E0002E0060436044834656432100300C80466D
:10A9F0005846794340440291844506D988468021CF
:10AA000049028C46E044414602913604010C360C62
:10AA100000048B4681191E0C1B041B0C03911900AA
:10AA200079438C46280075436544A8465843050C75
:10AA300045447743A94203D9802149028C466744A3
:10AA4000290C8C4639000004000C2D042D1861449B
:10AA5000AB4405915946049101990F043F0C080C31
:10AA6000390051434243904602008C46090C8B4604
:10AA700062437C4344445C44A04503D9802149029D
:10AA800088464244210C884661460904090C8C46DC
:10AA900039005943434370437E430F0CF618240496
:10AAA000BE19644442448C46B34203D980235B02FE
:10AAB00098464044029B61469846049B37044344B1
:10AAC0009B46AB45AD416B420D0405992D0C8C4660
:10AAD0007F196744FD18A8465D462D19A542A4417B
:10AAE00093466442A446C344DC448F42BF41984528
:10AAF0009B4193459241A445A4415B427F421F4341
:10AB0000360C52426442BF192243BF1862463818BD
:10AB10004302D20D039913436A020A43501E824135
:10AB20006146ED0D2A434E023243D90100D4B3E011
:10AB30000126500832400243DE0732435B08224CB4
:10AB40005444002C62DD510709D00F201040042826
:10AB500005D0101D9042924152429B180200D9012B
:10AB600004D580241948E400034054441848844222
:10AB700000DD27E75E075B02D2081F0B6305164363
:10AB80005B0DB2E6002399460133042700269B465D
:10AB900064E60323019781460C279B465EE601226B
:10ABA00001201743002276E6032303201F43434678
:10ABB00071E6C046FF07000001FCFFFF78E30000DC
:10ABC000FFFF0F800DFCFFFFFF030000FFFFFFFEF4
:10ABD000FE0700000023802700933F030026434B1D
:10ABE00083E6019B3200A446584670E6AC466EE60A
:10ABF000802701993F0339422DD03B422BD11F437F
:10AC00003F033F0B00951600384B6EE601252D1BC8
:10AC1000382D00DD66E61F2D40DC35481C00504411
:10AC2000160082408440EE40501E8241344314435B
:10AC3000EB40620709D00F222240042A05D02200EF
:10AC4000141D9442804140421B181A023ED5012334
:10AC50000027002649E68027019B3F031F433F034F
:10AC60003F0B0094214B40E603005A46283B9A4094
:10AC7000002601926DE6584600F064FC203057E64D
:10AC800003005246283B9A401300002293E65046A8
:10AC900000F058FC20307BE6CA4650E71F201E001B
:10ACA0004042041BE640202D03D0124C5444A340E4
:10ACB0001A43501E8241324307260027164009D00E
:10ACC0000F200023104014000428B9D122005E0791
:10ACD0005B021F0BD2081643002306E680273F03C2
:10ACE0001F433F033F0B1600004BFEE5FF0700002C
:10ACF0001E0400003E040000F8B557464E46454687
:10AD0000DE460C000903E0B5490A460F5F003143F7
:10AD10001E03DB0F760A9B46530F3343C84E650074
:10AD2000C000E40FD2006D0DA24681467F0D9C4607
:10AD30009046B74200D1B9E05B46012673409B467E
:10AD4000EE1BA34500D183E0002E63DD002F00D071
:10AD5000B1E06346134300D123E1731E002B00D002
:10AD6000BAE1861A6346B04280410125C91A4042C1
:10AD7000091A0B0200D447E149024B0A98464346A0
:10AD8000002B00D189E1404600F0DCFB0300083BCA
:10AD90001F2B00DD7CE120223000D21A4146D0403A
:10ADA000994002009E400A439D4200DD6AE15D1B1E
:10ADB0006B1C1F2B00DD94E1202110003500C91A07
:10ADC0008E40DA408840DD40711E8E41110007221E
:10ADD0002843002506433240002A09D00F23334080
:10ADE000042B05D0331DB342B641764289191E00AB
:10ADF0000B0200D43DE26A1C914B55056D0D9A4241
:10AE000000D119E18F4AF6080A405707520237432A
:10AE1000120B9BE0002E00D0C5E06E1C7605760D6F
:10AE2000012E00DC48E16746861ACB1BB042BF41C9
:10AE30007F42B8461F004346FF1A3B00B8461B023C
:10AE400000D55FE137439AD100220024002579E044
:10AE5000002E00DCFAE0002F00D18DE0784B9D42FF
:10AE600067D0802367461B041F43BC46382E00DC96
:10AE700052E1634613435A1E93411E188642804195
:10AE8000404209180B0200D4BEE06D4B01359D42D3
:10AE900000D1D2E06B4A73080A4001210E401E43E4
:10AEA0005108D30707221E43324095E71E00164380
:10AEB00000D045E740E7624B9D423AD08023674689
:10AEC0001B041F43BC46382E00DDEBE01F2E00DCC8
:10AED0003AE133006746203BDF403B00202E05D09F
:10AEE0004027BF1B6646BE40324390464646721E10
:10AEF00096413343DAE0002B00D114E2634613435A
:10AF000000D168E180234E07C008C9081B0306432F
:10AF1000194208D06046C008184204D163460100B7
:10AF2000D2085E071643F3009946C900720F444DDC
:10AF300011434B46DE08424B4F073743CA089D4238
:10AF400000D16EE012036D05120B6D0D002112038E
:10AF5000130B0A0D12051A433B4B2D0513402B43CF
:10AF60005B00E4075B082343380019003CBC9046B3
:10AF70009946A246AB46F8BD6346134311D0731EF3
:10AF8000002B00D007E18618864280416144404290
:10AF9000091801250B0237D502257BE73E006146E3
:10AFA00091463500C5E75C46002D00D0E1E00B007E
:10AFB0000343F3D0731C00D1ACE1214B9F4200D17D
:10AFC0003AE1F343382B00DD6FE11F2B00DD8CE10C
:10AFD00020250E00ED1AAE40B0460600AA46DE401F
:10AFE000454635432E005546D940A8406346451E88
:10AFF000A8415B1A9C463043161AB24292416346FE
:10B000005242991A3D00B4E607223240002A00D08D
:10B01000E4E60B4BF6084F073743CA089D4200D0C1
:10B0200090E73B00134300D1A6E180231B031A43A2
:10B030001203120B024D89E715000022002785E755
:10B04000FF070000FFFF7FFFFFFF0F80002E00D0F3
:10B05000C7E06B1C5E05760D012E00DCF0E0C84DEC
:10B06000AB4200D1B9E085180A00854289416244AB
:10B07000494251180722CE076D082E434908324035
:10B080001D00A9E6BF49ED1A114007223240A3E690
:10B09000320028388240002686E6300000F052FA5E
:10B0A000203073E6634613435A1E9341C61AB042DA
:10B0B00080414042091A5CE60E006746064317438A
:10B0C000002D5ED1002E00D0F3E0002F00D11EE154
:10B0D0005C46614691462CE7A94FBE427BD01E00DC
:10B0E000F1E610001F3DE840202B03D04021CB1A91
:10B0F0009A401643731E9E410722064332400021A8
:10B10000002583E7161A6346B2428041591A40422D
:10B110000B1A98465C4632E61F2E00DDABE0202776
:10B12000BB1B9A4663465746BB40994613004F46A1
:10B13000F3401F433B005746BA40571EBA411343E2
:10B140006246F240891898E62027BB1B9A46634660
:10B150005746BB40994613004F46F3401F433B0000
:10B160005746BA40571EBA4113436246F240891A05
:10B170009CE7834B9F425FD080252D047342294377
:10B1800020E7002E0CD1002F00D1D0E05C466146B4
:10B1900091467B4DCDE67A4FBE421CD01E0065E63F
:10B1A000002F18D0C0084E0706438020C9080003AE
:10B1B000014208D06346DC08044204D12100DA468B
:10B1C000D2085E071643F300994601245346C9008E
:10B1D000720F11431C406A4DABE61D000022002790
:10B1E000B4E6002D59D10B00034300D1D6E6731C01
:10B1F00000D1B2E0624B9F421ED0F343382B6FDC8C
:10B200001F2B00DD97E020250E00ED1AAE40B04662
:10B210000600AA46DE40454635432E005546A84066
:10B22000D940451EA8418C440643B6189642924127
:10B23000514261443D0025E63D006146914678E675
:10B240000B000343002D00D055E6002BF5D06346DC
:10B25000134300D16DE68618864280416144404226
:10B26000091800220B0200D4D0E6464B01351940E4
:10B27000B2E5B1465DE633006746203BDF403B0068
:10B28000202E05D04027BF1B6646BE403243904665
:10B290004646721E96413343EFE5394B9F42CBD071
:10B2A00080252D0473422943A8E70843411E8841A5
:10B2B000A2E6002F00D13CE66346861ACF1AB042C0
:10B2C0009B415B42FB1A98461B024ED5161A6346F9
:10B2D000B2429241591A5242891A5C4600227BE5D9
:10B2E00001430E00711E8E419FE71D000E00203DA0
:10B2F000EE40B046202B04D04025EB1A994008437D
:10B30000814648464346411E8841184374E6002260
:10B31000002417E6161A6346B2429241591A524265
:10B32000891A3D0025E561469146154D01E68022CA
:10B330000024120379E61D000E00203DEE40B046C9
:10B34000202B04D04025EB1A9940084381464E46F5
:10B350004346711E8E411E4367E7861896429B4105
:10B3600061445B42C9183D008CE547463743CED067
:10B3700007224146324049E600273A00E6E5C0464A
:10B38000FF070000FFFF7FFF70B50C4E0D031C038D
:10B3900049005B002D0B490D240B5B0DB14208D019
:10B3A000064900208B4203D114432000441EA041D3
:10B3B00070BD05430120002DFAD1F1E7FF07000021
:10B3C00030B5144D0A034B00120B5B0DC90F00245E
:10B3D000AB4211DD104CA34210DC802464032243F5
:10B3E0000E4CE41A1F2C0CDD0D48C31ADA40130072
:10B3F0005C42002900D11C00200030BD094BCC1854
:10B40000FAE7094DE040AC4663449A401300034319
:10B41000EEE7C046FE0300001D04000033040000F8
:10B4200013040000FFFFFF7FEDFBFFFF70B5002856
:10B430002DD0C317C5185D40C40F280000F082F856
:10B44000154B1B1A5B055B0D0A2815DD0B38854073
:10B4500000222D032D0B002110002D030A0D2D0BB2
:10B4600012052A430D4D1B052A4013435B00E407D8
:10B470005B082343190070BD02002900153291407A
:10B480000A000B21081AC5402D032D0BE3E7002409
:10B49000002300250022DEE71E040000FFFF0F80CE
:10B4A0004100090E4B1C70B5DBB24602750AC40F91
:10B4B000012B14DDE0239B006D07360BCB18002118
:10B4C0000A0D280012051C4D32435B052A405B081B
:10B4D00013435B00E4075B082343190070BD002998
:10B4E00014D1002D1ED0280000F02CF80A281CDCF6
:10B4F0000B232A001B1ADA40030015339D400F4B23
:10B5000012031B1A5B05160B5B0DD8E7002D06D046
:10B51000320B802636036D071643094BCFE7084BE5
:10B520000026CCE700230026C9E703002A000B3BD6
:10B530009A400025E3E7C046FFFF0F808903000023
:10B54000FF0700001C2101231B04984201D3000CBB
:10B5500010391B0A984201D3000A08391B09984286
:10B5600001D30009043902A2105C40187047C0469C
:10B5700004030202010101010000000000000000BC
:10B5800030B51C00094B05001B6885B0D868084B16
:10B59000002A01D1074B1A000292019300912B005F
:10B5A0002200054900F026F800F0A6FD84000020E6
:10B5B000B8E30000C8D10000C5E30000014B1868E3
:10B5C0007047C04684000020084B10B50400002BD3
:10B5D00002D0002100E000BF054B1868836A002BF1
:10B5E00000D09847200001F05DFBC046000000003D
:10B5F000F4E300000EB403B5010003AB044804CB30
:10B600000068019300F076F802B008BC03B0184758
:10B610008400002070B500260C4D0D4C641BA41056
:10B62000A64209D1002601F03FFB0A4D0A4C641BDB
:10B63000A410A64205D170BDB300EB58984701365F
:10B64000EEE7B300EB5898470136F2E754020020CA
:10B65000540200205402002064020020002310B590
:10B660009A4200D110BDCC5CC4540133F8E710B548
:10B67000884202D98B18984203D3002307E08B5CE1
:10B680008354013AFBD210BDCC5CC45401339A42BE
:10B69000FAD1F8E703001218934200D170471970ED
:10B6A0000133F9E7936810B5013B9360002B04DA8E
:10B6B0009469A34207DB0A2905D01368581C10605F
:10B6C0001970080010BD00F04BFC0100F9E7F8B557
:10B6D00006000F001400D518AC4201D1002007E08D
:10B6E00021783A003000FFF7DDFF0134431CF3D12D
:10B6F000F8BD0000F0B59FB002900F001600059352
:10B70000002805D083690493002B01D100F0F4FDDB
:10B710007B4B9F425BD1029B5F68BB891B0762D555
:10B720003B69002B5FD0002306AC63612033637656
:10B730001033A37635002B78002B01D0252B5CD15C
:10B74000AB1B04930CD0320039000298FFF7BFFF07
:10B75000431C00D1C4E06269049B94466344636166
:10B760002B78002B00D1BBE0012200235242626003
:10B7700002A9543252186E1C2360E360A360137058
:10B78000A365317805225F4800F0D4FE751C0028BF
:10B7900035D12268D30604D5532302A95B18202192
:10B7A0001970130704D5532302A95B182B211970B4
:10B7B00033782A2B2CD0350000210A20E3682A7820
:10B7C0006E1C303A092A64D900292ED026E04E4B4F
:10B7D0009F4202D1029B9F689FE74C4B9F429CD1A6
:10B7E000029BDF6899E73900029800F00FFC0028FF
:10B7F00099D0012040421FB0F0BD01359BE7414B7D
:10B800002268C01A01238340134323602E00B8E747
:10B81000059B191D1B680591002B01DB099304E0B2
:10B820005B42E3600223134323602B782E2B0AD163
:10B830006B782A2B35D1059B02351A1D1B680592A2
:10B84000002B2BDB0793324E29780322300000F0C7
:10B8500071FE002806D04023801B834022680135FA
:10B8600013432360297806222A486E1C217600F0B3
:10B8700061FE00283AD0284B002B25D10722059BDA
:10B8800007339343083305936369039A9B186361F5
:10B8900050E7434301219B18350090E701235B42A9
:10B8A000D0E700230A201A000135636029786E1C56
:10B8B0003039092903D9002BC5D00792C3E7424389
:10B8C000012352183500F1E705AB00933A00134B02
:10B8D0002100029800E000BF0390039B0133D3D105
:10B8E000BB895B0600D584E70B9884E705AB009322
:10B8F0003A000A4B2100029800F080F8ECE7C046BD
:10B900004CE40000F8E300006CE400002CE40000CC
:10B91000FEE3000002E4000000000000CFB60000DB
:10B92000F7B5150001938A680B6900900C009342EB
:10B9300000DA130022002B6043321278002A01D073
:10B9400001332B6023689B0602D52B6802332B60E2
:10B95000062723681F4027D0230043331B785A1E35
:10B9600093412268920630D4220001994332009814
:10B97000089EB047431C25D0062320682A68E1684A
:10B9800003400025042B03D18D1AEB43DB171D4028
:10B99000A3682269934201DD9B1AED180027BD427E
:10B9A00020D1002010E00137E3682A689B1ABB42CF
:10B9B000D2DD22000123193201990098089EB04778
:10B9C000431CF0D101204042FEBD3020E11843313C
:10B9D000087021005A1C45310978A21843320233FD
:10B9E0001170C1E7220001231A3201990098089EC4
:10B9F000B047431CE6D00137D1E70000F0B589B06D
:10BA000004920A0043320593039002920A7E0C00CE
:10BA10000E9B6E2A00D186E01FD8632A33D008D847
:10BA2000002A00D18CE0582A4DD0250042352A70DA
:10BA300030E0642A01D0692AF7D1196825680A1D07
:10BA4000280629D508681A60002803DA2D23029AEF
:10BA5000404213706B4E0A274FE0732A74D008D807
:10BA60006F2A1FD0702AE0D1202209680A43226081
:10BA700003E0752A16D0782AD7D1220078214532E2
:10BA80001170614E22E025001A684235111D1960BF
:10BA900013682B70012365E008681A606906D3D526
:10BAA00000B2D1E719682568081D186008682E06DD
:10BAB00005D5544E08276F2A1BD00A2719E06D06BA
:10BAC000F7D580B2F5E745314E4E0A701868226806
:10BAD000011D00681960150621D5D30702D5202362
:10BAE0001A4322601027002803D1202322689A439A
:10BAF00022602300002243331A706368A360002B86
:10BB000058DB0422216891432160002854D1029D12
:10BB1000002B5AD02500337842352B7055E055065E
:10BB2000DBD580B2D9E71A680D68101D4969186025
:10BB300013682E0601D5196002E06D06FBD5198049
:10BB40000023029D23614FE01A68111D19601568DA
:10BB500000216268280000F0EDFC002801D0401BA5
:10BB60006060636823610023029A13703CE02369DC
:10BB70002A0004990398059DA847431C3ED02368DA
:10BB80009B0715D4079BE068984239DA180037E024
:10BB900022000123193204990398059EB047431CE3
:10BBA0002CD00135E368079A9B1AAB42F0DCE9E739
:10BBB0000025F7E70028ADD0029D3900FDF722FCF3
:10BBC000735C013D2B700028F7D1082F09D1236841
:10BBD000DB0706D563682269934202DC3023013D0E
:10BBE0002B70029B5B1B2361059B07AA009321001E
:10BBF000049B0398FFF794FE431CB8D101204042F8
:10BC000009B0F0BD09E400001AE400000D4B70B566
:10BC10001C680500A36B002B0FD1182000F06EFCF0
:10BC2000094BA0630360094B01224360084B83600A
:10BC30000B2383810023026143610022A36B1D61FA
:10BC40005A6170BD840000200E33CDAB34126DE616
:10BC5000ECDE0500124B10B51C68A36B002B0FD156
:10BC6000182000F04BFC0F4BA06303600E4B012229
:10BC700043600E4B83600B23838100230261436189
:10BC8000A46B0B4A206961690A4BFDF7F7FC01229E
:10BC9000002380185941206161614800400810BDAF
:10BCA000840000200E33CDAB34126DE6ECDE0500CF
:10BCB0002D7F954C2DF451580CB430B5164B9DB0DA
:10BCC0000C1E1D6808DA8B2301202B6040421DB03A
:10BCD00030BC08BC02B01847822302A99B008B81AC
:10BCE0000023029008619C4200D0631E8B604B6170
:10BCF00001235B42CB81209A21AB2800019300F005
:10BD000055FD431C01DA8B232B60002CDFD0002370
:10BD1000029A1370DBE7C046840000200EB400B521
:10BD20000B499CB01DAB0290069007910491094805
:10BD3000094904CB0591006802A9019300F036FD82
:10BD40000023029A13701CB008BC03B01847C04609
:10BD5000FFFFFF7F840000200802FFFF020010B5F4
:10BD60001378541C002B05D1CC5CD4540133002C27
:10BD7000FAD110BD2200F3E7C9B20378002B04D03A
:10BD80008B4200D170470130F7E74B42594149429D
:10BD90000840F7E702780B78002A03D00130013120
:10BDA0009A42F7D0D01A70470023C25C0133002AB0
:10BDB000FBD1581E7047002330B59A420AD0013A91
:10BDC000C45CCD5CAC4204D1934202D00133002C60
:10BDD000F6D1631B180030BD30B50500002A00D134
:10BDE00030BD0C78013A6B1C2C700131002C05D150
:10BDF0009A189A42F4D01C700133FAE71D00EDE75F
:10BE000010B50378002B0FD10B785A4253415B4297
:10BE1000184010BD0023CA5C002AFAD0C45C9442CA
:10BE200001D10133F7E701300378002BF2D118007C
:10BE3000EFE70000F0B51F000E0087B005900191FC
:10BE400002920C98347800F0EAFA0822001943783C
:10BE5000751C134036D12D2C36D1B51C74780126B3
:10BE6000002F62D0102F09D1302C07D120222B783F
:10BE70009343582B54D110276C7802352D4B390041
:10BE8000F31818000393FDF7BDFA04910121002374
:10BE9000494202008C4618002100303909291AD87D
:10BEA0000C00A74223DD591C09D06346824206D309
:10BEB00002D10499A14202DB0123784320182C7897
:10BEC0000135E9E72E00BCE72B2C01D01E00C7E7A7
:10BED000B51C7478FAE721004139192901D8373C9B
:10BEE000DFE721006139192901D8573CD9E75A1CED
:10BEF00008D1059A23331360029B0398002B09D1C4
:10BF000007B0F0BD002E00D04042029A002AF7D0C0
:10BF1000002B01D06B1E0193029B019A1A60EFE780
:10BF20003024002FAAD10827A8E7302C9ED00A275A
:10BF3000A4E7C046FFFFFF7F37B51300064A0500A0
:10BF40001068046A002C00D1044C0A0000942900F7
:10BF5000FFF770FF3EBDC04684000020E8000020CF
:10BF6000F8B505000E001400002804D08369002BEA
:10BF700001D100F0C1F9224B9C422DD16C68A3691C
:10BF8000A360A3891B0731D52369002B2ED023681A
:10BF90002269F7B2981A6369F6B2834205DC210080
:10BFA000280000F03BF9002826D1A3680130013BAE
:10BFB000A36023685A1C22601F706369834204D007
:10BFC000A389DB071AD50A2E18D12100280000F01A
:10BFD00025F9002812D00FE00A4B9C4201D1AC6831
:10BFE000CDE7094B9C42CAD1EC68C8E72100280084
:10BFF00000F00CF80028CAD0012676423000F8BDC7
:10C000004CE400006CE400002CE40000364B70B5FA
:10C010001D6806000C00002D05D0AB69002B02D175
:10C02000280000F069F9314B9C420FD16C680C2359
:10C03000E25E93B219072DD4D90611D40923012049
:10C04000336037331343A381404270BD284B9C4279
:10C0500001D1AC68EBE7274B9C42E8D1EC68E6E7FE
:10C060005B0713D5616B002908D023004433994244
:10C0700002D0300000F06AFA002363632422A3890F
:10C080009343A38100236360236923600823A2896B
:10C090001343A3812369002B0BD1A0218022A38904
:10C0A000890092000B40934203D02100300000F041
:10C0B000E1F90123A289134011D00023A360636931
:10C0C0005B42A361002023698342BED10C23E25E60
:10C0D0001306BAD540231343A3810138B5E792076D
:10C0E00000D46369A360EDE7840000204CE4000005
:10C0F0006CE400002CE4000010B5062000F090FC79
:10C10000012000F0CFFD0000F7B58A8905000C0082
:10C11000130760D44B68002B04DC0B6C002B01DC94
:10C120000020FEBDE76A002FFAD000232E682B60A6
:10C1300080235B01216A1A4034D0606DA3895B07BC
:10C1400006D56368C01A636B002B01D0236CC01A3C
:10C150000200216A00232800E76AB847A189431C2E
:10C1600006D12B681D2B30D82B4ADA40D3072CD5AB
:10C170000023636023692360CB0405D5431C02D1EF
:10C180002B68002B00D16065616B2E600029C7D041
:10C1900023004433994202D0280000F0D7F9002050
:10C1A0006063BEE701232800B847431CC6D12B6853
:10C1B000002BC3D01D2B01D0162B01D12E60AFE771
:10C1C0004023A2891343A381ABE740230B43012003
:10C1D000A3814042A5E70F69002FA1D00B680F6033
:10C1E000DB1B01930023920700D14B69A360019BE5
:10C1F000002B00DC94E7019B3A00216A2800A66A24
:10C20000B047002803DC4023A2891343DFE7019BEA
:10C210003F181B1A0193EAE7010040200B6970B533
:10C2200005000C00002B01D1002070BD002804D0B7
:10C230008369002B01D100F05FF80B4B9C4209D1C0
:10C240006C680C22A35E002BEED021002800FFF7C3
:10C250005BFFEAE7054B9C4201D1AC68F1E7044B78
:10C260009C42EED1EC68ECE74CE400006CE400008A
:10C270002CE40000002310B50400036043608360D9
:10C2800081814366C2810361436183611900082291
:10C290005C30FFF7FFF9054B24626362044BA36235
:10C2A000044BE362044B236310BDC04661CA000027
:10C2B00089CA0000C1CA0000EDCA000010B50249D9
:10C2C00000F08CF810BDC0461DC2000070B5682596
:10C2D0004A1E55430E002900743100F081F9041EF6
:10C2E00008D000212A00016046600C30A06068324E
:10C2F000FFF7D0F9200070BD836913B50400002B4F
:10C3000028D18364C3640365134B144A1B6882629B
:10C310000193984201D101238361200000F020F8AD
:10C320006060200000F01CF8A060200000F018F809
:10C330000022E06004216068FFF79CFF01220921D0
:10C34000A068FFF797FF02221221E068FFF792FF33
:10C350000123A36113BDC046F4E30000BDC2000089
:10C36000F8B51C4B07001E68B369002B02D13000E2
:10C37000FFF7C2FF4836B4687368013B04D53368E1
:10C38000002B07D03668F6E70C22A55E002D0DD0F5
:10C390006834F2E704213800FFF798FF3060002886
:10C3A000F0D10C2304003B602000F8BD20000A4BB4
:10C3B000656625606560A560E36025616561A561CE
:10C3C000082229005C30FFF765F96563A563A56461
:10C3D000E564E9E7F4E300000100FFFFF7B50400BE
:10C3E0000700002601914834002C01D13000FEBD29
:10C3F0006368A5680093009B013B009301D5246806
:10C40000F2E7AB89012B08D90E22AB5E013304D0D1
:10C4100029003800019B984706436835EBE7EC306C
:10C420000068704770B50E001D000E23C95E96B0FF
:10C430001400002907DA00232B60B3891B0611D4EE
:10C440008023DB000FE06A4600F088FB0028F2DB67
:10C45000F022019B12021340054A9B185A42534195
:10C460002B60EDE740230020236016B070BDC0466E
:10C4700000E0FFFFF7B502268B8905000C00334270
:10C4800006D0230047332360236101236361F7BD96
:10C4900001AB6A46FFF7C6FF00990700280000F0CD
:10C4A0009FF8002808D10C22A35E9A05EFD403223E
:10C4B00093431E43A681E4E70F4BAB628023A2891E
:10C4C00020601343A381009B20616361019B002BCB
:10C4D0000DD00E23E15E280000F052FB002806D0AC
:10C4E0000322A38993431A0001231343A381A08944
:10C4F0003843A081CBE7C046BDC2000010B5034B56
:10C500000100186800F06CF810BDC04684000020DF
:10C5100082B0002900D101A9101E06D0002B06D040
:10C5200013780B601078431E984102B070470220C8
:10C530004042FAE7C9B28218904201D10020704708
:10C5400003788B42FBD00130F6E7000070B50500A0
:10C55000002910D00C1F2368002B00DAE4182800F3
:10C5600000F034FB1D4A1368002B05D16360146092
:10C57000280000F02CFB70BDA34209D92168601887
:10C580008342F3D118685B6841182160EEE713001D
:10C590005A68002A01D0A242F9D919685818A04255
:10C5A0000BD120680918581819608242E0D1106830
:10C5B0005268411819605A60DAE7A04202D90C2388
:10C5C0002B60D5E721686018824203D11068526859
:10C5D0004118216062605C60CAE7C046301C0020E0
:10C5E000032370B5CD1C9D43083506000C2D1ED2CB
:10C5F0000C25A9421DD8300000F0E8FA254A14683D
:10C600002100002919D1244C2368002B03D13000CC
:10C6100000F0CAF920602900300000F0C5F9431C81
:10C620002BD10C233000336000F0D1FA03E0002D51
:10C63000DFDA0C233360002070BD0B685B1B19D45C
:10C640000B2B03D90B60CC18256003E04B688C42A0
:10C650000DD11360300000F0BAFA200007220B3031
:10C66000231D9043C31AE7D05A42E250E4E76360C7
:10C670000C00EFE70C004968C3E70323C41C9C438C
:10C68000A042E1D0211A300000F08EF9431CDBD12A
:10C69000C7E7C046301C0020341C0020F8B5070056
:10C6A0000D001600002905D11100FFF799FF0400C5
:10C6B0002000F8BD002A03D1FFF748FF3400F7E758
:10C6C00000F086FA2C00B042F2D231003800FFF7B9
:10C6D00087FF041EECD029003200FEF7BFFF2900BF
:10C6E0003800FFF733FFE3E7F0B58E6885B0070049
:10C6F0000C00039201939E423CD890238A89DB0070
:10C700001A4234D00325096923685B1A02936369CE
:10C7100002985D43EB0F5D19019B6D1001331B18EF
:10C72000AB4200D91D00530532D529003800FFF770
:10C7300057FF061E09D10C233B6040230120A2892C
:10C7400040421343A38105B0F0BD029A2169FEF770
:10C7500085FFA389144A1A4080231343A381029BB7
:10C760002661F61826606561019EED1AA560019BA1
:10C770009E4200D9019E320003992068FEF777FFA0
:10C78000A36800209B1BA36023689E192660DAE73C
:10C790002A003800FFF782FF061EE0D12169380029
:10C7A000FFF7D4FEC7E7C0467FFBFFFFF0B59FB0A1
:10C7B000029005938B890F0016001B0611D50B699B
:10C7C000002B0ED14021FFF70BFF386038610028A5
:10C7D00005D10C23029A013813601FB0F0BD40232D
:10C7E0007B61002306AC6361203363761033A3764C
:10C7F00035002B78002B01D0252B46D1AB1B0493A1
:10C800000CD0320039000298FFF76EFF431C00D1B4
:10C81000AEE06269049B9446634463612B78002B0D
:10C8200000D1A5E0012200235242626002A95432E5
:10C8300052186E1C2360E360A3601370A365317807
:10C8400005225448FFF776FE751C00281FD1226888
:10C85000D30604D5532302A95B18202119701307AE
:10C8600004D5532302A95B182B21197033782A2B86
:10C8700016D0350000210A20E3682A786E1C303A71
:10C88000092A4ED9002918D010E00135B1E7414BF3
:10C890002268C01A01238340134323602E00CEE791
:10C8A000059B191D1B680591002B01DB099304E012
:10C8B0005B42E3600223134323602B782E2B0AD1C3
:10C8C0006B782A2B35D1059B02351A1D1B68059202
:10C8D000002B2BDB0793304E297803223000FFF723
:10C8E00029FE002806D04023801B834022680135A2
:10C8F000134323602978062228486E1C2176FFF70F
:10C9000019FE00283CD0264B002B25D10722059B81
:10C9100007339343083305936369039A9B18636154
:10C9200066E7434301219B183500A6E701235B42DC
:10C93000D0E700230A201A000135636029786E1CB5
:10C940003039092903D9002BC5D00792C3E74243E8
:10C95000012352183500F1E705AB00933A00114B63
:10C960002100029800E000BF0390039B0133D3D164
:10C97000BB890B985B0600D42FE7012040422CE7CF
:10C9800005AB00933A00074B21000298FFF736F8F9
:10C99000EAE7C046F8E30000FEE3000002E400001E
:10C9A00000000000E9C60000002370B5064C050039
:10C9B0000800236000F060F9431C03D12368002BBA
:10C9C00000D02B6070BDC046C42F002070B504009D
:10C9D0000D001F2904D9162303600120404270BDB9
:10C9E000436C002B04D08A009B181A68002A08D1D7
:10C9F000200000F031F82A000100200000F01AF8B1
:10CA0000EDE70020012AEAD0511C03D116230130A2
:10CA10002360E4E7002428001C6090472000DEE744
:10CA200010B5034B01001868FFF7D0FF10BDC046DA
:10CA300084000020002370B5064C0500080011009A
:10CA4000236000F001F9431C03D12368002B00D0C0
:10CA50002B6070BDC42F002010B500F0E5F810BDAC
:10CA600070B50C000E25495F00F0BAF8002803DB12
:10CA7000636D1B18636570BDA389024A1340A381CF
:10CA8000F9E7C046FFEFFFFFF8B51F008B890500EF
:10CA90000C001600DB0505D50E23C95E002202231B
:10CAA00000F080F8A389054A28001340A3813200D2
:10CAB0000E23E15E3B0000F02BF8F8BDFFEFFFFF17
:10CAC00070B50C000E25495F00F06CF8A389421C7C
:10CAD00003D1054A1340A38170BD80225201134344
:10CAE000A3816065F8E7C046FFEFFFFF10B50E2396
:10CAF000C95E00F021F810BD0B1E04D0FF2A04D936
:10CB00008A2303608B3B180070470A700123FAE701
:10CB100070B50500080011000022064C22601A00C2
:10CB200000F0B8F8431C03D12368002B00D02B6021
:10CB300070BDC046C42F0020002370B5064C050010
:10CB40000800236000F060F8431C03D12368002B29
:10CB500000D02B6070BDC046C42F0020002370B5EC
:10CB6000064C050008001100236000F055F8431C36
:10CB700003D12368002B00D02B6070BDC42F002090
:10CB8000002370B5064C05000800236000F054F83F
:10CB9000431C03D12368002B00D02B6070BDC0461E
:10CBA000C42F002070B50500080011000022064CBB
:10CBB00022601A0000F050F8431C03D12368002BB8
:10CBC00000D02B6070BDC046C42F00207047704756
:10CBD0000B1F1B68181F002B01DA0B58C018704779
:10CBE00070B50500080011000022064C22601A00F2
:10CBF00000F03AF8431C03D12368002B00D02B60CF
:10CC000070BDC046C42F002058220120014B404275
:10CC10001A607047C42F002058220120014B404267
:10CC20001A607047C42F002058220120014B404257
:10CC30001A607047C42F00205822024B00201A604F
:10CC40007047C046C42F002058220120014B4042AB
:10CC50001A607047C42F002058220120014B404227
:10CC60001A607047C42F002058220120014B404217
:10CC70001A607047C42F0020044A1368002B00D1AB
:10CC8000034B1818106018007047C046381C00206D
:10CC9000C82F002058220120014B40421A607047E3
:10CCA000C42F0020FEE7C046F8B5C046F8BC08BC5B
:10CCB0009E467047F8B5C046F8BC08BC9E46704713
:10CCC000646174610000000044CD0000EF010000C9
:10CCD0004DCD0000E302000055CD00000509000025
:10CCE0005CCD0000150A000061CD00002D0500009C
:10CCF0006CCD00005303000071CD00006D0C0000EE
:10CD00007DCD00001F02000087CD00000D0800004F
:10CD100095CD0000B9060000A2CD0000EF04000090
:10CD200072616E646F6D00616C6C006C6173740095
:10CD300066616C7365007472756500252E313573FC
:10CD40002E2E2E006D616B654C69737400616464F6
:10CD50004C6173740064656C657465006A6F696E1C
:10CD600000636F707946726F6D546F0066696E6410
:10CD7000006A6F696E537472696E677300756E69CD
:10CD8000636F6465417400756E69636F64655374A5
:10CD900072696E67006E657742797465417272617F
:10CDA0007900667265654D656D6F727900000000EF
:10CDB00015CE0000D51000001ACE0000F3100000C0
:10CDC00055CD0000F710000020CE0000D910000063
:10CDD0002ACE0000FB10000033CE0000FF10000040
:10CDE0003DCE00000311000048CE000007110000F6
:10CDF00054CE0000DD1000005DCE0000EB100000FE
:10CE000067CE0000E110000072CE0000EF100000BD
:10CE100066696C65006F70656E00636C6F736500AA
:10CE2000656E644F6646696C6500726561644C6945
:10CE30006E6500726561644279746573006170703B
:10CE4000656E644C696E6500617070656E644279F0
:10CE50007465730066696C6553697A650073746103
:10CE600072744C697374006E657874496E4C6973A2
:10CE7000740073797374656D496E666F000000000D
:10CE8000381300004813000062130000E013000094
:10CE9000181400004E14000086140000AC140000AA
:10CEA000E81400002A15000080150000C4150000D9
:10CEB00030160000781600009E160000D6160000FE
:10CEC0001C17000042170000701700009E1700009A
:10CED000E0170000641800002C190000A2190000DF
:10CEE0000C1A0000581A0000781A00009A1A000064
:10CEF0004C1B0000921B00000A1C0000381C0000A4
:10CF0000681C00009E1C0000061D00008A1D000019
:10CF1000D01D0000181E00008E1E0000041F00001F
:10CF20004C1F0000921F0000C81F00000E200000D0
:10CF3000542000009C200000F82000004C2100003C
:10CF40008A210000F42100002A2200007222000041
:10CF5000BA220000022300003C23000084230000CA
:10CF6000CC2300003625000070170000D616000004
:10CF700034240000381300006A24000096240000C6
:10CF8000D4240000002500003813000038130000EE
:10CF90003813000038130000B0250000F22500000F
:10CFA0003826000088260000B42600000427000070
:10CFB0002A2700005827000038130000381300000B
:10CFC0007C270000AC270000DC27000012280000AE
:10CFD0003C280000A8280000D2280000FA28000001
:10CFE000222900005229000082290000AC290000FB
:10CFF000D6290000062A0000302A0000381300005D
:10D0000038130000381300003813000038130000F4
:10D01000602A00008C2A0000B82A0000E42A0000E0
:10D02000102B0000462B00007C2B0000B22B0000D0
:10D03000E82B0000142C0000402C0000762C00008F
:10D0400038130000381300003813000038130000B4
:10D0500038130000381300003813000038130000A4
:10D060003813000038130000381300003813000094
:10D070003813000038130000AC2C0000E22C000034
:10D080005B2564206974656D206C6973745D00288C
:10D0900025642062797465732900286F626A65636C
:10D0A0007420747970653A20256429005374616393
:10D0B0006B20756E646572666C6F7700626F6F6C63
:10D0C00065616E006E756D62657200737472696E73
:10D0D00067006C69737400627974652061727261B3
:10D0E0007900000007000000030000003ED10000AE
:10D0F000052E000046D10000B52E00004FD10000E3
:10D100005F2F000058D10000092E000061D10000FF
:10D11000632F000069D100004D2F000000000000C7
:10D1200001000000020000000300000004000000F5
:10D130000A0000006D6963726F3A62697400686189
:10D1400073546F6E6500706C6179546F6E65006822
:10D150006173536572766F00736574536572766F91
:10D1600000646163496E6974006461635772697435
:10D170006500474320746F6F6B20256420757365CD
:10D1800063733B206672656520256420776F726447
:10D1900073003C496E74656765723E003C4C697370
:10D1A000743E003C4F626A6563743E003C42797491
:10D1B0006541727261793E000D0A564D2050616ED4
:10D1C00069633A2025730D0A006D697363000000DE
:10D1D00005D200002D3C00000ED20000BD3B000037
:10D1E00012D20000113B00001AD20000B73A000032
:10D1F00024D200004D3A000030D200004F39000028
:10D200006E756C6C00686578546F496E7400736954
:10D210006E006A736F6E476574006A736F6E436F5A
:10D22000756E74006A736F6E56616C75654174003B
:10D230006A736F6E4B6579417400000098D20000EC
:10D24000993C0000A0D200009D3C0000AAD2000042
:10D25000BB3C0000B3D20000C53C0000BED20000C1
:10D26000CF3C0000CAD20000D93C0000DFD2000051
:10D27000E33C0000F4D20000ED3C000000D30000CD
:10D28000F73C000010D30000A73C00001CD30000B6
:10D29000B13C00006E6574006861735769466900AF
:10D2A0007374617274576946690073746F7057695B
:10D2B00046690077696669537461747573006D79A6
:10D2C0004950416464726573730068747470536587
:10D2D0007276657247657452657175657374007214
:10D2E0006573706F6E64546F4874747052657175B5
:10D2F0006573740068747470436F6E6E6563740058
:10D30000687474704973436F6E6E6563746564000E
:10D3100068747470526571756573740068747470A4
:10D32000526573706F6E7365001A1B1C0304060749
:10D33000090A171819000000000008080800080A68
:10D340004A4000000A5FEA5FEA0ED92ED36E193216
:10D350004489330C924C924D080800000004880860
:10D3600008040804848488000A448A4000048EC4A7
:10D3700080000000048800000EC0000000000800CB
:10D3800001224488100C9252524C048C84848E1CCE
:10D39000824C901E1EC244924C06CA525FE21FF09D
:10D3A0001EC13E02448ED12E1FE24488100ED12EA3
:10D3B000D12E0ED12EC4880008000800000480047D
:10D3C000880244880482000EC00EC008048244888B
:10D3D0000ED126C0040ED135B36C0C925ED2521C15
:10D3E000925C925C0ED010100E1C9252525C1ED0B9
:10D3F0001C901E1ED01C90100ED013712E12525E67
:10D40000D2521C8808081C1FE242524C1254981435
:10D4100092101010101E113B75B131113935B371D6
:10D420000C9252524C1C925C90100C92524C861CE6
:10D43000925C92510ED00C825C1FE4848484125260
:10D4400052524C1131312A44113135BB7112524CB8
:10D450009252112A4484841EC488101E0EC80808E3
:10D460000E10080482410EC242424E048A4000005F
:10D47000000000001F0804800000000ED2524F1070
:10D48000101C925C000ED0100E02424ED24E0C9236
:10D490005C900E06C81C88080ED24EC24C10101CA0
:10D4A00092520800080808024002424C10149814D6
:10D4B000920808080806001B75B131001C925252F0
:10D4C000000C92524C001C925C90000ED24EC20096
:10D4D0000ED010100006C8049808080EC8070012E5
:10D4E00052524F0011312A4400113135BB00124C09
:10D4F0008C9200112A4498001EC4881E06C48C8495
:10D5000086080808080818080C881800000C8360B2
:10D510000000000001000000020000000300000005
:10D5200004000000050000000600000007000000E5
:10D5300008000000090000000A0000000B000000C5
:10D540000C0000000D0000000E0000000F000000A5
:10D55000100000001200000014000000160000007F
:10D56000180000001A0000001C0000001E0000004F
:10D570002000000023000000260000002900000019
:10D580002C0000002F0000003200000036000000D8
:10D590003A0000003E00000042000000460000008B
:10D5A0004B00000050000000550000005A00000031
:10D5B00061000000680000006F00000076000000BD
:10D5C0007D000000840000008B000000920000003D
:10D5D00099000000A0000000A7000000AE000000BD
:10D5E000B5000000BC000000C3000000CA0000003D
:10D5F000D1000000D8000000DF000000E6000000BD
:10D60000ED000000F4000000FB000000FF0000003F
:10D6100060D60000193D00006BD60000B542000046
:10D6200075D60000DD3E000082D6000025410000D6
:10D6300089D600007541000092D60000C541000067
:10D640009ED60000BD400000AFD600004D3F000058
:10D65000BCD600004D400000646973706C617900B5
:10D660006C696768744C6576656C006D62446973BB
:10D67000706C6179006D62446973706C61794F669A
:10D6800066006D62506C6F74006D62556E706C6FE9
:10D6900074006D62447261775368617065006D62F9
:10D6A0005368617065466F724C6574746572006E84
:10D6B000656F506978656C53656E64006E656F5078
:10D6C0006978656C53657450696E004E6F7420659F
:10D6D0006E6F75676820726F6F6D206576656E205E
:10D6E000616674657220636F6D70616374696F6EDB
:10D6F00000436F6D70616374656420466C6173688C
:10D7000020636F64652073746F72650A25642062FC
:10D71000797465732075736564202825642525292F
:10D72000206F6620256400426164207265636F7219
:10D730006420666F756E6420647572696E67206917
:10D740006E697469616C697A6174696F6E002564D1
:10D750002025642025642028256420776F72647357
:10D7600029002564207265636F7264732C20256420
:10D7700020776F7264732C206D6178494420256492
:10D780002C20636F6D70616374696F6E20637963C1
:10D790006C657320256400526573746F7265642034
:10D7A00025642073637269707473005374617274BA
:10D7B000656400726164696F000000004CD800006D
:10D7C000854C000059D80000214F000069D80000A6
:10D7D000A14E000077D80000B550000082D80000AC
:10D7E000AD4C000092D80000354D0000A6D80000D6
:10D7F0001D4D0000B5D8000097520000C1D80000B0
:10D8000015520000CAD80000B9510000D5D8000058
:10D8100001510000E0D800003D510000E9D80000AF
:10D8200071510000F2D80000BD4C000001D9000089
:10D830009D4C00000AD90000CD4C00006E6F6E6553
:10D84000006F746865720070616972006469736169
:10D85000626C65526164696F006D657373616765C1
:10D860005265636569766564007061636B657452C7
:10D87000656365697665007061636B657453656E99
:10D8800064007265636569766564496E7465676591
:10D89000720072656365697665644D65737361676F
:10D8A0006554797065007265636569766564537463
:10D8B00072696E670073656E64496E746567657240
:10D8C0000073656E64506169720073656E645374B1
:10D8D00072696E67007365744368616E6E656C0093
:10D8E00073657447726F757000736574506F7765F8
:10D8F00072007369676E616C537472656E677468E9
:10D90000006465766963654944006C6173744D65B4
:10D910007373616765494400556E6B6E6F776E2057
:10D920007072696D6974697665205B25733A257339
:10D930005D00000000000000963007772C610EEEBD
:10D94000BA51099919C46D078FF46A7035A563E956
:10D95000A395649E3288DB0EA4B8DC791EE9D5E07D
:10D9600088D9D2972B4CB609BD7CB17E072DB8E77C
:10D97000911DBF906410B71DF220B06A4871B9F3D1
:10D98000DE41BE847DD4DA1AEBE4DD6D51B5D4F40A
:10D99000C785D38356986C13C0A86B647AF962FD6F
:10D9A000ECC9658A4F5C0114D96C0663633D0FFABC
:10D9B000F50D088DC8206E3B5E10694CE44160D5C2
:10D9C000727167A2D1E4033C47D4044BFD850DD2AC
:10D9D0006BB50AA5FAA8B5356C98B242D6C9BBDBBF
:10D9E00040F9BCACE36CD832755CDF45CF0DD6DCBA
:10D9F000593DD1ABAC30D9263A00DE518051D7C861
:10DA00001661D0BFB5F4B42123C4B3569995BACFEB
:10DA10000FA5BDB89EB802280888055FB2D90CC60C
:10DA200024E90BB1877C6F2F114C6858AB1D61C185
:10DA30003D2D66B69041DC760671DB01BC20D298A4
:10DA40002A10D5EF8985B1711FB5B606A5E4BF9F31
:10DA500033D4B8E8A2C9077834F9000F8EA8099624
:10DA600018980EE1BB0D6A7F2D3D6D08976C64918F
:10DA7000015C63E6F4516B6B62616C1CD8306585A8
:10DA80004E0062F2ED95066C7BA5011BC1F4088285
:10DA900057C40FF5C6D9B06550E9B712EAB8BE8BC6
:10DAA0007C88B9FCDF1DDD62492DDA15F37CD38C4F
:10DAB000654CD4FB5861B24DCE51B53A7400BCA34D
:10DAC000E230BBD441A5DF4AD795D83D6DC4D1A47F
:10DAD000FBF4D6D36AE96943FCD96E34468867AD56
:10DAE000D0B860DA732D0444E51D03335F4C0AAAF5
:10DAF000C97C0DDD3C710550AA41022710100BBEF8
:10DB000086200CC925B56857B3856F2009D466B93E
:10DB10009FE461CE0EF9DE5E98C9D9292298D0B073
:10DB2000B4A8D7C7173DB359810DB42E3B5CBDB720
:10DB3000AD6CBAC02083B8EDB6B3BF9A0CE2B603A1
:10DB40009AD2B1743947D5EAAF77D29D1526DB0456
:10DB50008316DC73120B63E3843B64943E6A6D0DA1
:10DB6000A85A6A7A0BCF0EE49DFF099327AE000AEC
:10DB7000B19E077D44930FF0D2A3088768F2011E7F
:10DB8000FEC206695D5762F7CB67658071366C1916
:10DB9000E7066B6E761BD4FEE02BD3895A7ADA1037
:10DBA000CC4ADD676FDFB9F9F9EFBE8E43BEB71718
:10DBB000D58EB060E8A3D6D67E93D1A1C4C2D838A2
:10DBC00052F2DF4FF167BBD16757BCA6DD06B53F08
:10DBD0004B36B248DA2B0DD84C1B0AAFF64A033647
:10DBE000607A0441C3EF60DF55DF67A8EF8E6E31C6
:10DBF00079BE69468CB361CB1A8366BCA0D26F250F
:10DC000036E2685295770CCC03470BBBB91602225B
:10DC10002F260555BE3BBAC5280BBDB2925AB42B70
:10DC2000046AB35CA7FFD7C231CFD0B58B9ED92C85
:10DC30001DAEDE5BB0C2649B26F263EC9CA36A75EA
:10DC40000A936D02A906099C3F360EEB85670772A1
:10DC500013570005824ABF95147AB8E2AE2BB17B08
:10DC6000381BB60C9B8ED2920DBED5E5B7EFDC7C8F
:10DC700021DFDB0BD4D2D38642E2D4F1F8B3DD68E6
:10DC80006E83DA1FCD16BE815B26B9F6E177B06FE1
:10DC90007747B718E65A0888706A0FFFCA3B0666CE
:10DCA0005C0B0111FF9E658F69AE62F8D3FF6B615B
:10DCB00045CF6C1678E20AA0EED20DD75483044EFD
:10DCC000C2B30339612667A7F71660D04D4769498B
:10DCD000DB776E3E4A6AD1AEDC5AD6D9660BDF409E
:10DCE000F03BD83753AEBCA9C59EBBDE7FCFB24751
:10DCF000E9FFB5301CF2BDBD8AC2BACA3093B35336
:10DD0000A6A3B4240536D0BA9306D7CD2957DE543E
:10DD1000BF67D9232E7A66B3B84A61C4021B685D17
:10DD2000942B6F2A37BE0BB4A18E0CC31BDF055A90
:10DD30008DEF022D416C6C207461736B73207374D2
:10DD40006F707065640076313036002025732025B1
:10DD500073004D656D6F727920636C6561726564E7
:10DD6000004E6F2066726565207461736B20656E6E
:10DD70007472696573000000D0DD00005966000010
:10DD8000DDDD0000F9610000E9DD0000296600002A
:10DD9000EFDD000039660000F5DD00004966000097
:10DDA000FBDD00002D62000005DE0000B56600000E
:10DDB0000DDE00000964000016DE0000896200002C
:10DDC0001EDE00002163000073656E736F727300C6
:10DDD000616363656C65726174696F6E0074656D13
:10DDE00070657261747572650074696C7458007442
:10DDF000696C74590074696C745A00746F75636847
:10DE0000526561640069326352656164006932631E
:10DE100057726974650072656164444854006D69A5
:10DE200063726F70686F6E6500000000A0DE000016
:10DE300041670000AEDE000045670000B7DE00006D
:10DE400051670000C1DE000055670000CADE000017
:10DE500059670000CFDE00005D670000D4DE0000DF
:10DE600061670000E0DE000065670000E7DE00009B
:10DE700069670000F0DE00006D670000F5DE00005D
:10DE80007167000000DF0000756700000ADF000016
:10DE90004967000014DF00004D67000074667400DD
:10DEA000656E61626C65446973706C617900676569
:10DEB0007457696474680067657448656967687455
:10DEC00000736574506978656C006C696E650072EA
:10DED00065637400726F756E646564526563740087
:10DEE000636972636C6500747269616E676C65006A
:10DEF0007465787400746674546F75636865640043
:10DF0000746674546F7563685800746674546F75E2
:10DF100063685900746674546F75636850726573F2
:10DF20007375726500766172730000004CDF00004B
:10DF3000056C000056DF0000E56B00005FDF0000AD
:10DF4000C16B00006BDF00004D6B00007661724515
:10DF50007869737473007661724E616D65640073E5
:10DF600065745661724E616D6564007661724E61D2
:10DF70006D65466F72496E6465780057656C636FB6
:10DF80006D6520746F204D6963726F426C6F636BB7
:10DF9000732100705F73706920213D204E554C4CF9
:10DFA000002F686F6D652F6769742F2E706C617418
:10DFB000666F726D696F2F7061636B616765732F38
:10DFC0006672616D65776F726B2D61726475696ED3
:10DFD0006F6E6F726469636E7266352F6C69627200
:10DFE00061726965732F5350492F5350492E6370E6
:10DFF0007000535049436C6173733A3A535049432C
:10E000006C617373284E52465F5350495F54797068
:10E01000652A2C2075696E74385F742C2075696EC2
:10E0200074385F742C2075696E74385F7429000031
:10E030000000000000000000116E0000CD6D000027
:10E04000F36D0000FD6D0000076E0000F16D000033
:10E0500003000000020000000100000004000000B6
:10E0600005000000110000000C0000000B00000083
:10E07000120000000A000000060000001A00000064
:10E08000140000001700000016000000150000003A
:10E0900010000000FFFFFFFFFFFFFFFF0000000078
:10E0A0001E0000001900000018000000070000001A
:10E0B00008000000090000000D0000000E00000034
:10E0C0000F0000001C0000001B0000001D000000ED
:10E0D000130000000000000000000000E9720000D2
:10E0E000517B0000697300007D73000073730000B2
:10E0F000E5720000D972000089730000057300000A
:10E10000D572000000000000000000000000304355
:10E1100000000000000030C3737172740000000042
:10E12000FB21F93FFB2109407CD91240FB2119401A
:10E130007A6A1F407CD92240BBFD2540FB21294043
:10E140003A462C407A6A2F405C4731407CD93240B5
:10E150009C6B3440BBFD3540DB8F3740FB213940A1
:10E160001BB43A403A463C405AD83D407A6A3F4058
:10E170004C7E40405C4741406C1042407CD942405C
:10E180008CA243409C6B4440AC344540BBFD4540B1
:10E19000CBC64640DB8F4740EB584840FB21494007
:10E1A00083F9A200444E6E00FC291500D1572700C8
:10E1B000DD34F50062DBC0003C99950041904300DE
:10E1C0006351FE00BBDEAB00B761C5003A6E2400B0
:10E1D000D24D42004906E00009EA2E001C92D1000F
:10E1E000EB1DFE0029B11C00E83EA700F5358200BA
:10E1F00044BB2E009CE98400B4267000417E5F0081
:10E20000D6913900538339009CF439008B5F840028
:10E2100028F9BD00F81F3B00DEFF97000F980500AE
:10E22000112FEF000A5A8B006D1F6D00CF7E360054
:10E2300009CB2700464FB7009E663F002DEA5F00DE
:10E24000BA277500E5EBC7003D7BF100F739070001
:10E2500092528A00FB6BEA001FB15F00085D8D00DF
:10E26000300356007BFC4600F0AB6B0020BCCF00B7
:10E2700036F49A00E3A91D005E619100081BE600D8
:10E2800085996500A0145F008D40680080D8FF006C
:10E2900027734D0006063100CA561500C9A8730041
:10E2A0007BE260006B8CC00000000040FB21F93F66
:10E2B000000000002D44743E000000809846F83CA9
:10E2C0000000006051CC783B00000080831BF039D7
:10E2D0000000004020257A38000000802282E336CA
:10E2E000000000001DF3693502000000030000007B
:10E2F0000400000006000000C897000072970000AC
:10E3000072970000A09800006E9700006E970000C2
:10E3100096980000A09800006E9700009698000064
:10E320006E970000A0980000A4980000A498000038
:10E33000A4980000AC980000A4A2000016A1000060
:10E340005AA10000BEA000005AA100004AA200008D
:10E350005AA10000BEA0000016A1000016A10000F6
:10E360004AA20000BEA00000B6A00000B6A00000B7
:10E37000B6A0000058A20000CCA90000CEA8000062
:10E38000CEA80000ECAB0000C8A80000C8A80000A0
:10E39000D4AB0000ECAB0000C8A80000D4AB000078
:10E3A000C8A80000ECAB0000E2AB0000E2AB00004C
:10E3B000E2AB0000F0AB00002C2066756E63746960
:10E3C0006F6E3A2000617373657274696F6E2022FC
:10E3D000257322206661696C65643A2066696C6504
:10E3E00020222573222C206C696E652025642573FC
:10E3F00025730A0088000020232D302B2000686C34
:10E400004C00656667454647003031323334353657
:10E410003738394142434445460030313233343590
:10E4200036373839616263646566000000000000B9
:10E4300000000000000000000000000000000000DC
:10E4400000000000000000000000000000000000CC
:10E4500000000000000000000000000000000000BC
:10E4600000000000000000000000000000000000AC
:10E47000000000000000000000000000000000009C
:10E480000000000000000000000000004300504FAA
:10E490005349580000202020202020202020282818
:10E4A0002828282020202020202020202020202054
:10E4B0002020202020881010101010101010101094
:10E4C00010101010100404040404040404040410C4
:10E4D0001010101010104141414141410101010152
:10E4E000010101010101010101010101010101011C
:10E4F0001010101010104242424242420202020228
:10E5000002020202020202020202020202020202EB
:10E51000101010102000000000000000000000009B
:10E5200000000000000000000000000000000000EB
:10E5300000000000000000000000000000000000DB
:10E5400000000000000000000000000000000000CB
:10E5500000000000000000000000000000000000BB
:10E5600000000000000000000000000000000000AB
:10E57000000000000000000000000000000000009B
:10E58000000000000000000000000000000000008B
:0CE590000000000000000000000000007F
:08E59C006C1BFF7F0100000071
:10E5A400FFFFFFFFD007000001000000E803DC05C7
:10E5B400DC05DC05DC050000FFFFFFFFFFFFFFFFBC
:10E5C4001800000019FCFFFFFFFFFFFFFF00000021
:10E5D4000024F4000200000003000000FFFFFFFF1E
:10E5E4000000000001000000000002000100000023
:10E5F400FFFFFFFF00000000020000000000040015
:10E6040002000000FFFFFFFF000000000300000005
:10E6140000000800030000000A00000008000000D9
:10E624000100000088000020000000004CE400000D
:10E634006CE400002CE40000000000000000000076
:10E6440000000000000000000000000000000000C6
:10E6540000000000000000000000000000000000B6
:10E6640000000000000000000000000000000000A6
:10E674000000000000000000000000000000000096
:10E684000000000000000000430000000000000043
:10E694000000000000000000000000000000000076
:10E6A4000000000000000000430000000000000023
:10E6B4000000000000000000000000000000000056
:10E6C4000000000000000000430000000000000003
:10E6D4000000000000000000000000000000000036
:10E6E40000000000000000004300000000000000E3
:10E6F4000000000000000000000000000000000016
:10E7040000000000000000004300000000000000C2
:10E7140000000000000000000000000000000000F5
:10E7240000000000000000004300000000000000A2
:10E7340000000000000000000000000000000000D5
:10E744000000000000000000430000000000000082
:10E7540000000000000000000000000000000000B5
:10E764000000000000000000F9CA000011C500000C
:10E774000000000094E4000042CD0000C8D1000075
:10E78400C8D10000C8D10000C8D10000C8D1000021
:10E79400C8D10000C8D10000C8D10000C8D1000011
:10E7A400FFFFFFFFFFFFFFFFFFFFFFFFFFFF000073
:10E7B40001004153434949000000000000000000EB
:10E7C4000000000000000000000000000000000045
:10E7D40000004153434949000000000000000000CC
:10E7E4000000000000000000000000000000000025
:10E7F40000000000E90000009D6D00000D710000A4
:08E8040035760000C1000000A0
:04000003000071A9DF
:00000001FF
